Component: ARM Compiler 5.06 update 7 (build 960) Tool: armlink [4d3601]

==============================================================================

Section Cross References

    gpio.o(i.GPIO_Init) refers to gpio.o(i.PORT_Init) for PORT_Init
    gpio.o(i.GPIO_Init) refers to gpio.o(i.PORT_ClrBit) for PORT_ClrBit
    gpio.o(i.GPIO_Init) refers to gpio.o(i.PORT_SetBit) for PORT_SetBit
    gpio.o(i.PORT_Init) refers to gpio.o(i.__ARM_common_switch8) for __ARM_common_switch8
    sys_tick.o(i.SysTick_Handler) refers to sys_tick.o(.bss) for pfnSysTickCallBack
    sys_tick.o(i.SysTick_Handler) refers to sys_tick.o(.data) for g_u16SysRollingCounter1ms
    sys_tick.o(i.Sys_Tick_Timer_Call_Back_Reg) refers to sys_tick.o(.bss) for pfnSysTickCallBack
    sys_tick.o(i.Sys_Tick_Timer_Start) refers to system_bat32g137.o(i.SystemCoreClockUpdate) for SystemCoreClockUpdate
    sys_tick.o(i.Sys_Tick_Timer_Start) refers to aeabi_sdiv.o(.text) for __aeabi_uidivmod
    sys_tick.o(i.Sys_Tick_Timer_Start) refers to sys_tick.o(i.__NVIC_SetPriority) for __NVIC_SetPriority
    sys_tick.o(i.Sys_Tick_Timer_Start) refers to sys_tick.o(.bss) for g_stSysTickTimer
    sys_tick.o(i.Sys_Tick_Timer_Start) refers to sys_tick.o(.data) for g_u16SysRollingCounter50us
    sys_tick.o(i.Sys_Tick_Timer_Start) refers to system_bat32g137.o(.data) for SystemCoreClock
    adc.o(i.ADC_Converse) refers to adc.o(i.INTC_DisableIRQ) for INTC_DisableIRQ
    adc.o(i.ADC_Converse) refers to adc.o(i.INTC_GetPendingIRQ) for INTC_GetPendingIRQ
    adc.o(i.ADC_Converse) refers to adc.o(i.INTC_ClearPendingIRQ) for INTC_ClearPendingIRQ
    adc.o(i.ADC_Converse) refers to aeabi_sdiv.o(.text) for __aeabi_uidivmod
    adc.o(i.ADC_Get_Conversion_Result) refers to adc.o(.data) for u8ADCSequenceRunningFlag
    adc.o(i.ADC_Get_Conversion_Status) refers to adc.o(.data) for u8ADCSequenceRunningFlag
    adc.o(i.ADC_Init) refers to adc.o(i.INTC_DisableIRQ) for INTC_DisableIRQ
    adc.o(i.ADC_Init) refers to adc.o(i.INTC_ClearPendingIRQ) for INTC_ClearPendingIRQ
    adc.o(i.ADC_Init) refers to adc.o(i.__NVIC_ClearPendingIRQ) for __NVIC_ClearPendingIRQ
    adc.o(i.ADC_MidAvg_Filter) refers to aeabi_sdiv.o(.text) for __aeabi_uidivmod
    adc.o(i.ADC_SelfTest) refers to adc.o(i.INTC_DisableIRQ) for INTC_DisableIRQ
    adc.o(i.ADC_SelfTest) refers to aeabi_sdiv.o(.text) for __aeabi_uidivmod
    adc.o(i.ADC_SelfTest) refers to adc.o(i.INTC_GetPendingIRQ) for INTC_GetPendingIRQ
    adc.o(i.ADC_SelfTest) refers to adc.o(i.INTC_ClearPendingIRQ) for INTC_ClearPendingIRQ
    adc.o(i.ADC_Start) refers to adc.o(i.INTC_ClearPendingIRQ) for INTC_ClearPendingIRQ
    adc.o(i.ADC_Start) refers to adc.o(i.__NVIC_ClearPendingIRQ) for __NVIC_ClearPendingIRQ
    adc.o(i.ADC_Start_Conversion) refers to adc.o(i.ADC_Start) for ADC_Start
    adc.o(i.ADC_Start_Conversion) refers to adc.o(.data) for u8ADCChannelCount
    adc.o(i.ADC_Start_Conversion) refers to analog_signals.o(.constdata) for u8ADCChList
    adc.o(i.ADC_Stop) refers to adc.o(i.INTC_DisableIRQ) for INTC_DisableIRQ
    adc.o(i.ADC_Stop) refers to adc.o(i.INTC_ClearPendingIRQ) for INTC_ClearPendingIRQ
    adc.o(i.ADC_Stop) refers to adc.o(i.__NVIC_ClearPendingIRQ) for __NVIC_ClearPendingIRQ
    adc.o(i.ADC_Stop_Conversion) refers to adc.o(i.ADC_Stop) for ADC_Stop
    adc.o(i.Analog_Signal_Conv_Real_Time_Run) refers to adc.o(i.ADC_Start) for ADC_Start
    adc.o(i.Analog_Signal_Conv_Real_Time_Run) refers to adc.o(.data) for u8ADCChannelCount
    adc.o(i.Analog_Signal_Conv_Real_Time_Run) refers to analog_signals.o(.constdata) for u8ADCChList
    analog_circuits.o(i.ADC_Input_Voltage_Calc) refers to aeabi_sdiv.o(.text) for __aeabi_uidivmod
    analog_circuits.o(i.ADC_Res_Calc_Circuit101) refers to llmul.o(.text) for __aeabi_lmul
    analog_circuits.o(i.ADC_Res_Calc_Circuit101) refers to lludiv.o(.text) for __aeabi_uldivmod
    analog_circuits.o(i.ADC_Res_Calc_Circuit101) refers to aeabi_sdiv.o(.text) for __aeabi_uidivmod
    analog_circuits.o(i.ADC_Res_Calc_Circuit102) refers to llmul.o(.text) for __aeabi_lmul
    analog_circuits.o(i.ADC_Res_Calc_Circuit102) refers to lludiv.o(.text) for __aeabi_uldivmod
    analog_circuits.o(i.ADC_Res_Calc_Circuit102) refers to aeabi_sdiv.o(.text) for __aeabi_uidivmod
    analog_circuits.o(i.ADC_Res_Calc_Circuit103) refers to llmul.o(.text) for __aeabi_lmul
    analog_circuits.o(i.ADC_Res_Calc_Circuit103) refers to lludiv.o(.text) for __aeabi_uldivmod
    analog_circuits.o(i.ADC_Res_Calc_Circuit103) refers to aeabi_sdiv.o(.text) for __aeabi_uidivmod
    analog_circuits.o(i.ADC_Res_Calc_Circuit201) refers to llmul.o(.text) for __aeabi_lmul
    analog_circuits.o(i.ADC_Res_Calc_Circuit201) refers to lludiv.o(.text) for __aeabi_uldivmod
    analog_circuits.o(i.ADC_Res_Calc_Circuit201) refers to aeabi_sdiv.o(.text) for __aeabi_uidivmod
    analog_circuits.o(i.ADC_Res_Calc_Circuit202) refers to llmul.o(.text) for __aeabi_lmul
    analog_circuits.o(i.ADC_Res_Calc_Circuit202) refers to lludiv.o(.text) for __aeabi_uldivmod
    analog_circuits.o(i.ADC_Res_Calc_Circuit202) refers to aeabi_sdiv.o(.text) for __aeabi_uidivmod
    analog_circuits.o(i.ADC_Res_Calc_Circuit203) refers to llmul.o(.text) for __aeabi_lmul
    analog_circuits.o(i.ADC_Res_Calc_Circuit203) refers to lludiv.o(.text) for __aeabi_uldivmod
    analog_circuits.o(i.ADC_Res_Calc_Circuit203) refers to aeabi_sdiv.o(.text) for __aeabi_uidivmod
    analog_circuits.o(i.ADC_Res_Calc_Circuit301) refers to aeabi_sdiv.o(.text) for __aeabi_uidivmod
    analog_circuits.o(i.ADC_Res_Calc_Circuit302) refers to aeabi_sdiv.o(.text) for __aeabi_uidivmod
    analog_circuits.o(i.ADC_Res_Calc_Circuit303) refers to llmul.o(.text) for __aeabi_lmul
    analog_circuits.o(i.ADC_Res_Calc_Circuit303) refers to lludiv.o(.text) for __aeabi_uldivmod
    analog_circuits.o(i.ADC_Res_Calc_Circuit303) refers to aeabi_sdiv.o(.text) for __aeabi_uidivmod
    analog_circuits.o(i.ADC_VRef_Calibrate) refers to aeabi_sdiv.o(.text) for __aeabi_uidivmod
    analog_circuits.o(i.ADC_Voltage_Calc_Circuit101) refers to aeabi_sdiv.o(.text) for __aeabi_idivmod
    analog_circuits.o(i.ADC_Voltage_Calc_Circuit102) refers to llmul.o(.text) for __aeabi_lmul
    analog_circuits.o(i.ADC_Voltage_Calc_Circuit102) refers to lludiv.o(.text) for __aeabi_uldivmod
    analog_signals.o(i.ADC_Conv_Single_Channel) refers to adc.o(i.ADC_Get_Conversion_Status) for ADC_Get_Conversion_Status
    analog_signals.o(i.ADC_Conv_Single_Channel) refers to adc.o(i.ADC_Start_Conversion) for ADC_Start_Conversion
    analog_signals.o(i.ADC_Conv_Single_Channel) refers to adc.o(i.ADC_Get_Conversion_Result) for ADC_Get_Conversion_Result
    analog_signals.o(i.ADC_Conv_Single_Channel) refers to analog_circuits.o(i.ADC_Input_Voltage_Calc) for ADC_Input_Voltage_Calc
    analog_signals.o(i.ADC_Conv_Single_Channel) refers to analog_circuits.o(i.ADC_Data_Calibrate) for ADC_Data_Calibrate
    analog_signals.o(i.ADC_Conv_Single_Channel) refers to analog_signals.o(.data) for u16ADCSample
    analog_signals.o(i.ADC_Conv_Single_Channel) refers to analog_signals.o(.constdata) for stADCChCfg
    analog_signals.o(i.ADC_Read_Signal) refers to analog_signals.o(.bss) for stADCData
    analog_signals.o(i.ADC_Read_Signal_Valid) refers to analog_signals.o(.bss) for stADCData
    analog_signals.o(i.Analog_Signal_Conv_Init) refers to adc.o(i.ADC_Stop_Conversion) for ADC_Stop_Conversion
    analog_signals.o(i.Analog_Signal_Conv_Init) refers to adc.o(i.ADC_Get_Conversion_Status) for ADC_Get_Conversion_Status
    analog_signals.o(i.Analog_Signal_Conv_Init) refers to adc.o(i.ADC_Init) for ADC_Init
    analog_signals.o(i.Analog_Signal_Conv_Init) refers to analog_signals.o(.bss) for stADCData
    analog_signals.o(i.Analog_Signal_Conv_Init) refers to analog_signals.o(.data) for stADCCtrl
    analog_signals.o(i.Analog_Signal_Conv_Init) refers to adc.o(.data) for u8ADCSequenceRunningFlag
    analog_signals.o(i.Analog_Signal_Conv_Service) refers to gpio.o(i.__ARM_common_switch8) for __ARM_common_switch8
    analog_signals.o(i.Analog_Signal_Conv_Service) refers to adc.o(i.ADC_Start_Conversion) for ADC_Start_Conversion
    analog_signals.o(i.Analog_Signal_Conv_Service) refers to adc.o(i.ADC_Get_Conversion_Status) for ADC_Get_Conversion_Status
    analog_signals.o(i.Analog_Signal_Conv_Service) refers to adc.o(i.ADC_Stop_Conversion) for ADC_Stop_Conversion
    analog_signals.o(i.Analog_Signal_Conv_Service) refers to adc.o(i.ADC_Get_Conversion_Result) for ADC_Get_Conversion_Result
    analog_signals.o(i.Analog_Signal_Conv_Service) refers to analog_circuits.o(i.ADC_Input_Voltage_Calc) for ADC_Input_Voltage_Calc
    analog_signals.o(i.Analog_Signal_Conv_Service) refers to analog_signals.o(i.ADC_Read_Signal) for ADC_Read_Signal
    analog_signals.o(i.Analog_Signal_Conv_Service) refers to analog_signals.o(i.ADC_Read_Signal_Valid) for ADC_Read_Signal_Valid
    analog_signals.o(i.Analog_Signal_Conv_Service) refers to analog_circuits.o(i.ADC_Data_Calibrate) for ADC_Data_Calibrate
    analog_signals.o(i.Analog_Signal_Conv_Service) refers to analog_signals.o(i.Analog_Signal_Conv_Init) for Analog_Signal_Conv_Init
    analog_signals.o(i.Analog_Signal_Conv_Service) refers to analog_signals.o(.data) for stADCCtrl
    analog_signals.o(i.Analog_Signal_Conv_Service) refers to analog_signals.o(.constdata) for stADCChCfg
    analog_signals.o(i.Analog_Signal_Conv_Service) refers to analog_signals.o(.bss) for stADCData
    analog_signals.o(i.Analog_Signal_Conv_Stop) refers to adc.o(i.ADC_Stop) for ADC_Stop
    analog_signals.o(i.Analog_Signal_Conv_Stop) refers to analog_signals.o(.bss) for stADCData
    analog_signals.o(i.Analog_Signal_Conv_Stop) refers to analog_signals.o(.data) for stADCCtrl
    analog_signals.o(.constdata) refers to analog_circuits.o(i.ADC_Voltage_Calc_Circuit102) for ADC_Voltage_Calc_Circuit102
    sci.o(i.IIC00_MasterReceive) refers to sci.o(i.IIC00_StartCondition) for IIC00_StartCondition
    sci.o(i.IIC00_MasterReceive) refers to sci.o(i.INTC_ClearPendingIRQ) for INTC_ClearPendingIRQ
    sci.o(i.IIC00_MasterReceive) refers to sci.o(i.__NVIC_ClearPendingIRQ) for __NVIC_ClearPendingIRQ
    sci.o(i.IIC00_MasterReceive) refers to sci.o(i.INTC_EnableIRQ) for INTC_EnableIRQ
    sci.o(i.IIC00_MasterReceive) refers to sci.o(i.__NVIC_SetPriority) for __NVIC_SetPriority
    sci.o(i.IIC00_MasterReceive) refers to sci.o(.data) for g_iic00_master_status_flag
    sci.o(i.IIC00_MasterSend) refers to sci.o(i.IIC00_StartCondition) for IIC00_StartCondition
    sci.o(i.IIC00_MasterSend) refers to sci.o(i.INTC_ClearPendingIRQ) for INTC_ClearPendingIRQ
    sci.o(i.IIC00_MasterSend) refers to sci.o(i.__NVIC_ClearPendingIRQ) for __NVIC_ClearPendingIRQ
    sci.o(i.IIC00_MasterSend) refers to sci.o(i.INTC_EnableIRQ) for INTC_EnableIRQ
    sci.o(i.IIC00_MasterSend) refers to sci.o(i.__NVIC_SetPriority) for __NVIC_SetPriority
    sci.o(i.IIC00_MasterSend) refers to sci.o(.data) for g_iic00_master_status_flag
    sci.o(i.IIC00_Stop) refers to sci.o(i.INTC_DisableIRQ) for INTC_DisableIRQ
    sci.o(i.IIC00_Stop) refers to sci.o(i.INTC_ClearPendingIRQ) for INTC_ClearPendingIRQ
    sci.o(i.IIC00_StopCondition) refers to sci.o(.data) for g_iic00_master_status_flag
    sci.o(i.IIC01_MasterReceive) refers to sci.o(i.IIC01_StartCondition) for IIC01_StartCondition
    sci.o(i.IIC01_MasterReceive) refers to sci.o(i.INTC_ClearPendingIRQ) for INTC_ClearPendingIRQ
    sci.o(i.IIC01_MasterReceive) refers to sci.o(i.__NVIC_ClearPendingIRQ) for __NVIC_ClearPendingIRQ
    sci.o(i.IIC01_MasterReceive) refers to sci.o(i.INTC_EnableIRQ) for INTC_EnableIRQ
    sci.o(i.IIC01_MasterReceive) refers to sci.o(.data) for g_iic01_master_status_flag
    sci.o(i.IIC01_MasterSend) refers to sci.o(i.IIC01_StartCondition) for IIC01_StartCondition
    sci.o(i.IIC01_MasterSend) refers to sci.o(i.INTC_ClearPendingIRQ) for INTC_ClearPendingIRQ
    sci.o(i.IIC01_MasterSend) refers to sci.o(i.__NVIC_ClearPendingIRQ) for __NVIC_ClearPendingIRQ
    sci.o(i.IIC01_MasterSend) refers to sci.o(i.INTC_EnableIRQ) for INTC_EnableIRQ
    sci.o(i.IIC01_MasterSend) refers to sci.o(.data) for g_iic01_master_status_flag
    sci.o(i.IIC01_Stop) refers to sci.o(i.INTC_DisableIRQ) for INTC_DisableIRQ
    sci.o(i.IIC01_Stop) refers to sci.o(i.INTC_ClearPendingIRQ) for INTC_ClearPendingIRQ
    sci.o(i.IIC10_MasterReceive) refers to sci.o(i.IIC10_StartCondition) for IIC10_StartCondition
    sci.o(i.IIC10_MasterReceive) refers to sci.o(i.INTC_ClearPendingIRQ) for INTC_ClearPendingIRQ
    sci.o(i.IIC10_MasterReceive) refers to sci.o(i.__NVIC_ClearPendingIRQ) for __NVIC_ClearPendingIRQ
    sci.o(i.IIC10_MasterReceive) refers to sci.o(i.INTC_EnableIRQ) for INTC_EnableIRQ
    sci.o(i.IIC10_MasterReceive) refers to sci.o(i.__NVIC_SetPriority) for __NVIC_SetPriority
    sci.o(i.IIC10_MasterReceive) refers to sci.o(.data) for g_iic10_master_status_flag
    sci.o(i.IIC10_MasterSend) refers to sci.o(i.IIC10_StartCondition) for IIC10_StartCondition
    sci.o(i.IIC10_MasterSend) refers to sci.o(i.INTC_ClearPendingIRQ) for INTC_ClearPendingIRQ
    sci.o(i.IIC10_MasterSend) refers to sci.o(i.__NVIC_ClearPendingIRQ) for __NVIC_ClearPendingIRQ
    sci.o(i.IIC10_MasterSend) refers to sci.o(i.INTC_EnableIRQ) for INTC_EnableIRQ
    sci.o(i.IIC10_MasterSend) refers to sci.o(i.__NVIC_SetPriority) for __NVIC_SetPriority
    sci.o(i.IIC10_MasterSend) refers to sci.o(.data) for g_iic10_master_status_flag
    sci.o(i.IIC10_Stop) refers to sci.o(i.INTC_DisableIRQ) for INTC_DisableIRQ
    sci.o(i.IIC10_Stop) refers to sci.o(i.INTC_ClearPendingIRQ) for INTC_ClearPendingIRQ
    sci.o(i.IIC10_StopCondition) refers to sci.o(.data) for g_iic10_master_status_flag
    sci.o(i.IIC11_MasterReceive) refers to sci.o(i.IIC11_StartCondition) for IIC11_StartCondition
    sci.o(i.IIC11_MasterReceive) refers to sci.o(i.INTC_ClearPendingIRQ) for INTC_ClearPendingIRQ
    sci.o(i.IIC11_MasterReceive) refers to sci.o(i.__NVIC_ClearPendingIRQ) for __NVIC_ClearPendingIRQ
    sci.o(i.IIC11_MasterReceive) refers to sci.o(i.INTC_EnableIRQ) for INTC_EnableIRQ
    sci.o(i.IIC11_MasterReceive) refers to sci.o(.data) for g_iic11_master_status_flag
    sci.o(i.IIC11_MasterSend) refers to sci.o(i.IIC11_StartCondition) for IIC11_StartCondition
    sci.o(i.IIC11_MasterSend) refers to sci.o(i.INTC_ClearPendingIRQ) for INTC_ClearPendingIRQ
    sci.o(i.IIC11_MasterSend) refers to sci.o(i.__NVIC_ClearPendingIRQ) for __NVIC_ClearPendingIRQ
    sci.o(i.IIC11_MasterSend) refers to sci.o(i.INTC_EnableIRQ) for INTC_EnableIRQ
    sci.o(i.IIC11_MasterSend) refers to sci.o(.data) for g_iic11_master_status_flag
    sci.o(i.IIC11_Stop) refers to sci.o(i.INTC_DisableIRQ) for INTC_DisableIRQ
    sci.o(i.IIC11_Stop) refers to sci.o(i.INTC_ClearPendingIRQ) for INTC_ClearPendingIRQ
    sci.o(i.IIC20_MasterReceive) refers to sci.o(i.IIC20_StartCondition) for IIC20_StartCondition
    sci.o(i.IIC20_MasterReceive) refers to sci.o(i.INTC_ClearPendingIRQ) for INTC_ClearPendingIRQ
    sci.o(i.IIC20_MasterReceive) refers to sci.o(i.__NVIC_ClearPendingIRQ) for __NVIC_ClearPendingIRQ
    sci.o(i.IIC20_MasterReceive) refers to sci.o(i.INTC_EnableIRQ) for INTC_EnableIRQ
    sci.o(i.IIC20_MasterReceive) refers to sci.o(i.__NVIC_SetPriority) for __NVIC_SetPriority
    sci.o(i.IIC20_MasterReceive) refers to sci.o(.data) for g_iic20_master_status_flag
    sci.o(i.IIC20_MasterSend) refers to sci.o(i.IIC20_StartCondition) for IIC20_StartCondition
    sci.o(i.IIC20_MasterSend) refers to sci.o(i.INTC_ClearPendingIRQ) for INTC_ClearPendingIRQ
    sci.o(i.IIC20_MasterSend) refers to sci.o(i.__NVIC_ClearPendingIRQ) for __NVIC_ClearPendingIRQ
    sci.o(i.IIC20_MasterSend) refers to sci.o(i.INTC_EnableIRQ) for INTC_EnableIRQ
    sci.o(i.IIC20_MasterSend) refers to sci.o(i.__NVIC_SetPriority) for __NVIC_SetPriority
    sci.o(i.IIC20_MasterSend) refers to sci.o(.data) for g_iic20_master_status_flag
    sci.o(i.IIC20_Stop) refers to sci.o(i.INTC_DisableIRQ) for INTC_DisableIRQ
    sci.o(i.IIC20_Stop) refers to sci.o(i.INTC_ClearPendingIRQ) for INTC_ClearPendingIRQ
    sci.o(i.IIC20_StopCondition) refers to sci.o(.data) for g_iic20_master_status_flag
    sci.o(i.IIC21_MasterReceive) refers to sci.o(i.IIC21_StartCondition) for IIC21_StartCondition
    sci.o(i.IIC21_MasterReceive) refers to sci.o(i.INTC_ClearPendingIRQ) for INTC_ClearPendingIRQ
    sci.o(i.IIC21_MasterReceive) refers to sci.o(i.__NVIC_ClearPendingIRQ) for __NVIC_ClearPendingIRQ
    sci.o(i.IIC21_MasterReceive) refers to sci.o(i.INTC_EnableIRQ) for INTC_EnableIRQ
    sci.o(i.IIC21_MasterReceive) refers to sci.o(.data) for g_iic21_master_status_flag
    sci.o(i.IIC21_MasterSend) refers to sci.o(i.IIC21_StartCondition) for IIC21_StartCondition
    sci.o(i.IIC21_MasterSend) refers to sci.o(i.INTC_ClearPendingIRQ) for INTC_ClearPendingIRQ
    sci.o(i.IIC21_MasterSend) refers to sci.o(i.__NVIC_ClearPendingIRQ) for __NVIC_ClearPendingIRQ
    sci.o(i.IIC21_MasterSend) refers to sci.o(i.INTC_EnableIRQ) for INTC_EnableIRQ
    sci.o(i.IIC21_MasterSend) refers to sci.o(.data) for g_iic21_master_status_flag
    sci.o(i.IIC21_Stop) refers to sci.o(i.INTC_DisableIRQ) for INTC_DisableIRQ
    sci.o(i.IIC21_Stop) refers to sci.o(i.INTC_ClearPendingIRQ) for INTC_ClearPendingIRQ
    sci.o(i.SPI00_MasterReceive) refers to sci.o(i.SPI00_Start) for SPI00_Start
    sci.o(i.SPI00_MasterReceive) refers to sci.o(.data) for dummy_sio00
    sci.o(i.SPI00_MasterSend) refers to sci.o(i.SPI00_Start) for SPI00_Start
    sci.o(i.SPI00_MasterSend) refers to sci.o(.data) for g_spi00_tx_count
    sci.o(i.SPI00_MasterSendReceive) refers to sci.o(i.SPI00_Start) for SPI00_Start
    sci.o(i.SPI00_MasterSendReceive) refers to sci.o(.data) for g_spi00_rx_count
    sci.o(i.SPI00_SlaveReceive) refers to sci.o(i.SPI00_Start) for SPI00_Start
    sci.o(i.SPI00_SlaveReceive) refers to sci.o(.data) for g_spi00_rx_count
    sci.o(i.SPI00_SlaveSend) refers to sci.o(i.SPI00_Start) for SPI00_Start
    sci.o(i.SPI00_SlaveSend) refers to sci.o(.data) for g_spi00_tx_count
    sci.o(i.SPI00_Start) refers to sci.o(i.INTC_ClearPendingIRQ) for INTC_ClearPendingIRQ
    sci.o(i.SPI00_Start) refers to sci.o(i.__NVIC_ClearPendingIRQ) for __NVIC_ClearPendingIRQ
    sci.o(i.SPI00_Start) refers to sci.o(i.INTC_EnableIRQ) for INTC_EnableIRQ
    sci.o(i.SPI00_Stop) refers to sci.o(i.INTC_DisableIRQ) for INTC_DisableIRQ
    sci.o(i.SPI00_Stop) refers to sci.o(i.INTC_ClearPendingIRQ) for INTC_ClearPendingIRQ
    sci.o(i.SPI01_MasterReceive) refers to sci.o(i.SPI01_Start) for SPI01_Start
    sci.o(i.SPI01_MasterReceive) refers to sci.o(.data) for g_spi01_rx_count
    sci.o(i.SPI01_MasterSend) refers to sci.o(i.SPI01_Start) for SPI01_Start
    sci.o(i.SPI01_MasterSend) refers to sci.o(.data) for g_spi01_tx_count
    sci.o(i.SPI01_SlaveInit) refers to sci.o(i.__NVIC_SetPriority) for __NVIC_SetPriority
    sci.o(i.SPI01_SlaveReceive) refers to sci.o(i.SPI01_Start) for SPI01_Start
    sci.o(i.SPI01_SlaveReceive) refers to sci.o(.data) for g_spi01_rx_count
    sci.o(i.SPI01_SlaveSend) refers to sci.o(i.SPI01_Start) for SPI01_Start
    sci.o(i.SPI01_SlaveSend) refers to sci.o(.data) for g_spi01_tx_count
    sci.o(i.SPI01_SlaveSendReceive) refers to sci.o(i.SPI01_Start) for SPI01_Start
    sci.o(i.SPI01_SlaveSendReceive) refers to sci.o(.data) for g_spi01_rx_count
    sci.o(i.SPI01_Start) refers to sci.o(i.INTC_ClearPendingIRQ) for INTC_ClearPendingIRQ
    sci.o(i.SPI01_Start) refers to sci.o(i.__NVIC_ClearPendingIRQ) for __NVIC_ClearPendingIRQ
    sci.o(i.SPI01_Start) refers to sci.o(i.INTC_EnableIRQ) for INTC_EnableIRQ
    sci.o(i.SPI01_Stop) refers to sci.o(i.INTC_DisableIRQ) for INTC_DisableIRQ
    sci.o(i.SPI01_Stop) refers to sci.o(i.INTC_ClearPendingIRQ) for INTC_ClearPendingIRQ
    sci.o(i.SPI01_Stop) refers to sci.o(i.__NVIC_ClearPendingIRQ) for __NVIC_ClearPendingIRQ
    sci.o(i.SPI10_MasterReceive) refers to sci.o(i.SPI10_Start) for SPI10_Start
    sci.o(i.SPI10_MasterReceive) refers to sci.o(.data) for dummy_sio10
    sci.o(i.SPI10_MasterSend) refers to sci.o(i.SPI10_Start) for SPI10_Start
    sci.o(i.SPI10_MasterSend) refers to sci.o(.data) for g_spi10_tx_count
    sci.o(i.SPI10_MasterSendReceive) refers to sci.o(i.SPI10_Start) for SPI10_Start
    sci.o(i.SPI10_MasterSendReceive) refers to sci.o(.data) for g_spi10_rx_count
    sci.o(i.SPI10_SlaveInit) refers to sci.o(i.__NVIC_SetPriority) for __NVIC_SetPriority
    sci.o(i.SPI10_SlaveReceive) refers to sci.o(i.SPI10_Start) for SPI10_Start
    sci.o(i.SPI10_SlaveReceive) refers to sci.o(.data) for g_spi10_rx_count
    sci.o(i.SPI10_SlaveSend) refers to sci.o(i.SPI10_Start) for SPI10_Start
    sci.o(i.SPI10_SlaveSend) refers to sci.o(.data) for g_spi10_tx_count
    sci.o(i.SPI10_Start) refers to sci.o(i.INTC_ClearPendingIRQ) for INTC_ClearPendingIRQ
    sci.o(i.SPI10_Start) refers to sci.o(i.__NVIC_ClearPendingIRQ) for __NVIC_ClearPendingIRQ
    sci.o(i.SPI10_Start) refers to sci.o(i.INTC_EnableIRQ) for INTC_EnableIRQ
    sci.o(i.SPI10_Stop) refers to sci.o(i.INTC_DisableIRQ) for INTC_DisableIRQ
    sci.o(i.SPI10_Stop) refers to sci.o(i.INTC_ClearPendingIRQ) for INTC_ClearPendingIRQ
    sci.o(i.SPI10_Stop) refers to sci.o(i.__NVIC_ClearPendingIRQ) for __NVIC_ClearPendingIRQ
    sci.o(i.SPI11_MasterReceive) refers to sci.o(i.SPI11_Start) for SPI11_Start
    sci.o(i.SPI11_MasterReceive) refers to sci.o(.data) for dummy_sio11
    sci.o(i.SPI11_MasterSend) refers to sci.o(i.SPI11_Start) for SPI11_Start
    sci.o(i.SPI11_MasterSend) refers to sci.o(.data) for g_spi11_tx_count
    sci.o(i.SPI11_SlaveInit) refers to sci.o(i.__NVIC_SetPriority) for __NVIC_SetPriority
    sci.o(i.SPI11_SlaveReceive) refers to sci.o(i.SPI11_Start) for SPI11_Start
    sci.o(i.SPI11_SlaveReceive) refers to sci.o(.data) for g_spi11_rx_count
    sci.o(i.SPI11_SlaveSend) refers to sci.o(i.SPI11_Start) for SPI11_Start
    sci.o(i.SPI11_SlaveSend) refers to sci.o(.data) for g_spi11_tx_count
    sci.o(i.SPI11_SlaveSendReceive) refers to sci.o(i.SPI11_Start) for SPI11_Start
    sci.o(i.SPI11_SlaveSendReceive) refers to sci.o(.data) for g_spi11_rx_count
    sci.o(i.SPI11_Start) refers to sci.o(i.INTC_ClearPendingIRQ) for INTC_ClearPendingIRQ
    sci.o(i.SPI11_Start) refers to sci.o(i.__NVIC_ClearPendingIRQ) for __NVIC_ClearPendingIRQ
    sci.o(i.SPI11_Start) refers to sci.o(i.INTC_EnableIRQ) for INTC_EnableIRQ
    sci.o(i.SPI11_Stop) refers to sci.o(i.INTC_DisableIRQ) for INTC_DisableIRQ
    sci.o(i.SPI11_Stop) refers to sci.o(i.INTC_ClearPendingIRQ) for INTC_ClearPendingIRQ
    sci.o(i.SPI11_Stop) refers to sci.o(i.__NVIC_ClearPendingIRQ) for __NVIC_ClearPendingIRQ
    sci.o(i.SPI20_MasterReceive) refers to sci.o(i.SPI20_Start) for SPI20_Start
    sci.o(i.SPI20_MasterReceive) refers to sci.o(i.INTC_GetPendingIRQ) for INTC_GetPendingIRQ
    sci.o(i.SPI20_MasterReceive) refers to sci.o(i.INTC_ClearPendingIRQ) for INTC_ClearPendingIRQ
    sci.o(i.SPI20_MasterReceive) refers to sci.o(i.SPI20_Stop) for SPI20_Stop
    sci.o(i.SPI20_MasterReceive) refers to sci.o(.data) for dummy_sio20
    sci.o(i.SPI20_MasterSend) refers to sci.o(i.SPI20_Start) for SPI20_Start
    sci.o(i.SPI20_MasterSend) refers to sci.o(i.INTC_GetPendingIRQ) for INTC_GetPendingIRQ
    sci.o(i.SPI20_MasterSend) refers to sci.o(i.INTC_ClearPendingIRQ) for INTC_ClearPendingIRQ
    sci.o(i.SPI20_MasterSend) refers to sci.o(i.SPI20_Stop) for SPI20_Stop
    sci.o(i.SPI20_SlaveInit) refers to sci.o(i.__NVIC_SetPriority) for __NVIC_SetPriority
    sci.o(i.SPI20_SlaveReceive) refers to sci.o(i.SPI20_Start) for SPI20_Start
    sci.o(i.SPI20_SlaveReceive) refers to sci.o(.data) for g_spi20_rx_count
    sci.o(i.SPI20_SlaveSend) refers to sci.o(i.SPI20_Start) for SPI20_Start
    sci.o(i.SPI20_SlaveSend) refers to sci.o(.data) for g_spi20_tx_count
    sci.o(i.SPI20_Start) refers to sci.o(i.INTC_ClearPendingIRQ) for INTC_ClearPendingIRQ
    sci.o(i.SPI20_Start) refers to sci.o(i.__NVIC_ClearPendingIRQ) for __NVIC_ClearPendingIRQ
    sci.o(i.SPI20_Start) refers to sci.o(i.INTC_EnableIRQ) for INTC_EnableIRQ
    sci.o(i.SPI20_Stop) refers to sci.o(i.INTC_DisableIRQ) for INTC_DisableIRQ
    sci.o(i.SPI20_Stop) refers to sci.o(i.INTC_ClearPendingIRQ) for INTC_ClearPendingIRQ
    sci.o(i.SPI21_MasterReceive) refers to sci.o(i.SPI21_Start) for SPI21_Start
    sci.o(i.SPI21_MasterReceive) refers to sci.o(.data) for g_spi21_rx_count
    sci.o(i.SPI21_MasterSend) refers to sci.o(i.SPI21_Start) for SPI21_Start
    sci.o(i.SPI21_MasterSend) refers to sci.o(.data) for g_spi21_tx_count
    sci.o(i.SPI21_MasterSendReceive) refers to sci.o(i.SPI21_Start) for SPI21_Start
    sci.o(i.SPI21_MasterSendReceive) refers to sci.o(.data) for g_spi21_rx_count
    sci.o(i.SPI21_SlaveInit) refers to sci.o(i.__NVIC_SetPriority) for __NVIC_SetPriority
    sci.o(i.SPI21_SlaveReceive) refers to sci.o(i.SPI21_Start) for SPI21_Start
    sci.o(i.SPI21_SlaveReceive) refers to sci.o(.data) for g_spi21_rx_count
    sci.o(i.SPI21_SlaveSend) refers to sci.o(i.SPI21_Start) for SPI21_Start
    sci.o(i.SPI21_SlaveSend) refers to sci.o(.data) for g_spi21_tx_count
    sci.o(i.SPI21_Start) refers to sci.o(i.INTC_ClearPendingIRQ) for INTC_ClearPendingIRQ
    sci.o(i.SPI21_Start) refers to sci.o(i.__NVIC_ClearPendingIRQ) for __NVIC_ClearPendingIRQ
    sci.o(i.SPI21_Start) refers to sci.o(i.INTC_EnableIRQ) for INTC_EnableIRQ
    sci.o(i.SPI21_Stop) refers to sci.o(i.INTC_DisableIRQ) for INTC_DisableIRQ
    sci.o(i.SPI21_Stop) refers to sci.o(i.INTC_ClearPendingIRQ) for INTC_ClearPendingIRQ
    sci.o(i.UART0_BaudRate) refers to sci.o(i.UART_BaudRateCal) for UART_BaudRateCal
    sci.o(i.UART0_Init) refers to sci.o(i.UART0_BaudRate) for UART0_BaudRate
    sci.o(i.UART1_BaudRate) refers to sci.o(i.UART_BaudRateCal) for UART_BaudRateCal
    sci.o(i.UART1_Init) refers to sci.o(i.INTC_DisableIRQ) for INTC_DisableIRQ
    sci.o(i.UART1_Init) refers to sci.o(i.INTC_ClearPendingIRQ) for INTC_ClearPendingIRQ
    sci.o(i.UART1_Init) refers to sci.o(i.UART1_BaudRate) for UART1_BaudRate
    sci.o(i.UART1_Init) refers to sci.o(i.UART1_Start) for UART1_Start
    sci.o(i.UART1_Receive) refers to sci.o(.data) for g_uart1_rx_count
    sci.o(i.UART1_Send) refers to sci.o(.data) for gp_uart1_tx_address
    sci.o(i.UART1_Start) refers to sci.o(i.INTC_ClearPendingIRQ) for INTC_ClearPendingIRQ
    sci.o(i.UART1_Start) refers to sci.o(i.__NVIC_ClearPendingIRQ) for __NVIC_ClearPendingIRQ
    sci.o(i.UART1_Start) refers to sci.o(i.INTC_EnableIRQ) for INTC_EnableIRQ
    sci.o(i.UART1_Stop) refers to sci.o(i.INTC_DisableIRQ) for INTC_DisableIRQ
    sci.o(i.UART1_Stop) refers to sci.o(i.INTC_ClearPendingIRQ) for INTC_ClearPendingIRQ
    sci.o(i.UART2_BaudRate) refers to sci.o(i.UART_BaudRateCal) for UART_BaudRateCal
    sci.o(i.UART2_Init) refers to sci.o(i.INTC_DisableIRQ) for INTC_DisableIRQ
    sci.o(i.UART2_Init) refers to sci.o(i.INTC_ClearPendingIRQ) for INTC_ClearPendingIRQ
    sci.o(i.UART2_Init) refers to system_bat32g137.o(i.SystemCoreClockUpdate) for SystemCoreClockUpdate
    sci.o(i.UART2_Init) refers to sci.o(i.UART2_BaudRate) for UART2_BaudRate
    sci.o(i.UART2_Init) refers to sci.o(i.UART2_Start) for UART2_Start
    sci.o(i.UART2_Init) refers to system_bat32g137.o(.data) for SystemCoreClock
    sci.o(i.UART2_Init) refers to sci_user.o(.data) for g_uart2_tx_state
    sci.o(i.UART2_Receive) refers to sci.o(.data) for g_uart2_rx_count
    sci.o(i.UART2_Send) refers to sci.o(.data) for gp_uart2_tx_address
    sci.o(i.UART2_Start) refers to sci.o(i.INTC_ClearPendingIRQ) for INTC_ClearPendingIRQ
    sci.o(i.UART2_Start) refers to sci.o(i.__NVIC_ClearPendingIRQ) for __NVIC_ClearPendingIRQ
    sci.o(i.UART2_Start) refers to sci.o(i.INTC_EnableIRQ) for INTC_EnableIRQ
    sci.o(i.UART2_Stop) refers to sci.o(i.INTC_DisableIRQ) for INTC_DisableIRQ
    sci.o(i.UART2_Stop) refers to sci.o(i.INTC_ClearPendingIRQ) for INTC_ClearPendingIRQ
    sci.o(i.UART_BaudRateCal) refers to aeabi_sdiv.o(.text) for __aeabi_uidivmod
    sci.o(i.UART_BaudRateCal) refers to sci.o(.constdata) for sps_tbl
    sci_user.o(i.Get_Uart2_State) refers to sci_user.o(.data) for g_uart2_tx_state
    sci_user.o(i.IRQ07_Handler) refers to sci_user.o(i.INTC_ClearPendingIRQ) for INTC_ClearPendingIRQ
    sci_user.o(i.IRQ07_Handler) refers to sci_user.o(i.uart2_callback_sendend) for uart2_callback_sendend
    sci_user.o(i.IRQ07_Handler) refers to sci.o(.data) for g_uart2_tx_count
    sci_user.o(i.IRQ08_Handler) refers to sci_user.o(i.INTC_ClearPendingIRQ) for INTC_ClearPendingIRQ
    sci_user.o(i.IRQ08_Handler) refers to sci_user.o(i.uart2_callback_error) for uart2_callback_error
    sci_user.o(i.IRQ08_Handler) refers to sci_user.o(i.uart2_callback_receiveend) for uart2_callback_receiveend
    sci_user.o(i.IRQ08_Handler) refers to sci.o(.data) for g_uart2_rx_count
    sci_user.o(i.IRQ08_Handler) refers to sci_user.o(.data) for lastData
    sci_user.o(i.IRQ08_Handler) refers to mcu_core_protocol.o(.bss) for Uart2_rx_buf
    sci_user.o(i.UART_Ch2_Send_Multiple_Byte) refers to mcu_core_protocol.o(.bss) for Uart2_tx_buf
    sci_user.o(i.UART_Ch2_Send_Multiple_Byte) refers to sci.o(.data) for gp_uart2_tx_address
    sci_user.o(i.UART_Ch2_Send_Multiple_Byte) refers to sci_user.o(.data) for g_uart2_tx_state
    sci_user.o(i.uart0_interrupt_receive) refers to sci_user.o(i.INTC_ClearPendingIRQ) for INTC_ClearPendingIRQ
    sci_user.o(i.uart0_interrupt_receive) refers to sci_user.o(i.uart0_callback_error) for uart0_callback_error
    sci_user.o(i.uart0_interrupt_receive) refers to sci_user.o(i.uart0_callback_receiveend) for uart0_callback_receiveend
    sci_user.o(i.uart0_interrupt_receive) refers to sci_user.o(i.uart0_callback_softwareoverrun) for uart0_callback_softwareoverrun
    sci_user.o(i.uart0_interrupt_receive) refers to sci.o(.data) for g_uart0_rx_length
    sci_user.o(i.uart0_interrupt_send) refers to sci_user.o(i.INTC_ClearPendingIRQ) for INTC_ClearPendingIRQ
    sci_user.o(i.uart0_interrupt_send) refers to sci_user.o(i.uart0_callback_sendend) for uart0_callback_sendend
    sci_user.o(i.uart0_interrupt_send) refers to sci.o(.data) for g_uart0_tx_count
    sci_user.o(i.uart2_callback_error) refers to sci.o(.data) for g_uart2_rx_count
    sci_user.o(i.uart2_callback_receiveend) refers to sci.o(.data) for g_uart2_rx_count
    sci_user.o(i.uart2_callback_sendend) refers to sci_user.o(.data) for g_uart2_tx_state
    main.o(i.main) refers to sys_scheduler.o(i.Sys_Init) for Sys_Init
    main.o(i.main) refers to sys_scheduler.o(i.Sys_Scheduling_Service) for Sys_Scheduling_Service
    main.o(i.main) refers to wdt.o(i.WDT_Restart) for WDT_Restart
    tasks.o(i.Sys_Exact_50us_Tasks) refers to system_monitor_user.o(i.Sys_Rolling) for Sys_Rolling
    tasks.o(i.Sys_Run_Mode_10ms_Tasks) refers to line_in.o(i.Line_In_Debounce_Service) for Line_In_Debounce_Service
    tasks.o(i.Sys_Run_Mode_2ms_Tasks) refers to analog_signals.o(i.Analog_Signal_Conv_Service) for Analog_Signal_Conv_Service
    tasks.o(i.Sys_Run_Mode_2ms_Tasks) refers to mcu_core_protocol.o(i.MCU_Send_Service) for MCU_Send_Service
    tasks.o(i.Sys_Run_Mode_Pseudo_Real_Time_Tasks) refers to adc.o(i.Analog_Signal_Conv_Real_Time_Run) for Analog_Signal_Conv_Real_Time_Run
    tasks.o(i.Sys_Run_Mode_Pseudo_Real_Time_Tasks) refers to powermanagement.o(i.Power_Management_Service) for Power_Management_Service
    sys_scheduler.o(i.Sys_Exact_100ms_Task_Handler) refers to tasks.o(i.Sys_Exact_100ms_Tasks) for Sys_Exact_100ms_Tasks
    sys_scheduler.o(i.Sys_Exact_50us_Task_Handler) refers to tasks.o(i.Sys_Exact_50us_Tasks) for Sys_Exact_50us_Tasks
    sys_scheduler.o(i.Sys_Init) refers to sys_tick.o(i.Sys_Tick_Timer_Call_Back_Reg) for Sys_Tick_Timer_Call_Back_Reg
    sys_scheduler.o(i.Sys_Init) refers to init.o(i.Sys_Startup_Init) for Sys_Startup_Init
    sys_scheduler.o(i.Sys_Init) refers to sys_scheduler.o(.bss) for SysScheduling
    sys_scheduler.o(i.Sys_Init) refers to sys_scheduler.o(i.Sys_Exact_50us_Task_Handler) for Sys_Exact_50us_Task_Handler
    sys_scheduler.o(i.Sys_Init) refers to sys_scheduler.o(i.Sys_Exact_100ms_Task_Handler) for Sys_Exact_100ms_Task_Handler
    sys_scheduler.o(i.Sys_Scheduling_Service) refers to tasks.o(i.Sys_Run_Mode_Pseudo_Real_Time_Tasks) for Sys_Run_Mode_Pseudo_Real_Time_Tasks
    sys_scheduler.o(i.Sys_Scheduling_Service) refers to tasks.o(i.Sys_Run_Mode_2ms_Tasks) for Sys_Run_Mode_2ms_Tasks
    sys_scheduler.o(i.Sys_Scheduling_Service) refers to tasks.o(i.Sys_Run_Mode_5ms_Tasks) for Sys_Run_Mode_5ms_Tasks
    sys_scheduler.o(i.Sys_Scheduling_Service) refers to tasks.o(i.Sys_Run_Mode_10ms_Tasks) for Sys_Run_Mode_10ms_Tasks
    sys_scheduler.o(i.Sys_Scheduling_Service) refers to tasks.o(i.Sys_Run_Mode_20ms_Tasks) for Sys_Run_Mode_20ms_Tasks
    sys_scheduler.o(i.Sys_Scheduling_Service) refers to tasks.o(i.Sys_Run_Mode_50ms_Tasks) for Sys_Run_Mode_50ms_Tasks
    sys_scheduler.o(i.Sys_Scheduling_Service) refers to tasks.o(i.Sys_Run_Mode_100ms_Tasks) for Sys_Run_Mode_100ms_Tasks
    sys_scheduler.o(i.Sys_Scheduling_Service) refers to sys_tick.o(.data) for g_u16SysRollingCounter1ms
    sys_scheduler.o(i.Sys_Scheduling_Service) refers to sys_scheduler.o(.bss) for SysScheduling
    init.o(i.Sys_Startup_Init) refers to gpio.o(i.GPIO_Init) for GPIO_Init
    init.o(i.Sys_Startup_Init) refers to sys_tick.o(i.Sys_Tick_Timer_Start) for Sys_Tick_Timer_Start
    init.o(i.Sys_Startup_Init) refers to analog_signals.o(i.Analog_Signal_Conv_Init) for Analog_Signal_Conv_Init
    init.o(i.Sys_Startup_Init) refers to sci.o(i.UART2_Init) for UART2_Init
    init.o(i.Sys_Startup_Init) refers to powermanagement_user.o(i.Power_Management_Lib_Init) for Power_Management_Lib_Init
    init.o(i.Sys_Startup_Init) refers to powermanagement.o(i.Power_Management_Init) for Power_Management_Init
    line_in.o(i.LINE_IN_Get_ABS) refers to gpio.o(i.PORT_GetBit) for PORT_GetBit
    line_in.o(i.LINE_IN_Get_Gear_1) refers to gpio.o(i.PORT_GetBit) for PORT_GetBit
    line_in.o(i.LINE_IN_Get_Gear_2) refers to gpio.o(i.PORT_GetBit) for PORT_GetBit
    line_in.o(i.LINE_IN_Get_Gear_3) refers to gpio.o(i.PORT_GetBit) for PORT_GetBit
    line_in.o(i.LINE_IN_Get_Gear_4) refers to gpio.o(i.PORT_GetBit) for PORT_GetBit
    line_in.o(i.LINE_IN_Get_Gear_5) refers to gpio.o(i.PORT_GetBit) for PORT_GetBit
    line_in.o(i.LINE_IN_Get_Gear_6) refers to gpio.o(i.PORT_GetBit) for PORT_GetBit
    line_in.o(i.LINE_IN_Get_Gear_N) refers to gpio.o(i.PORT_GetBit) for PORT_GetBit
    line_in.o(i.LINE_IN_Get_HighBeam) refers to gpio.o(i.PORT_GetBit) for PORT_GetBit
    line_in.o(i.LINE_IN_Get_Key1) refers to gpio.o(i.PORT_GetBit) for PORT_GetBit
    line_in.o(i.LINE_IN_Get_Key2) refers to gpio.o(i.PORT_GetBit) for PORT_GetBit
    line_in.o(i.LINE_IN_Get_LeftTurn) refers to gpio.o(i.PORT_GetBit) for PORT_GetBit
    line_in.o(i.LINE_IN_Get_OilPressure) refers to gpio.o(i.PORT_GetBit) for PORT_GetBit
    line_in.o(i.LINE_IN_Get_RightTurn) refers to gpio.o(i.PORT_GetBit) for PORT_GetBit
    line_in.o(i.Line_In_Debounce_Handle) refers to line_in.o(.constdata) for g_stLineInAttribute
    line_in.o(i.Line_In_Debounce_Handle) refers to line_in.o(.bss) for g_stLineInControl
    line_in.o(i.Line_In_Debounce_Service) refers to line_in.o(i.Line_In_Debounce_Handle) for Line_In_Debounce_Handle
    line_in.o(i.Line_In_Debounce_Service) refers to line_in.o(.constdata) for g_stLineInAttribute
    line_in.o(i.Line_In_Debounce_Service) refers to line_in.o(.data) for g_enLineInPowerStatus
    line_in.o(i.Line_In_Get_Status) refers to line_in.o(.bss) for g_stLineInControl
    line_in.o(i.Line_In_KL15_OFF_Init) refers to line_in.o(.data) for g_enLineInPowerStatus
    line_in.o(i.Line_In_KL15_OFF_Init) refers to line_in.o(.constdata) for g_stLineInAttribute
    line_in.o(i.Line_In_KL15_OFF_Init) refers to line_in.o(.bss) for g_stLineInControl
    line_in.o(i.Line_In_KL15_ON_Init) refers to line_in.o(.data) for g_enLineInPowerStatus
    line_in.o(i.Line_In_KL15_ON_Init) refers to line_in.o(.constdata) for g_stLineInAttribute
    line_in.o(i.Line_In_KL15_ON_Init) refers to line_in.o(.bss) for g_stLineInControl
    line_in.o(i.Line_In_KL30_Init) refers to line_in.o(.data) for g_enLineInPowerStatus
    line_in.o(i.Line_In_KL30_Init) refers to line_in.o(.bss) for g_stLineInControl
    line_in.o(i.Line_In_SetPowerSt) refers to line_in.o(.data) for g_enLineInPowerStatus
    line_in.o(.constdata) refers to line_in.o(i.LINE_IN_Get_RightTurn) for LINE_IN_Get_RightTurn
    line_in.o(.constdata) refers to line_in.o(i.LINE_IN_Get_LeftTurn) for LINE_IN_Get_LeftTurn
    line_in.o(.constdata) refers to line_in.o(i.LINE_IN_Get_HighBeam) for LINE_IN_Get_HighBeam
    line_in.o(.constdata) refers to line_in.o(i.LINE_IN_Get_ABS) for LINE_IN_Get_ABS
    line_in.o(.constdata) refers to line_in.o(i.LINE_IN_Get_OilPressure) for LINE_IN_Get_OilPressure
    line_in.o(.constdata) refers to line_in.o(i.LINE_IN_Get_Key1) for LINE_IN_Get_Key1
    line_in.o(.constdata) refers to line_in.o(i.LINE_IN_Get_Key2) for LINE_IN_Get_Key2
    line_in.o(.constdata) refers to line_in.o(i.LINE_IN_Get_Gear_N) for LINE_IN_Get_Gear_N
    line_in.o(.constdata) refers to line_in.o(i.LINE_IN_Get_Gear_1) for LINE_IN_Get_Gear_1
    line_in.o(.constdata) refers to line_in.o(i.LINE_IN_Get_Gear_2) for LINE_IN_Get_Gear_2
    line_in.o(.constdata) refers to line_in.o(i.LINE_IN_Get_Gear_3) for LINE_IN_Get_Gear_3
    line_in.o(.constdata) refers to line_in.o(i.LINE_IN_Get_Gear_4) for LINE_IN_Get_Gear_4
    line_in.o(.constdata) refers to line_in.o(i.LINE_IN_Get_Gear_5) for LINE_IN_Get_Gear_5
    line_in.o(.constdata) refers to line_in.o(i.LINE_IN_Get_Gear_6) for LINE_IN_Get_Gear_6
    powermanagement.o(i.PowerMemInit) refers to powermanagement.o(.bss) for pFuncPower
    powermanagement.o(i.PowerMemInit) refers to powermanagement.o(.data) for g_Power_St
    powermanagement.o(i.Power_Management_Init) refers to powermanagement.o(.bss) for pFuncPower
    powermanagement.o(i.Power_Management_Init) refers to powermanagement.o(.data) for g_Power_St
    powermanagement.o(i.Power_Management_Service) refers to gpio.o(i.__ARM_common_switch8) for __ARM_common_switch8
    powermanagement.o(i.Power_Management_Service) refers to powermanagement.o(.data) for g_Power_St
    powermanagement.o(i.Power_Management_Service) refers to powermanagement.o(.bss) for pFuncPower
    powermanagement_user.o(i.Power_IG_OFF_Init) refers to line_in.o(i.Line_In_KL15_OFF_Init) for Line_In_KL15_OFF_Init
    powermanagement_user.o(i.Power_IG_ON_Init) refers to line_in.o(i.Line_In_KL15_ON_Init) for Line_In_KL15_ON_Init
    powermanagement_user.o(i.Power_KL30_Init) refers to system_monitor_user.o(i.Sys_KL30_Init) for Sys_KL30_Init
    powermanagement_user.o(i.Power_KL30_Init) refers to line_in.o(i.Line_In_KL30_Init) for Line_In_KL30_Init
    powermanagement_user.o(i.Power_Management_Lib_Init) refers to powermanagement.o(i.PowerMemInit) for PowerMemInit
    powermanagement_user.o(i.Power_Management_Lib_Init) refers to powermanagement_user.o(i.Power_IG_OFF_Init) for Power_IG_OFF_Init
    powermanagement_user.o(i.Power_Management_Lib_Init) refers to powermanagement_user.o(i.Power_IG_ON_Init) for Power_IG_ON_Init
    powermanagement_user.o(i.Power_Management_Lib_Init) refers to powermanagement_user.o(i.Power_Sleep_Init) for Power_Sleep_Init
    powermanagement_user.o(i.Power_Management_Lib_Init) refers to powermanagement_user.o(i.Power_IG_OVP_Init) for Power_IG_OVP_Init
    powermanagement_user.o(i.Power_Management_Lib_Init) refers to powermanagement_user.o(i.Power_IG_LVP_Init) for Power_IG_LVP_Init
    powermanagement_user.o(i.Power_Management_Lib_Init) refers to powermanagement_user.o(i.Power_KL30_Init) for Power_KL30_Init
    powermanagement_user.o(i.Power_Management_Lib_Init) refers to powermanagement_user.o(i.Power_Wakeup_Init) for Power_Wakeup_Init
    powermanagement_user.o(i.Power_Management_Lib_Init) refers to powermanagement_user.o(i.Power_Stay_OFF) for Power_Stay_OFF
    powermanagement_user.o(i.Power_Management_Lib_Init) refers to powermanagement_user.o(i.Power_Stay_ON) for Power_Stay_ON
    powermanagement_user.o(i.Power_Management_Lib_Init) refers to powermanagement_user.o(i.Power_Stay_Sleep) for Power_Stay_Sleep
    powermanagement_user.o(i.Power_Management_Lib_Init) refers to powermanagement_user.o(i.Power_Stay_Protect) for Power_Stay_Protect
    powermanagement_user.o(i.Power_Sleep_Init) refers to gpio.o(i.GPIO_Init) for GPIO_Init
    powermanagement_user.o(i.Power_Stay_OFF) refers to common_interface.o(i.Common_Get_IG_Sts) for Common_Get_IG_Sts
    powermanagement_user.o(i.Power_Stay_OFF) refers to common_interface.o(i.Common_Get_IG_Sts_Valid) for Common_Get_IG_Sts_Valid
    powermanagement_user.o(i.Power_Stay_ON) refers to common_interface.o(i.Common_Get_IG_Sts) for Common_Get_IG_Sts
    powermanagement_user.o(i.Power_Stay_ON) refers to common_interface.o(i.Common_Get_IG_Sts_Valid) for Common_Get_IG_Sts_Valid
    powermanagement_user.o(i.Power_Stay_ON) refers to system_monitor.o(i.System_FUN_KL30_Status_Get) for System_FUN_KL30_Status_Get
    powermanagement_user.o(i.Power_Wakeup_Init) refers to system_monitor_user.o(i.Sys_WakeUp_Init) for Sys_WakeUp_Init
    powermanagement_user.o(i.Power_Wakeup_Init) refers to line_in.o(i.Line_In_KL30_Init) for Line_In_KL30_Init
    system_monitor.o(i.Read_KL30_ConvertFinish) refers to system_monitor.o(.data) for SysWakeUpMode
    system_monitor.o(i.Sys_Set_DebounceTimer) refers to system_monitor.o(.data) for t_NM_KL30_Debounce
    system_monitor.o(i.Sys_Set_VolRange) refers to system_monitor.o(.data) for FUNSysVol_Range
    system_monitor.o(i.Sys_Status_Update_Service) refers to system_monitor.o(i.System_Fun_Process) for System_Fun_Process
    system_monitor.o(i.Sys_Status_Update_Service) refers to system_monitor.o(i.System_NM_Process) for System_NM_Process
    system_monitor.o(i.Sys_Status_Update_Service) refers to system_monitor_user.o(i.Sys_LogicProcess) for Sys_LogicProcess
    system_monitor.o(i.System_Calc_FunRange) refers to system_monitor.o(.data) for FUNSysVol_Range
    system_monitor.o(i.System_Calc_NMRange) refers to system_monitor.o(.data) for NMSysVol_Range
    system_monitor.o(i.System_FUN_KL15_Status_Get) refers to system_monitor.o(.bss) for SysFun_KL15Monitor
    system_monitor.o(i.System_FUN_KL30_Status_Get) refers to system_monitor.o(.bss) for SysFun_KL30Monitor
    system_monitor.o(i.System_Fast_WakeUp) refers to system_monitor_user.o(i.Sys_Force_Read_KL30_Voltage) for Sys_Force_Read_KL30_Voltage
    system_monitor.o(i.System_Fast_WakeUp) refers to system_monitor_user.o(i.Sys_Force_Read_KL15_Voltage) for Sys_Force_Read_KL15_Voltage
    system_monitor.o(i.System_Fast_WakeUp) refers to system_monitor_user.o(i.Sys_BlockDelay) for Sys_BlockDelay
    system_monitor.o(i.System_Fast_WakeUp) refers to system_monitor_user.o(i.System_LINE_KL15) for System_LINE_KL15
    system_monitor.o(i.System_Fast_WakeUp) refers to system_monitor_user.o(i.Sys_LogicProcess) for Sys_LogicProcess
    system_monitor.o(i.System_Fast_WakeUp) refers to system_monitor.o(.data) for FUNSysVol_Range
    system_monitor.o(i.System_Fast_WakeUp) refers to system_monitor.o(.bss) for SysNM_KL30Monitor
    system_monitor.o(i.System_Fun_Process) refers to system_monitor_user.o(i.System_LINE_KL15) for System_LINE_KL15
    system_monitor.o(i.System_Fun_Process) refers to system_monitor_user.o(i.Sys_Read_KL30_Valid) for Sys_Read_KL30_Valid
    system_monitor.o(i.System_Fun_Process) refers to system_monitor_user.o(i.Sys_Read_KL15_Valid) for Sys_Read_KL15_Valid
    system_monitor.o(i.System_Fun_Process) refers to system_monitor_user.o(i.Sys_Read_KL15_Voltage) for Sys_Read_KL15_Voltage
    system_monitor.o(i.System_Fun_Process) refers to system_monitor_user.o(i.Sys_Read_KL30_Voltage) for Sys_Read_KL30_Voltage
    system_monitor.o(i.System_Fun_Process) refers to aeabi_sdiv.o(.text) for __aeabi_uidivmod
    system_monitor.o(i.System_Fun_Process) refers to system_monitor.o(i.System_Calc_FunRange) for System_Calc_FunRange
    system_monitor.o(i.System_Fun_Process) refers to system_monitor.o(.bss) for SysFun_KL15Monitor
    system_monitor.o(i.System_Fun_Process) refers to system_monitor.o(.data) for t_FUN_KL15_Debounce
    system_monitor.o(i.System_Monitor_KL30Init) refers to system_monitor.o(.data) for SysWakeUpMode
    system_monitor.o(i.System_Monitor_KL30Init) refers to system_monitor.o(.bss) for SysFun_KL30Monitor
    system_monitor.o(i.System_Monitor_WakeupInit) refers to system_monitor.o(.data) for SysWakeUpMode
    system_monitor.o(i.System_Monitor_WakeupInit) refers to system_monitor.o(.bss) for SysFun_KL30Monitor
    system_monitor.o(i.System_NM_KL15_Status_Get) refers to system_monitor.o(.bss) for SysNM_KL15Monitor
    system_monitor.o(i.System_NM_KL30_Status_Get) refers to system_monitor.o(.bss) for SysNM_KL30Monitor
    system_monitor.o(i.System_NM_Process) refers to system_monitor_user.o(i.System_LINE_KL15) for System_LINE_KL15
    system_monitor.o(i.System_NM_Process) refers to system_monitor_user.o(i.Sys_Read_KL30_Valid) for Sys_Read_KL30_Valid
    system_monitor.o(i.System_NM_Process) refers to system_monitor_user.o(i.Sys_Read_KL15_Valid) for Sys_Read_KL15_Valid
    system_monitor.o(i.System_NM_Process) refers to system_monitor_user.o(i.Sys_Read_KL15_Voltage) for Sys_Read_KL15_Voltage
    system_monitor.o(i.System_NM_Process) refers to system_monitor_user.o(i.Sys_Read_KL30_Voltage) for Sys_Read_KL30_Voltage
    system_monitor.o(i.System_NM_Process) refers to aeabi_sdiv.o(.text) for __aeabi_uidivmod
    system_monitor.o(i.System_NM_Process) refers to system_monitor.o(i.System_Calc_NMRange) for System_Calc_NMRange
    system_monitor.o(i.System_NM_Process) refers to system_monitor.o(.bss) for SysNM_KL15Monitor
    system_monitor.o(i.System_NM_Process) refers to system_monitor.o(.data) for t_NM_KL15_Debounce
    system_monitor_user.o(i.Sys_BlockDelay) refers to system_monitor_user.o(i.Sys_RollingClear) for Sys_RollingClear
    system_monitor_user.o(i.Sys_BlockDelay) refers to system_monitor_user.o(i.Sys_Get_ms_Rolling_Counter) for Sys_Get_ms_Rolling_Counter
    system_monitor_user.o(i.Sys_BlockDelay) refers to wdt.o(i.WDT_Restart) for WDT_Restart
    system_monitor_user.o(i.Sys_Force_Read_KL15_Voltage) refers to rte_adc.o(i.RTE_ForceRead_KL15_Voltage) for RTE_ForceRead_KL15_Voltage
    system_monitor_user.o(i.Sys_Force_Read_KL30_Voltage) refers to rte_adc.o(i.RTE_ForceRead_KL30_Voltage) for RTE_ForceRead_KL30_Voltage
    system_monitor_user.o(i.Sys_Get_ms_Rolling_Counter) refers to system_monitor_user.o(.data) for u32SysRollingCounter
    system_monitor_user.o(i.Sys_KL30_Init) refers to system_monitor.o(i.Sys_Set_DebounceTimer) for Sys_Set_DebounceTimer
    system_monitor_user.o(i.Sys_KL30_Init) refers to system_monitor.o(i.Sys_Set_VolRange) for Sys_Set_VolRange
    system_monitor_user.o(i.Sys_KL30_Init) refers to system_monitor.o(i.System_Monitor_KL30Init) for System_Monitor_KL30Init
    system_monitor_user.o(i.Sys_KL30_Init) refers to system_monitor.o(i.System_Fast_WakeUp) for System_Fast_WakeUp
    system_monitor_user.o(i.Sys_KL30_Init) refers to system_monitor_user.o(.constdata) for SysNM_Range
    system_monitor_user.o(i.Sys_Read_KL15_Valid) refers to rte_adc.o(i.RTE_Read_KL15_Valid) for RTE_Read_KL15_Valid
    system_monitor_user.o(i.Sys_Read_KL15_Voltage) refers to rte_adc.o(i.RTE_Read_KL15_Voltage) for RTE_Read_KL15_Voltage
    system_monitor_user.o(i.Sys_Read_KL30_Valid) refers to rte_adc.o(i.RTE_Read_KL30_Valid) for RTE_Read_KL30_Valid
    system_monitor_user.o(i.Sys_Read_KL30_Voltage) refers to rte_adc.o(i.RTE_Read_KL30_Voltage) for RTE_Read_KL30_Voltage
    system_monitor_user.o(i.Sys_Rolling) refers to system_monitor_user.o(.data) for u32SysRollingCounter
    system_monitor_user.o(i.Sys_RollingClear) refers to system_monitor_user.o(.data) for u32SysRollingCounter
    system_monitor_user.o(i.Sys_WakeUp_Init) refers to system_monitor.o(i.Sys_Set_DebounceTimer) for Sys_Set_DebounceTimer
    system_monitor_user.o(i.Sys_WakeUp_Init) refers to system_monitor.o(i.Sys_Set_VolRange) for Sys_Set_VolRange
    system_monitor_user.o(i.Sys_WakeUp_Init) refers to system_monitor.o(i.System_Monitor_WakeupInit) for System_Monitor_WakeupInit
    system_monitor_user.o(i.Sys_WakeUp_Init) refers to system_monitor.o(i.System_Fast_WakeUp) for System_Fast_WakeUp
    system_monitor_user.o(i.Sys_WakeUp_Init) refers to system_monitor_user.o(.constdata) for SysNM_Range
    system_monitor_user.o(i.System_LINE_KL15) refers to gpio.o(i.PORT_GetBit) for PORT_GetBit
    rte_adc.o(i.RTE_ADC_Init) refers to analog_signals.o(i.Analog_Signal_Conv_Init) for Analog_Signal_Conv_Init
    rte_adc.o(i.RTE_ForceRead_FUEL1_1_Voltage) refers to analog_signals.o(i.ADC_Conv_Single_Channel) for ADC_Conv_Single_Channel
    rte_adc.o(i.RTE_ForceRead_FUEL1_2_Voltage) refers to analog_signals.o(i.ADC_Conv_Single_Channel) for ADC_Conv_Single_Channel
    rte_adc.o(i.RTE_ForceRead_FUEL2_2_Voltage) refers to analog_signals.o(i.ADC_Conv_Single_Channel) for ADC_Conv_Single_Channel
    rte_adc.o(i.RTE_ForceRead_KL15_Voltage) refers to analog_signals.o(i.ADC_Conv_Single_Channel) for ADC_Conv_Single_Channel
    rte_adc.o(i.RTE_ForceRead_KL30_Voltage) refers to analog_signals.o(i.ADC_Conv_Single_Channel) for ADC_Conv_Single_Channel
    rte_adc.o(i.RTE_Read_FUEL1_1_Valid) refers to analog_signals.o(i.ADC_Read_Signal_Valid) for ADC_Read_Signal_Valid
    rte_adc.o(i.RTE_Read_FUEL1_1_Voltage) refers to analog_signals.o(i.ADC_Read_Signal) for ADC_Read_Signal
    rte_adc.o(i.RTE_Read_FUEL1_2_Valid) refers to analog_signals.o(i.ADC_Read_Signal_Valid) for ADC_Read_Signal_Valid
    rte_adc.o(i.RTE_Read_FUEL1_2_Voltage) refers to analog_signals.o(i.ADC_Read_Signal) for ADC_Read_Signal
    rte_adc.o(i.RTE_Read_FUEL2_2_Valid) refers to analog_signals.o(i.ADC_Read_Signal_Valid) for ADC_Read_Signal_Valid
    rte_adc.o(i.RTE_Read_FUEL2_2_Voltage) refers to analog_signals.o(i.ADC_Read_Signal) for ADC_Read_Signal
    rte_adc.o(i.RTE_Read_KL15_Valid) refers to analog_signals.o(i.ADC_Read_Signal_Valid) for ADC_Read_Signal_Valid
    rte_adc.o(i.RTE_Read_KL15_Voltage) refers to analog_signals.o(i.ADC_Read_Signal) for ADC_Read_Signal
    rte_adc.o(i.RTE_Read_KL30_Valid) refers to analog_signals.o(i.ADC_Read_Signal_Valid) for ADC_Read_Signal_Valid
    rte_adc.o(i.RTE_Read_KL30_Voltage) refers to analog_signals.o(i.ADC_Read_Signal) for ADC_Read_Signal
    common_interface.o(i.Common_BlockDelay) refers to common_interface.o(i.Common_RollingCounterClear) for Common_RollingCounterClear
    common_interface.o(i.Common_BlockDelay) refers to common_interface.o(i.Common_ReadRollingCounter) for Common_ReadRollingCounter
    common_interface.o(i.Common_DataInit) refers to common_interface.o(.data) for PowerSts
    common_interface.o(i.Common_GetIgnOffTime) refers to common_interface.o(.data) for PowerIgnOffTimeLine
    common_interface.o(i.Common_GetIgnOnTime) refers to common_interface.o(.data) for PowerIgnOnTimeLine
    common_interface.o(i.Common_Get_Act_E_Speed) refers to common_interface.o(.data) for Act_E_Speed
    common_interface.o(i.Common_Get_Act_E_Speed_Valid) refers to common_interface.o(.data) for Act_E_Speed_Valid
    common_interface.o(i.Common_Get_Act_V_Speed) refers to common_interface.o(.data) for Act_V_Speed
    common_interface.o(i.Common_Get_Act_V_Speed_Valid) refers to common_interface.o(.data) for Act_V_Speed_Valid
    common_interface.o(i.Common_Get_ConnectPhoneSts) refers to common_interface.o(.data) for g_ConnectPhone
    common_interface.o(i.Common_Get_DispMode) refers to common_interface.o(.data) for g_Disp_Mode
    common_interface.o(i.Common_Get_DispSpeed) refers to aeabi_sdiv.o(.text) for __aeabi_uidivmod
    common_interface.o(i.Common_Get_DispSpeed) refers to common_interface.o(.data) for Disp_V_Speed_Valid
    common_interface.o(i.Common_Get_Disp_E_Speed) refers to common_interface.o(.data) for Disp_E_Speed
    common_interface.o(i.Common_Get_Disp_E_Speed_Valid) refers to common_interface.o(.data) for Disp_E_Speed_Valid
    common_interface.o(i.Common_Get_Disp_V_Speed) refers to common_interface.o(.data) for Disp_V_Speed
    common_interface.o(i.Common_Get_Disp_V_Speed_Valid) refers to common_interface.o(.data) for Disp_V_Speed_Valid
    common_interface.o(i.Common_Get_IG_Sts) refers to common_interface.o(.data) for PowerSts
    common_interface.o(i.Common_Get_IG_Sts_Valid) refers to common_interface.o(.data) for PowerSts_Valid
    common_interface.o(i.Common_Get_Language) refers to common_interface.o(.data) for g_Language
    common_interface.o(i.Common_Get_Theme) refers to common_interface.o(.data) for g_Theme
    common_interface.o(i.Common_ReadRollingCounter) refers to common_interface.o(.data) for SysRollingCounter
    common_interface.o(i.Common_RollingCounterAdd) refers to common_interface.o(.data) for SysRollingCounter
    common_interface.o(i.Common_RollingCounterClear) refers to common_interface.o(.data) for SysRollingCounter
    common_interface.o(i.Common_Set_Act_E_Speed) refers to common_interface.o(.data) for Act_E_Speed
    common_interface.o(i.Common_Set_Act_E_Speed_Valid) refers to common_interface.o(.data) for Act_E_Speed_Valid
    common_interface.o(i.Common_Set_Act_V_Speed) refers to common_interface.o(.data) for Act_V_Speed
    common_interface.o(i.Common_Set_Act_V_Speed_Valid) refers to common_interface.o(.data) for Act_V_Speed_Valid
    common_interface.o(i.Common_Set_Disp_E_Speed) refers to common_interface.o(.data) for Disp_E_Speed
    common_interface.o(i.Common_Set_Disp_E_Speed_Valid) refers to common_interface.o(.data) for Disp_E_Speed_Valid
    common_interface.o(i.Common_Set_Disp_V_Speed) refers to common_interface.o(.data) for Disp_V_Speed
    common_interface.o(i.Common_Set_Disp_V_Speed_Valid) refers to common_interface.o(.data) for Disp_V_Speed_Valid
    common_interface.o(i.Common_Set_IG_Sts) refers to common_interface.o(.data) for PowerSts
    common_interface.o(i.Common_Set_IG_Sts_Valid) refers to common_interface.o(.data) for PowerSts_Valid
    mcu_core_protocol.o(i.Get_ID_01_Data) refers to common_interface.o(i.Common_Get_DispMode) for Common_Get_DispMode
    mcu_core_protocol.o(i.Get_ID_01_Data) refers to common_interface.o(i.Common_Get_IG_Sts) for Common_Get_IG_Sts
    mcu_core_protocol.o(i.Get_ID_01_Data) refers to common_interface.o(i.Common_Get_Language) for Common_Get_Language
    mcu_core_protocol.o(i.Get_ID_01_Data) refers to common_interface.o(i.Common_Get_Theme) for Common_Get_Theme
    mcu_core_protocol.o(i.Get_ID_01_Data) refers to common_interface.o(i.Common_Get_ConnectPhoneSts) for Common_Get_ConnectPhoneSts
    mcu_core_protocol.o(i.Get_ID_01_Data) refers to mcu_core_protocol.o(.data) for Send_ID_01_00
    mcu_core_protocol.o(i.Get_ID_01_Data) refers to mcu_core_protocol.o(.bss) for Send_ID_01_02
    mcu_core_protocol.o(i.Get_ID_02_Data) refers to common_interface.o(i.Common_Get_IG_Sts) for Common_Get_IG_Sts
    mcu_core_protocol.o(i.Get_ID_02_Data) refers to mcu_core_protocol.o(.bss) for Send_ID_02
    mcu_core_protocol.o(i.MCU_Send_Service) refers to sci_user.o(i.Get_Uart2_State) for Get_Uart2_State
    mcu_core_protocol.o(i.MCU_Send_Service) refers to mcu_core_protocol.o(i.Send_To_Core) for Send_To_Core
    mcu_core_protocol.o(i.MCU_Send_Service) refers to mcu_core_protocol.o(.data) for SendCtrl_Tbl
    mcu_core_protocol.o(i.Send_To_Core) refers to mcu_core_protocol.o(i.TFT_CreateCRCCheckSum) for TFT_CreateCRCCheckSum
    mcu_core_protocol.o(i.Send_To_Core) refers to sci_user.o(i.UART_Ch2_Send_Multiple_Byte) for UART_Ch2_Send_Multiple_Byte
    mcu_core_protocol.o(i.Send_To_Core) refers to mcu_core_protocol.o(.bss) for Uart2_tx_buf
    mcu_core_protocol.o(i.Send_To_Core) refers to mcu_core_protocol.o(.data) for PackageCnt
    mcu_core_protocol.o(i.Send_To_Core) refers to sci_user.o(.data) for g_uart2_tx_state
    mcu_core_protocol.o(i.TFT_CreateCRCCheckSum) refers to mcu_core_protocol.o(.constdata) for CRC16_TAB_H
    mcu_core_protocol.o(.data) refers to mcu_core_protocol.o(i.Get_ID_01_Data) for Get_ID_01_Data
    mcu_core_protocol.o(.data) refers to mcu_core_protocol.o(i.Get_ID_02_Data) for Get_ID_02_Data
    startup_bat32g137.o(STACK) refers (Special) to heapauxi.o(.text) for __use_two_region_memory
    startup_bat32g137.o(HEAP) refers (Special) to heapauxi.o(.text) for __use_two_region_memory
    startup_bat32g137.o(RESET) refers (Special) to heapauxi.o(.text) for __use_two_region_memory
    startup_bat32g137.o(RESET) refers to startup_bat32g137.o(STACK) for __initial_sp
    startup_bat32g137.o(RESET) refers to startup_bat32g137.o(.text) for Reset_Handler
    startup_bat32g137.o(RESET) refers to sys_tick.o(i.SysTick_Handler) for SysTick_Handler
    startup_bat32g137.o(RESET) refers to sci_user.o(i.IRQ07_Handler) for IRQ07_Handler
    startup_bat32g137.o(RESET) refers to sci_user.o(i.IRQ08_Handler) for IRQ08_Handler
    startup_bat32g137.o(RESET) refers to sci_user.o(i.uart0_interrupt_send) for IRQ10_Handler
    startup_bat32g137.o(RESET) refers to sci_user.o(i.uart0_interrupt_receive) for IRQ11_Handler
    startup_bat32g137.o(.text) refers (Special) to heapauxi.o(.text) for __use_two_region_memory
    startup_bat32g137.o(.text) refers to system_bat32g137.o(i.SystemInit) for SystemInit
    startup_bat32g137.o(.text) refers to __main.o(!!!main) for __main
    startup_bat32g137.o(.text) refers to startup_bat32g137.o(HEAP) for Heap_Mem
    startup_bat32g137.o(.text) refers to startup_bat32g137.o(STACK) for Stack_Mem
    system_bat32g137.o(i.CLK_GetCoreFreq) refers to gpio.o(i.__ARM_common_switch8) for __ARM_common_switch8
    system_bat32g137.o(i.SystemCoreClockUpdate) refers to system_bat32g137.o(i.CLK_GetCoreFreq) for CLK_GetCoreFreq
    system_bat32g137.o(i.SystemCoreClockUpdate) refers to system_bat32g137.o(.data) for SystemCoreClock
    system_bat32g137.o(i.SystemInit) refers to system_bat32g137.o(i.CLK_GetCoreFreq) for CLK_GetCoreFreq
    system_bat32g137.o(i.SystemInit) refers to system_bat32g137.o(.data) for SystemCoreClock
    __main.o(!!!main) refers to __rtentry.o(.ARM.Collect$$rtentry$$00000000) for __rt_entry
    __rtentry.o(.ARM.Collect$$rtentry$$00000000) refers (Special) to __rtentry2.o(.ARM.Collect$$rtentry$$0000000A) for __rt_entry_li
    __rtentry.o(.ARM.Collect$$rtentry$$00000000) refers (Special) to __rtentry2.o(.ARM.Collect$$rtentry$$0000000D) for __rt_entry_main
    __rtentry.o(.ARM.Collect$$rtentry$$00000000) refers (Special) to __rtentry2.o(.ARM.Collect$$rtentry$$0000000C) for __rt_entry_postli_1
    __rtentry.o(.ARM.Collect$$rtentry$$00000000) refers (Special) to __rtentry2.o(.ARM.Collect$$rtentry$$00000009) for __rt_entry_postsh_1
    __rtentry.o(.ARM.Collect$$rtentry$$00000000) refers (Special) to __rtentry2.o(.ARM.Collect$$rtentry$$00000002) for __rt_entry_presh_1
    __rtentry.o(.ARM.Collect$$rtentry$$00000000) refers (Special) to __rtentry4.o(.ARM.Collect$$rtentry$$00000004) for __rt_entry_sh
    aeabi_idiv0_sigfpe.o(.text) refers to rt_div0.o(.text) for __rt_div0
    aeabi_ldiv0_sigfpe.o(.text) refers to rt_div0.o(.text) for __rt_div0
    __rtentry2.o(.ARM.Collect$$rtentry$$00000008) refers to boardinit2.o(.text) for _platform_post_stackheap_init
    __rtentry2.o(.ARM.Collect$$rtentry$$0000000A) refers to libinit.o(.ARM.Collect$$libinit$$00000000) for __rt_lib_init
    __rtentry2.o(.ARM.Collect$$rtentry$$0000000B) refers to boardinit3.o(.text) for _platform_post_lib_init
    __rtentry2.o(.ARM.Collect$$rtentry$$0000000D) refers to main.o(i.main) for main
    __rtentry2.o(.ARM.Collect$$rtentry$$0000000D) refers to exit.o(.text) for exit
    __rtentry2.o(.ARM.exidx) refers to __rtentry2.o(.ARM.Collect$$rtentry$$00000001) for .ARM.Collect$$rtentry$$00000001
    __rtentry2.o(.ARM.exidx) refers to __rtentry2.o(.ARM.Collect$$rtentry$$00000008) for .ARM.Collect$$rtentry$$00000008
    __rtentry2.o(.ARM.exidx) refers to __rtentry2.o(.ARM.Collect$$rtentry$$0000000A) for .ARM.Collect$$rtentry$$0000000A
    __rtentry2.o(.ARM.exidx) refers to __rtentry2.o(.ARM.Collect$$rtentry$$0000000B) for .ARM.Collect$$rtentry$$0000000B
    __rtentry2.o(.ARM.exidx) refers to __rtentry2.o(.ARM.Collect$$rtentry$$0000000D) for .ARM.Collect$$rtentry$$0000000D
    __rtentry4.o(.ARM.Collect$$rtentry$$00000004) refers to sys_stackheap_outer.o(.text) for __user_setup_stackheap
    __rtentry4.o(.ARM.exidx) refers to __rtentry4.o(.ARM.Collect$$rtentry$$00000004) for .ARM.Collect$$rtentry$$00000004
    rt_div0.o(.text) refers to defsig_fpe_outer.o(.text) for __rt_SIGFPE
    sys_stackheap_outer.o(.text) refers to libspace.o(.text) for __user_perproc_libspace
    sys_stackheap_outer.o(.text) refers to startup_bat32g137.o(.text) for __user_initial_stackheap
    sys_stackheap_outer.o(__vectab_stack_and_reset_area) refers to tempstk.o(.text) for __temporary_stack_top
    sys_stackheap_outer.o(__vectab_stack_and_reset_area) refers to __main.o(!!!main) for __main
    exit.o(.text) refers to rtexit.o(.ARM.Collect$$rtexit$$00000000) for __rt_exit
    defsig_fpe_outer.o(.text) refers to defsig_fpe_inner.o(.text) for __rt_SIGFPE_inner
    defsig_fpe_outer.o(.text) refers to defsig_exit.o(.text) for __sig_exit
    defsig_fpe_formal.o(.text) refers to rt_raise.o(.text) for __rt_raise
    libinit.o(.ARM.Collect$$libinit$$00000000) refers (Special) to libinit2.o(.ARM.Collect$$libinit$$0000002E) for __rt_lib_init_alloca_1
    libinit.o(.ARM.Collect$$libinit$$00000000) refers (Special) to libinit2.o(.ARM.Collect$$libinit$$0000002C) for __rt_lib_init_argv_1
    libinit.o(.ARM.Collect$$libinit$$00000000) refers (Special) to libinit2.o(.ARM.Collect$$libinit$$0000001B) for __rt_lib_init_atexit_1
    libinit.o(.ARM.Collect$$libinit$$00000000) refers (Special) to libinit2.o(.ARM.Collect$$libinit$$00000021) for __rt_lib_init_clock_1
    libinit.o(.ARM.Collect$$libinit$$00000000) refers (Special) to libinit2.o(.ARM.Collect$$libinit$$00000032) for __rt_lib_init_cpp_1
    libinit.o(.ARM.Collect$$libinit$$00000000) refers (Special) to libinit2.o(.ARM.Collect$$libinit$$00000030) for __rt_lib_init_exceptions_1
    libinit.o(.ARM.Collect$$libinit$$00000000) refers (Special) to libinit2.o(.ARM.Collect$$libinit$$00000002) for __rt_lib_init_fp_1
    libinit.o(.ARM.Collect$$libinit$$00000000) refers (Special) to libinit2.o(.ARM.Collect$$libinit$$0000001F) for __rt_lib_init_fp_trap_1
    libinit.o(.ARM.Collect$$libinit$$00000000) refers (Special) to libinit2.o(.ARM.Collect$$libinit$$00000023) for __rt_lib_init_getenv_1
    libinit.o(.ARM.Collect$$libinit$$00000000) refers (Special) to libinit2.o(.ARM.Collect$$libinit$$0000000A) for __rt_lib_init_heap_1
    libinit.o(.ARM.Collect$$libinit$$00000000) refers (Special) to libinit2.o(.ARM.Collect$$libinit$$00000011) for __rt_lib_init_lc_collate_1
    libinit.o(.ARM.Collect$$libinit$$00000000) refers (Special) to libinit2.o(.ARM.Collect$$libinit$$00000013) for __rt_lib_init_lc_ctype_1
    libinit.o(.ARM.Collect$$libinit$$00000000) refers (Special) to libinit2.o(.ARM.Collect$$libinit$$00000015) for __rt_lib_init_lc_monetary_1
    libinit.o(.ARM.Collect$$libinit$$00000000) refers (Special) to libinit2.o(.ARM.Collect$$libinit$$00000017) for __rt_lib_init_lc_numeric_1
    libinit.o(.ARM.Collect$$libinit$$00000000) refers (Special) to libinit2.o(.ARM.Collect$$libinit$$00000019) for __rt_lib_init_lc_time_1
    libinit.o(.ARM.Collect$$libinit$$00000000) refers (Special) to libinit2.o(.ARM.Collect$$libinit$$00000004) for __rt_lib_init_preinit_1
    libinit.o(.ARM.Collect$$libinit$$00000000) refers (Special) to libinit2.o(.ARM.Collect$$libinit$$0000000E) for __rt_lib_init_rand_1
    libinit.o(.ARM.Collect$$libinit$$00000000) refers (Special) to libinit2.o(.ARM.Collect$$libinit$$00000033) for __rt_lib_init_return
    libinit.o(.ARM.Collect$$libinit$$00000000) refers (Special) to libinit2.o(.ARM.Collect$$libinit$$0000001D) for __rt_lib_init_signal_1
    libinit.o(.ARM.Collect$$libinit$$00000000) refers (Special) to libinit2.o(.ARM.Collect$$libinit$$00000025) for __rt_lib_init_stdio_1
    libinit.o(.ARM.Collect$$libinit$$00000000) refers (Special) to libinit2.o(.ARM.Collect$$libinit$$0000000C) for __rt_lib_init_user_alloc_1
    libspace.o(.text) refers to libspace.o(.bss) for __libspace_start
    rtexit.o(.ARM.Collect$$rtexit$$00000000) refers (Special) to rtexit2.o(.ARM.Collect$$rtexit$$00000004) for __rt_exit_exit
    rtexit.o(.ARM.Collect$$rtexit$$00000000) refers (Special) to rtexit2.o(.ARM.Collect$$rtexit$$00000003) for __rt_exit_ls
    rtexit.o(.ARM.Collect$$rtexit$$00000000) refers (Special) to rtexit2.o(.ARM.Collect$$rtexit$$00000002) for __rt_exit_prels_1
    rtexit.o(.ARM.exidx) refers (Special) to rtexit2.o(.ARM.Collect$$rtexit$$00000004) for __rt_exit_exit
    rtexit.o(.ARM.exidx) refers (Special) to rtexit2.o(.ARM.Collect$$rtexit$$00000003) for __rt_exit_ls
    rtexit.o(.ARM.exidx) refers (Special) to rtexit2.o(.ARM.Collect$$rtexit$$00000002) for __rt_exit_prels_1
    rtexit.o(.ARM.exidx) refers to rtexit.o(.ARM.Collect$$rtexit$$00000000) for .ARM.Collect$$rtexit$$00000000
    rt_raise.o(.text) refers to __raise.o(.text) for __raise
    rt_raise.o(.text) refers to sys_exit.o(.text) for _sys_exit
    defsig_exit.o(.text) refers to sys_exit.o(.text) for _sys_exit
    defsig_fpe_inner.o(.text) refers to defsig_general.o(.text) for __default_signal_display
    libinit2.o(.ARM.Collect$$libinit$$00000010) refers to libinit2.o(.ARM.Collect$$libinit$$0000000F) for .ARM.Collect$$libinit$$0000000F
    libinit2.o(.ARM.Collect$$libinit$$00000012) refers to libinit2.o(.ARM.Collect$$libinit$$0000000F) for .ARM.Collect$$libinit$$0000000F
    libinit2.o(.ARM.Collect$$libinit$$00000014) refers to libinit2.o(.ARM.Collect$$libinit$$0000000F) for .ARM.Collect$$libinit$$0000000F
    libinit2.o(.ARM.Collect$$libinit$$00000016) refers to libinit2.o(.ARM.Collect$$libinit$$0000000F) for .ARM.Collect$$libinit$$0000000F
    libinit2.o(.ARM.Collect$$libinit$$00000018) refers to libinit2.o(.ARM.Collect$$libinit$$0000000F) for .ARM.Collect$$libinit$$0000000F
    libinit2.o(.ARM.Collect$$libinit$$00000026) refers to argv_veneer.o(.text) for __ARM_argv_veneer
    libinit2.o(.ARM.Collect$$libinit$$00000027) refers to argv_veneer.o(.text) for __ARM_argv_veneer
    sys_exit.o(.text) refers (Special) to use_no_semi.o(.text) for __I$use$semihosting
    sys_exit.o(.text) refers (Special) to indicate_semi.o(.text) for __semihosting_library_function
    rtexit2.o(.ARM.Collect$$rtexit$$00000003) refers to libshutdown.o(.ARM.Collect$$libshutdown$$00000000) for __rt_lib_shutdown
    rtexit2.o(.ARM.Collect$$rtexit$$00000004) refers to sys_exit.o(.text) for _sys_exit
    rtexit2.o(.ARM.exidx) refers to rtexit2.o(.ARM.Collect$$rtexit$$00000001) for .ARM.Collect$$rtexit$$00000001
    rtexit2.o(.ARM.exidx) refers to rtexit2.o(.ARM.Collect$$rtexit$$00000003) for .ARM.Collect$$rtexit$$00000003
    rtexit2.o(.ARM.exidx) refers to rtexit2.o(.ARM.Collect$$rtexit$$00000004) for .ARM.Collect$$rtexit$$00000004
    __raise.o(.text) refers to defsig.o(CL$$defsig) for __default_signal_handler
    defsig_general.o(.text) refers to sys_wrch.o(.text) for _ttywrch
    sys_wrch.o(.text) refers (Special) to use_no_semi.o(.text) for __I$use$semihosting
    sys_wrch.o(.text) refers (Special) to indicate_semi.o(.text) for __semihosting_library_function
    defsig.o(CL$$defsig) refers to defsig_fpe_inner.o(.text) for __rt_SIGFPE_inner
    defsig.o(CL$$defsig) refers to defsig_rtmem_inner.o(.text) for __rt_SIGRTMEM_inner
    _get_argv_nomalloc.o(.text) refers (Special) to hrguard.o(.text) for __heap_region$guard
    _get_argv_nomalloc.o(.text) refers to defsig_rtmem_outer.o(.text) for __rt_SIGRTMEM
    _get_argv_nomalloc.o(.text) refers to sys_command.o(.text) for _sys_command_string
    libshutdown.o(.ARM.Collect$$libshutdown$$00000000) refers (Special) to libshutdown2.o(.ARM.Collect$$libshutdown$$00000004) for __rt_lib_shutdown_cpp_1
    libshutdown.o(.ARM.Collect$$libshutdown$$00000000) refers (Special) to libshutdown2.o(.ARM.Collect$$libshutdown$$00000002) for __rt_lib_shutdown_fini_1
    libshutdown.o(.ARM.Collect$$libshutdown$$00000000) refers (Special) to libshutdown2.o(.ARM.Collect$$libshutdown$$00000009) for __rt_lib_shutdown_fp_trap_1
    libshutdown.o(.ARM.Collect$$libshutdown$$00000000) refers (Special) to libshutdown2.o(.ARM.Collect$$libshutdown$$00000011) for __rt_lib_shutdown_heap_1
    libshutdown.o(.ARM.Collect$$libshutdown$$00000000) refers (Special) to libshutdown2.o(.ARM.Collect$$libshutdown$$00000012) for __rt_lib_shutdown_return
    libshutdown.o(.ARM.Collect$$libshutdown$$00000000) refers (Special) to libshutdown2.o(.ARM.Collect$$libshutdown$$0000000C) for __rt_lib_shutdown_signal_1
    libshutdown.o(.ARM.Collect$$libshutdown$$00000000) refers (Special) to libshutdown2.o(.ARM.Collect$$libshutdown$$00000006) for __rt_lib_shutdown_stdio_1
    libshutdown.o(.ARM.Collect$$libshutdown$$00000000) refers (Special) to libshutdown2.o(.ARM.Collect$$libshutdown$$0000000E) for __rt_lib_shutdown_user_alloc_1
    sys_command.o(.text) refers (Special) to use_no_semi.o(.text) for __I$use$semihosting
    sys_command.o(.text) refers (Special) to indicate_semi.o(.text) for __semihosting_library_function
    defsig_abrt_inner.o(.text) refers to defsig_general.o(.text) for __default_signal_display
    defsig_rtred_inner.o(.text) refers to defsig_general.o(.text) for __default_signal_display
    defsig_rtmem_inner.o(.text) refers to defsig_general.o(.text) for __default_signal_display
    defsig_rtmem_outer.o(.text) refers to defsig_rtmem_inner.o(.text) for __rt_SIGRTMEM_inner
    defsig_rtmem_outer.o(.text) refers to defsig_exit.o(.text) for __sig_exit
    defsig_rtmem_formal.o(.text) refers to rt_raise.o(.text) for __rt_raise
    defsig_stak_inner.o(.text) refers to defsig_general.o(.text) for __default_signal_display
    defsig_pvfn_inner.o(.text) refers to defsig_general.o(.text) for __default_signal_display
    defsig_cppl_inner.o(.text) refers to defsig_general.o(.text) for __default_signal_display
    defsig_segv_inner.o(.text) refers to defsig_general.o(.text) for __default_signal_display
    defsig_other.o(.text) refers to defsig_general.o(.text) for __default_signal_display


==============================================================================

Removing Unused input sections from the image.

    Removing gpio.o(.rev16_text), (4 bytes).
    Removing gpio.o(.revsh_text), (4 bytes).
    Removing gpio.o(i.GPIO_Get_Value), (6 bytes).
    Removing gpio.o(i.GPIO_Input_Enable), (32 bytes).
    Removing gpio.o(i.GPIO_Nch_OpenDrain), (20 bytes).
    Removing gpio.o(i.GPIO_Output_Enable), (32 bytes).
    Removing gpio.o(i.GPIO_PullUp_Disable), (20 bytes).
    Removing gpio.o(i.GPIO_PullUp_Enable), (20 bytes).
    Removing gpio.o(i.GPIO_Set_Value), (4 bytes).
    Removing gpio.o(i.GPIO_Ttl_Input), (20 bytes).
    Removing gpio.o(i.PORT_ToggleBit), (36 bytes).
    Removing wdt.o(.rev16_text), (4 bytes).
    Removing wdt.o(.revsh_text), (4 bytes).
    Removing sys_tick.o(.rev16_text), (4 bytes).
    Removing sys_tick.o(.revsh_text), (4 bytes).
    Removing sys_tick.o(i.Sys_Tick_Timer_Stop), (20 bytes).
    Removing adc.o(.rev16_text), (4 bytes).
    Removing adc.o(.revsh_text), (4 bytes).
    Removing adc.o(i.ADC_Converse), (128 bytes).
    Removing adc.o(i.ADC_MidAvg_Filter), (116 bytes).
    Removing adc.o(i.ADC_SelfTest), (152 bytes).
    Removing adc.o(i.ADC_Set_Clock), (36 bytes).
    Removing adc.o(i.ADC_Set_HardTrigger), (52 bytes).
    Removing adc.o(i.ADC_Set_OperationOff), (20 bytes).
    Removing adc.o(i.ADC_Set_OperationOn), (20 bytes).
    Removing adc.o(i.ADC_Set_RefVoltage), (60 bytes).
    Removing adc.o(i.INTC_GetPendingIRQ), (68 bytes).
    Removing analog_circuits.o(.rev16_text), (4 bytes).
    Removing analog_circuits.o(.revsh_text), (4 bytes).
    Removing analog_circuits.o(i.ADC_Res_Calc_Circuit101), (172 bytes).
    Removing analog_circuits.o(i.ADC_Res_Calc_Circuit102), (304 bytes).
    Removing analog_circuits.o(i.ADC_Res_Calc_Circuit103), (368 bytes).
    Removing analog_circuits.o(i.ADC_Res_Calc_Circuit201), (176 bytes).
    Removing analog_circuits.o(i.ADC_Res_Calc_Circuit202), (248 bytes).
    Removing analog_circuits.o(i.ADC_Res_Calc_Circuit203), (324 bytes).
    Removing analog_circuits.o(i.ADC_Res_Calc_Circuit301), (96 bytes).
    Removing analog_circuits.o(i.ADC_Res_Calc_Circuit302), (136 bytes).
    Removing analog_circuits.o(i.ADC_Res_Calc_Circuit303), (232 bytes).
    Removing analog_circuits.o(i.ADC_VRef_Calibrate), (60 bytes).
    Removing analog_circuits.o(i.ADC_Voltage_Calc_Circuit101), (22 bytes).
    Removing analog_signals.o(.rev16_text), (4 bytes).
    Removing analog_signals.o(.revsh_text), (4 bytes).
    Removing analog_signals.o(i.Analog_Signal_Conv_Stop), (60 bytes).
    Removing sci.o(.rev16_text), (4 bytes).
    Removing sci.o(.revsh_text), (4 bytes).
    Removing sci.o(i.IIC00_Init), (208 bytes).
    Removing sci.o(i.IIC00_MasterReceive), (124 bytes).
    Removing sci.o(i.IIC00_MasterSend), (112 bytes).
    Removing sci.o(i.IIC00_StartCondition), (88 bytes).
    Removing sci.o(i.IIC00_Stop), (32 bytes).
    Removing sci.o(i.IIC00_StopCondition), (108 bytes).
    Removing sci.o(i.IIC01_Init), (172 bytes).
    Removing sci.o(i.IIC01_MasterReceive), (116 bytes).
    Removing sci.o(i.IIC01_MasterSend), (104 bytes).
    Removing sci.o(i.IIC01_StartCondition), (92 bytes).
    Removing sci.o(i.IIC01_Stop), (32 bytes).
    Removing sci.o(i.IIC01_StopCondition), (100 bytes).
    Removing sci.o(i.IIC10_Init), (212 bytes).
    Removing sci.o(i.IIC10_MasterReceive), (124 bytes).
    Removing sci.o(i.IIC10_MasterSend), (112 bytes).
    Removing sci.o(i.IIC10_StartCondition), (92 bytes).
    Removing sci.o(i.IIC10_Stop), (32 bytes).
    Removing sci.o(i.IIC10_StopCondition), (108 bytes).
    Removing sci.o(i.IIC11_Init), (216 bytes).
    Removing sci.o(i.IIC11_MasterReceive), (116 bytes).
    Removing sci.o(i.IIC11_MasterSend), (104 bytes).
    Removing sci.o(i.IIC11_StartCondition), (92 bytes).
    Removing sci.o(i.IIC11_Stop), (32 bytes).
    Removing sci.o(i.IIC11_StopCondition), (100 bytes).
    Removing sci.o(i.IIC20_Init), (208 bytes).
    Removing sci.o(i.IIC20_MasterReceive), (124 bytes).
    Removing sci.o(i.IIC20_MasterSend), (112 bytes).
    Removing sci.o(i.IIC20_StartCondition), (88 bytes).
    Removing sci.o(i.IIC20_Stop), (32 bytes).
    Removing sci.o(i.IIC20_StopCondition), (108 bytes).
    Removing sci.o(i.IIC21_Init), (172 bytes).
    Removing sci.o(i.IIC21_MasterReceive), (116 bytes).
    Removing sci.o(i.IIC21_MasterSend), (104 bytes).
    Removing sci.o(i.IIC21_StartCondition), (92 bytes).
    Removing sci.o(i.IIC21_Stop), (32 bytes).
    Removing sci.o(i.IIC21_StopCondition), (100 bytes).
    Removing sci.o(i.INTC_GetPendingIRQ), (68 bytes).
    Removing sci.o(i.SPI00_MasterInit), (336 bytes).
    Removing sci.o(i.SPI00_MasterReceive), (216 bytes).
    Removing sci.o(i.SPI00_MasterSend), (200 bytes).
    Removing sci.o(i.SPI00_MasterSendReceive), (240 bytes).
    Removing sci.o(i.SPI00_SlaveInit), (244 bytes).
    Removing sci.o(i.SPI00_SlaveReceive), (164 bytes).
    Removing sci.o(i.SPI00_SlaveSend), (196 bytes).
    Removing sci.o(i.SPI00_Start), (72 bytes).
    Removing sci.o(i.SPI00_Stop), (68 bytes).
    Removing sci.o(i.SPI01_MasterInit), (284 bytes).
    Removing sci.o(i.SPI01_MasterReceive), (88 bytes).
    Removing sci.o(i.SPI01_MasterSend), (104 bytes).
    Removing sci.o(i.SPI01_SlaveInit), (168 bytes).
    Removing sci.o(i.SPI01_SlaveReceive), (88 bytes).
    Removing sci.o(i.SPI01_SlaveSend), (104 bytes).
    Removing sci.o(i.SPI01_SlaveSendReceive), (108 bytes).
    Removing sci.o(i.SPI01_Start), (72 bytes).
    Removing sci.o(i.SPI01_Stop), (76 bytes).
    Removing sci.o(i.SPI10_MasterInit), (364 bytes).
    Removing sci.o(i.SPI10_MasterReceive), (228 bytes).
    Removing sci.o(i.SPI10_MasterSend), (196 bytes).
    Removing sci.o(i.SPI10_MasterSendReceive), (248 bytes).
    Removing sci.o(i.SPI10_SlaveInit), (224 bytes).
    Removing sci.o(i.SPI10_SlaveReceive), (164 bytes).
    Removing sci.o(i.SPI10_SlaveSend), (192 bytes).
    Removing sci.o(i.SPI10_Start), (72 bytes).
    Removing sci.o(i.SPI10_Stop), (76 bytes).
    Removing sci.o(i.SPI11_MasterInit), (364 bytes).
    Removing sci.o(i.SPI11_MasterReceive), (236 bytes).
    Removing sci.o(i.SPI11_MasterSend), (200 bytes).
    Removing sci.o(i.SPI11_SlaveInit), (224 bytes).
    Removing sci.o(i.SPI11_SlaveReceive), (168 bytes).
    Removing sci.o(i.SPI11_SlaveSend), (200 bytes).
    Removing sci.o(i.SPI11_SlaveSendReceive), (236 bytes).
    Removing sci.o(i.SPI11_Start), (72 bytes).
    Removing sci.o(i.SPI11_Stop), (76 bytes).
    Removing sci.o(i.SPI20_MasterInit), (336 bytes).
    Removing sci.o(i.SPI20_MasterReceive), (72 bytes).
    Removing sci.o(i.SPI20_MasterSend), (68 bytes).
    Removing sci.o(i.SPI20_SlaveInit), (224 bytes).
    Removing sci.o(i.SPI20_SlaveReceive), (88 bytes).
    Removing sci.o(i.SPI20_SlaveSend), (104 bytes).
    Removing sci.o(i.SPI20_Start), (72 bytes).
    Removing sci.o(i.SPI20_Stop), (68 bytes).
    Removing sci.o(i.SPI21_MasterInit), (268 bytes).
    Removing sci.o(i.SPI21_MasterReceive), (88 bytes).
    Removing sci.o(i.SPI21_MasterSend), (108 bytes).
    Removing sci.o(i.SPI21_MasterSendReceive), (112 bytes).
    Removing sci.o(i.SPI21_SlaveInit), (168 bytes).
    Removing sci.o(i.SPI21_SlaveReceive), (88 bytes).
    Removing sci.o(i.SPI21_SlaveSend), (104 bytes).
    Removing sci.o(i.SPI21_Start), (72 bytes).
    Removing sci.o(i.SPI21_Stop), (68 bytes).
    Removing sci.o(i.UART0_BaudRate), (100 bytes).
    Removing sci.o(i.UART0_Init), (260 bytes).
    Removing sci.o(i.UART0_Receive), (28 bytes).
    Removing sci.o(i.UART0_Send), (28 bytes).
    Removing sci.o(i.UART1_BaudRate), (80 bytes).
    Removing sci.o(i.UART1_Init), (312 bytes).
    Removing sci.o(i.UART1_Receive), (44 bytes).
    Removing sci.o(i.UART1_Send), (68 bytes).
    Removing sci.o(i.UART1_Start), (80 bytes).
    Removing sci.o(i.UART1_Stop), (60 bytes).
    Removing sci.o(i.UART2_Receive), (44 bytes).
    Removing sci.o(i.UART2_Send), (68 bytes).
    Removing sci.o(i.UART2_Stop), (60 bytes).
    Removing sci.o(i.__NVIC_SetPriority), (120 bytes).
    Removing sci_user.o(.rev16_text), (4 bytes).
    Removing sci_user.o(.revsh_text), (4 bytes).
    Removing main.o(.rev16_text), (4 bytes).
    Removing main.o(.revsh_text), (4 bytes).
    Removing tasks.o(.rev16_text), (4 bytes).
    Removing tasks.o(.revsh_text), (4 bytes).
    Removing tasks.o(i.APP_Startup_Init), (2 bytes).
    Removing tasks.o(i.Sys_Sleep_Mode_Tasks), (2 bytes).
    Removing sys_scheduler.o(.rev16_text), (4 bytes).
    Removing sys_scheduler.o(.revsh_text), (4 bytes).
    Removing init.o(.rev16_text), (4 bytes).
    Removing init.o(.revsh_text), (4 bytes).
    Removing init.o(i.Sys_Sleep_Init), (2 bytes).
    Removing init.o(i.Sys_Startup_Pre_Init), (2 bytes).
    Removing init.o(i.Sys_Wakeup_Init), (2 bytes).
    Removing line_in.o(.rev16_text), (4 bytes).
    Removing line_in.o(.revsh_text), (4 bytes).
    Removing line_in.o(i.Line_In_Get_Status), (16 bytes).
    Removing line_in.o(i.Line_In_SetPowerSt), (12 bytes).
    Removing powermanagement.o(i.Get_PwrLibVersion), (4 bytes).
    Removing powermanagement_user.o(.rev16_text), (4 bytes).
    Removing powermanagement_user.o(.revsh_text), (4 bytes).
    Removing system_monitor.o(.rev16_text), (4 bytes).
    Removing system_monitor.o(.revsh_text), (4 bytes).
    Removing system_monitor.o(i.Read_KL30_ConvertFinish), (12 bytes).
    Removing system_monitor.o(i.Sys_Status_Update_Service), (16 bytes).
    Removing system_monitor.o(i.System_Calc_FunRange), (36 bytes).
    Removing system_monitor.o(i.System_Calc_NMRange), (36 bytes).
    Removing system_monitor.o(i.System_FUN_KL15_Status_Get), (12 bytes).
    Removing system_monitor.o(i.System_Fun_Process), (384 bytes).
    Removing system_monitor.o(i.System_NM_KL15_Status_Get), (12 bytes).
    Removing system_monitor.o(i.System_NM_KL30_Status_Get), (12 bytes).
    Removing system_monitor.o(i.System_NM_Process), (364 bytes).
    Removing system_monitor_user.o(.rev16_text), (4 bytes).
    Removing system_monitor_user.o(.revsh_text), (4 bytes).
    Removing system_monitor_user.o(i.Sys_Read_KL15_Valid), (12 bytes).
    Removing system_monitor_user.o(i.Sys_Read_KL15_Voltage), (12 bytes).
    Removing system_monitor_user.o(i.Sys_Read_KL30_Valid), (12 bytes).
    Removing system_monitor_user.o(i.Sys_Read_KL30_Voltage), (12 bytes).
    Removing rte_adc.o(.rev16_text), (4 bytes).
    Removing rte_adc.o(.revsh_text), (4 bytes).
    Removing rte_adc.o(i.RTE_ADC_Init), (8 bytes).
    Removing rte_adc.o(i.RTE_ForceRead_FUEL1_1_Voltage), (16 bytes).
    Removing rte_adc.o(i.RTE_ForceRead_FUEL1_2_Voltage), (16 bytes).
    Removing rte_adc.o(i.RTE_ForceRead_FUEL2_2_Voltage), (16 bytes).
    Removing rte_adc.o(i.RTE_Read_FUEL1_1_Valid), (16 bytes).
    Removing rte_adc.o(i.RTE_Read_FUEL1_1_Voltage), (16 bytes).
    Removing rte_adc.o(i.RTE_Read_FUEL1_2_Valid), (16 bytes).
    Removing rte_adc.o(i.RTE_Read_FUEL1_2_Voltage), (16 bytes).
    Removing rte_adc.o(i.RTE_Read_FUEL2_2_Valid), (16 bytes).
    Removing rte_adc.o(i.RTE_Read_FUEL2_2_Voltage), (16 bytes).
    Removing rte_adc.o(i.RTE_Read_KL15_Valid), (16 bytes).
    Removing rte_adc.o(i.RTE_Read_KL15_Voltage), (16 bytes).
    Removing rte_adc.o(i.RTE_Read_KL30_Valid), (16 bytes).
    Removing rte_adc.o(i.RTE_Read_KL30_Voltage), (16 bytes).
    Removing common_interface.o(.rev16_text), (4 bytes).
    Removing common_interface.o(.revsh_text), (4 bytes).
    Removing common_interface.o(i.Common_BlockDelay), (56 bytes).
    Removing common_interface.o(i.Common_DataInit), (108 bytes).
    Removing common_interface.o(i.Common_GetIgnOffTime), (12 bytes).
    Removing common_interface.o(i.Common_GetIgnOnTime), (12 bytes).
    Removing common_interface.o(i.Common_Get_Act_E_Speed), (12 bytes).
    Removing common_interface.o(i.Common_Get_Act_E_Speed_Valid), (12 bytes).
    Removing common_interface.o(i.Common_Get_Act_V_Speed), (12 bytes).
    Removing common_interface.o(i.Common_Get_Act_V_Speed_Valid), (12 bytes).
    Removing common_interface.o(i.Common_Get_DispSpeed), (52 bytes).
    Removing common_interface.o(i.Common_Get_Disp_E_Speed), (12 bytes).
    Removing common_interface.o(i.Common_Get_Disp_E_Speed_Valid), (12 bytes).
    Removing common_interface.o(i.Common_Get_Disp_V_Speed), (12 bytes).
    Removing common_interface.o(i.Common_Get_Disp_V_Speed_Valid), (12 bytes).
    Removing common_interface.o(i.Common_Input_Para), (2 bytes).
    Removing common_interface.o(i.Common_ReadRollingCounter), (12 bytes).
    Removing common_interface.o(i.Common_RollingCounterAdd), (16 bytes).
    Removing common_interface.o(i.Common_RollingCounterClear), (12 bytes).
    Removing common_interface.o(i.Common_Set_Act_E_Speed), (12 bytes).
    Removing common_interface.o(i.Common_Set_Act_E_Speed_Valid), (12 bytes).
    Removing common_interface.o(i.Common_Set_Act_V_Speed), (12 bytes).
    Removing common_interface.o(i.Common_Set_Act_V_Speed_Valid), (12 bytes).
    Removing common_interface.o(i.Common_Set_Disp_E_Speed), (12 bytes).
    Removing common_interface.o(i.Common_Set_Disp_E_Speed_Valid), (12 bytes).
    Removing common_interface.o(i.Common_Set_Disp_V_Speed), (12 bytes).
    Removing common_interface.o(i.Common_Set_Disp_V_Speed_Valid), (12 bytes).
    Removing common_interface.o(i.Common_Set_IG_Sts), (12 bytes).
    Removing common_interface.o(i.Common_Set_IG_Sts_Valid), (12 bytes).
    Removing mcu_core_protocol.o(.rev16_text), (4 bytes).
    Removing mcu_core_protocol.o(.revsh_text), (4 bytes).
    Removing system_bat32g137.o(.rev16_text), (4 bytes).
    Removing system_bat32g137.o(.revsh_text), (4 bytes).
    Removing system_bat32g137.o(i.CLK_GetHocoFreq), (64 bytes).

238 unused section(s) (total 18784 bytes) removed from the image.

==============================================================================

Image Symbol Table

    Local Symbols

    Symbol Name                              Value     Ov Type        Size  Object(Section)

    RESET                                    0x00000000   Section      192  startup_bat32g137.o(RESET)
    ../clib/../cmprslib/zerorunl2.c          0x00000000   Number         0  __dczerorl2.o ABSOLUTE
    ../clib/angel/boardlib.s                 0x00000000   Number         0  boardshut.o ABSOLUTE
    ../clib/angel/boardlib.s                 0x00000000   Number         0  boardinit3.o ABSOLUTE
    ../clib/angel/boardlib.s                 0x00000000   Number         0  boardinit2.o ABSOLUTE
    ../clib/angel/boardlib.s                 0x00000000   Number         0  boardinit1.o ABSOLUTE
    ../clib/angel/handlers.s                 0x00000000   Number         0  __scatter_zi.o ABSOLUTE
    ../clib/angel/kernel.s                   0x00000000   Number         0  __rtentry.o ABSOLUTE
    ../clib/angel/kernel.s                   0x00000000   Number         0  rtexit2.o ABSOLUTE
    ../clib/angel/kernel.s                   0x00000000   Number         0  rtexit.o ABSOLUTE
    ../clib/angel/kernel.s                   0x00000000   Number         0  __rtentry2.o ABSOLUTE
    ../clib/angel/kernel.s                   0x00000000   Number         0  __rtentry4.o ABSOLUTE
    ../clib/angel/rt.s                       0x00000000   Number         0  rt_div0.o ABSOLUTE
    ../clib/angel/rt.s                       0x00000000   Number         0  rt_raise.o ABSOLUTE
    ../clib/angel/rt.s                       0x00000000   Number         0  aeabi_idiv0.o ABSOLUTE
    ../clib/angel/rt.s                       0x00000000   Number         0  aeabi_idiv0_sigfpe.o ABSOLUTE
    ../clib/angel/rt.s                       0x00000000   Number         0  aeabi_ldiv0.o ABSOLUTE
    ../clib/angel/rt.s                       0x00000000   Number         0  aeabi_ldiv0_sigfpe.o ABSOLUTE
    ../clib/angel/scatterp.s                 0x00000000   Number         0  __scatter.o ABSOLUTE
    ../clib/angel/startup.s                  0x00000000   Number         0  __main.o ABSOLUTE
    ../clib/angel/sys.s                      0x00000000   Number         0  indicate_semi.o ABSOLUTE
    ../clib/angel/sys.s                      0x00000000   Number         0  libspace.o ABSOLUTE
    ../clib/angel/sys.s                      0x00000000   Number         0  use_no_semi.o ABSOLUTE
    ../clib/angel/sys.s                      0x00000000   Number         0  tempstk.o ABSOLUTE
    ../clib/angel/sys.s                      0x00000000   Number         0  sys_stackheap_outer.o ABSOLUTE
    ../clib/angel/sysapp.c                   0x00000000   Number         0  sys_command.o ABSOLUTE
    ../clib/angel/sysapp.c                   0x00000000   Number         0  sys_exit.o ABSOLUTE
    ../clib/angel/sysapp.c                   0x00000000   Number         0  sys_wrch.o ABSOLUTE
    ../clib/armsys.c                         0x00000000   Number         0  _get_argv_nomalloc.o ABSOLUTE
    ../clib/armsys.c                         0x00000000   Number         0  argv_veneer.o ABSOLUTE
    ../clib/armsys.c                         0x00000000   Number         0  no_argv.o ABSOLUTE
    ../clib/division.c                       0x00000000   Number         0  lludiv.o ABSOLUTE
    ../clib/division.s                       0x00000000   Number         0  aeabi_sdiv.o ABSOLUTE
    ../clib/division.s                       0x00000000   Number         0  aeabi_sdiv_div0.o ABSOLUTE
    ../clib/heapalloc.c                      0x00000000   Number         0  hrguard.o ABSOLUTE
    ../clib/heapaux.c                        0x00000000   Number         0  heapauxi.o ABSOLUTE
    ../clib/libinit.s                        0x00000000   Number         0  libshutdown2.o ABSOLUTE
    ../clib/libinit.s                        0x00000000   Number         0  libinit2.o ABSOLUTE
    ../clib/libinit.s                        0x00000000   Number         0  libinit.o ABSOLUTE
    ../clib/libinit.s                        0x00000000   Number         0  libshutdown.o ABSOLUTE
    ../clib/longlong.c                       0x00000000   Number         0  llmul.o ABSOLUTE
    ../clib/signal.c                         0x00000000   Number         0  defsig_fpe_outer.o ABSOLUTE
    ../clib/signal.c                         0x00000000   Number         0  defsig_fpe_formal.o ABSOLUTE
    ../clib/signal.c                         0x00000000   Number         0  defsig_exit.o ABSOLUTE
    ../clib/signal.c                         0x00000000   Number         0  defsig_other.o ABSOLUTE
    ../clib/signal.c                         0x00000000   Number         0  defsig_segv_inner.o ABSOLUTE
    ../clib/signal.c                         0x00000000   Number         0  defsig_cppl_inner.o ABSOLUTE
    ../clib/signal.c                         0x00000000   Number         0  defsig_pvfn_inner.o ABSOLUTE
    ../clib/signal.c                         0x00000000   Number         0  defsig_stak_inner.o ABSOLUTE
    ../clib/signal.c                         0x00000000   Number         0  defsig_rtmem_formal.o ABSOLUTE
    ../clib/signal.c                         0x00000000   Number         0  defsig_fpe_inner.o ABSOLUTE
    ../clib/signal.c                         0x00000000   Number         0  defsig_rtmem_inner.o ABSOLUTE
    ../clib/signal.c                         0x00000000   Number         0  defsig_rtred_inner.o ABSOLUTE
    ../clib/signal.c                         0x00000000   Number         0  defsig_abrt_inner.o ABSOLUTE
    ../clib/signal.c                         0x00000000   Number         0  defsig_general.o ABSOLUTE
    ../clib/signal.c                         0x00000000   Number         0  __raise.o ABSOLUTE
    ../clib/signal.c                         0x00000000   Number         0  defsig_rtmem_outer.o ABSOLUTE
    ../clib/signal.s                         0x00000000   Number         0  defsig.o ABSOLUTE
    ../clib/stdlib.c                         0x00000000   Number         0  exit.o ABSOLUTE
    ../fplib/cfplib/fpinit.c                 0x00000000   Number         0  fpinit.o ABSOLUTE
    RTE\Device\BAT32G137GH64FB\startup_BAT32G137.s 0x00000000   Number         0  startup_bat32g137.o ABSOLUTE
    RTE\Device\BAT32G137GH64FB\system_BAT32G137.c 0x00000000   Number         0  system_bat32g137.o ABSOLUTE
    RTE\\Device\\BAT32G137GH64FB\\system_BAT32G137.c 0x00000000   Number         0  system_bat32g137.o ABSOLUTE
    dc.s                                     0x00000000   Number         0  dc.o ABSOLUTE
    source\Application\LINE_IN\Line_In.c     0x00000000   Number         0  line_in.o ABSOLUTE
    source\Application\MCU_Core_Protocol\MCU_Core_Protocol.c 0x00000000   Number         0  mcu_core_protocol.o ABSOLUTE
    source\Application\PowerManagement\PowerManagement.c 0x00000000   Number         0  powermanagement.o ABSOLUTE
    source\Application\PowerManagement\PowerManagement_user.c 0x00000000   Number         0  powermanagement_user.o ABSOLUTE
    source\Application\PowerManagement\System_Monitor.c 0x00000000   Number         0  system_monitor.o ABSOLUTE
    source\Application\PowerManagement\System_Monitor_user.c 0x00000000   Number         0  system_monitor_user.o ABSOLUTE
    source\Application\RTE\Common_Interface.c 0x00000000   Number         0  common_interface.o ABSOLUTE
    source\Application\RTE\RTE_ADC.c         0x00000000   Number         0  rte_adc.o ABSOLUTE
    source\Driver\src\Analog_Circuits.c      0x00000000   Number         0  analog_circuits.o ABSOLUTE
    source\Driver\src\Analog_Signals.c       0x00000000   Number         0  analog_signals.o ABSOLUTE
    source\Driver\src\Sys_Tick.c             0x00000000   Number         0  sys_tick.o ABSOLUTE
    source\Driver\src\adc.c                  0x00000000   Number         0  adc.o ABSOLUTE
    source\Driver\src\gpio.c                 0x00000000   Number         0  gpio.o ABSOLUTE
    source\Driver\src\sci.c                  0x00000000   Number         0  sci.o ABSOLUTE
    source\Driver\src\sci_user.c             0x00000000   Number         0  sci_user.o ABSOLUTE
    source\Driver\src\wdt.c                  0x00000000   Number         0  wdt.o ABSOLUTE
    source\System\init.c                     0x00000000   Number         0  init.o ABSOLUTE
    source\System\main.c                     0x00000000   Number         0  main.o ABSOLUTE
    source\System\sys_scheduler.c            0x00000000   Number         0  sys_scheduler.o ABSOLUTE
    source\System\tasks.c                    0x00000000   Number         0  tasks.o ABSOLUTE
    source\\Application\\LINE_IN\\Line_In.c  0x00000000   Number         0  line_in.o ABSOLUTE
    source\\Application\\MCU_Core_Protocol\\MCU_Core_Protocol.c 0x00000000   Number         0  mcu_core_protocol.o ABSOLUTE
    source\\Application\\PowerManagement\\PowerManagement_user.c 0x00000000   Number         0  powermanagement_user.o ABSOLUTE
    source\\Application\\PowerManagement\\System_Monitor.c 0x00000000   Number         0  system_monitor.o ABSOLUTE
    source\\Application\\PowerManagement\\System_Monitor_user.c 0x00000000   Number         0  system_monitor_user.o ABSOLUTE
    source\\Application\\RTE\\Common_Interface.c 0x00000000   Number         0  common_interface.o ABSOLUTE
    source\\Application\\RTE\\RTE_ADC.c      0x00000000   Number         0  rte_adc.o ABSOLUTE
    source\\Driver\\src\\Analog_Circuits.c   0x00000000   Number         0  analog_circuits.o ABSOLUTE
    source\\Driver\\src\\Analog_Signals.c    0x00000000   Number         0  analog_signals.o ABSOLUTE
    source\\Driver\\src\\Sys_Tick.c          0x00000000   Number         0  sys_tick.o ABSOLUTE
    source\\Driver\\src\\adc.c               0x00000000   Number         0  adc.o ABSOLUTE
    source\\Driver\\src\\gpio.c              0x00000000   Number         0  gpio.o ABSOLUTE
    source\\Driver\\src\\sci.c               0x00000000   Number         0  sci.o ABSOLUTE
    source\\Driver\\src\\sci_user.c          0x00000000   Number         0  sci_user.o ABSOLUTE
    source\\Driver\\src\\wdt.c               0x00000000   Number         0  wdt.o ABSOLUTE
    source\\System\\init.c                   0x00000000   Number         0  init.o ABSOLUTE
    source\\System\\main.c                   0x00000000   Number         0  main.o ABSOLUTE
    source\\System\\sys_scheduler.c          0x00000000   Number         0  sys_scheduler.o ABSOLUTE
    source\\System\\tasks.c                  0x00000000   Number         0  tasks.o ABSOLUTE
    .ARM.__AT_0x000000C0                     0x000000c0   Section        4  system_bat32g137.o(.ARM.__AT_0x000000C0)
    __tagsym$$used                           0x000000c0   Number         0  system_bat32g137.o(.ARM.__AT_0x000000C0)
    !!!main                                  0x000000c4   Section        8  __main.o(!!!main)
    !!!scatter                               0x000000cc   Section       60  __scatter.o(!!!scatter)
    !!handler_zi                             0x00000108   Section       28  __scatter_zi.o(!!handler_zi)
    .ARM.Collect$$libinit$$00000000          0x00000124   Section        2  libinit.o(.ARM.Collect$$libinit$$00000000)
    .ARM.Collect$$libinit$$00000002          0x00000126   Section        0  libinit2.o(.ARM.Collect$$libinit$$00000002)
    .ARM.Collect$$libinit$$00000004          0x00000126   Section        0  libinit2.o(.ARM.Collect$$libinit$$00000004)
    .ARM.Collect$$libinit$$0000000A          0x00000126   Section        0  libinit2.o(.ARM.Collect$$libinit$$0000000A)
    .ARM.Collect$$libinit$$0000000C          0x00000126   Section        0  libinit2.o(.ARM.Collect$$libinit$$0000000C)
    .ARM.Collect$$libinit$$0000000E          0x00000126   Section        0  libinit2.o(.ARM.Collect$$libinit$$0000000E)
    .ARM.Collect$$libinit$$00000011          0x00000126   Section        0  libinit2.o(.ARM.Collect$$libinit$$00000011)
    .ARM.Collect$$libinit$$00000013          0x00000126   Section        0  libinit2.o(.ARM.Collect$$libinit$$00000013)
    .ARM.Collect$$libinit$$00000015          0x00000126   Section        0  libinit2.o(.ARM.Collect$$libinit$$00000015)
    .ARM.Collect$$libinit$$00000017          0x00000126   Section        0  libinit2.o(.ARM.Collect$$libinit$$00000017)
    .ARM.Collect$$libinit$$00000019          0x00000126   Section        0  libinit2.o(.ARM.Collect$$libinit$$00000019)
    .ARM.Collect$$libinit$$0000001B          0x00000126   Section        0  libinit2.o(.ARM.Collect$$libinit$$0000001B)
    .ARM.Collect$$libinit$$0000001D          0x00000126   Section        0  libinit2.o(.ARM.Collect$$libinit$$0000001D)
    .ARM.Collect$$libinit$$0000001F          0x00000126   Section        0  libinit2.o(.ARM.Collect$$libinit$$0000001F)
    .ARM.Collect$$libinit$$00000021          0x00000126   Section        0  libinit2.o(.ARM.Collect$$libinit$$00000021)
    .ARM.Collect$$libinit$$00000023          0x00000126   Section        0  libinit2.o(.ARM.Collect$$libinit$$00000023)
    .ARM.Collect$$libinit$$00000025          0x00000126   Section        0  libinit2.o(.ARM.Collect$$libinit$$00000025)
    .ARM.Collect$$libinit$$0000002C          0x00000126   Section        0  libinit2.o(.ARM.Collect$$libinit$$0000002C)
    .ARM.Collect$$libinit$$0000002E          0x00000126   Section        0  libinit2.o(.ARM.Collect$$libinit$$0000002E)
    .ARM.Collect$$libinit$$00000030          0x00000126   Section        0  libinit2.o(.ARM.Collect$$libinit$$00000030)
    .ARM.Collect$$libinit$$00000032          0x00000126   Section        0  libinit2.o(.ARM.Collect$$libinit$$00000032)
    .ARM.Collect$$libinit$$00000033          0x00000126   Section        2  libinit2.o(.ARM.Collect$$libinit$$00000033)
    .ARM.Collect$$libshutdown$$00000000      0x00000128   Section        2  libshutdown.o(.ARM.Collect$$libshutdown$$00000000)
    .ARM.Collect$$libshutdown$$00000002      0x0000012a   Section        0  libshutdown2.o(.ARM.Collect$$libshutdown$$00000002)
    .ARM.Collect$$libshutdown$$00000004      0x0000012a   Section        0  libshutdown2.o(.ARM.Collect$$libshutdown$$00000004)
    .ARM.Collect$$libshutdown$$00000006      0x0000012a   Section        0  libshutdown2.o(.ARM.Collect$$libshutdown$$00000006)
    .ARM.Collect$$libshutdown$$00000009      0x0000012a   Section        0  libshutdown2.o(.ARM.Collect$$libshutdown$$00000009)
    .ARM.Collect$$libshutdown$$0000000C      0x0000012a   Section        0  libshutdown2.o(.ARM.Collect$$libshutdown$$0000000C)
    .ARM.Collect$$libshutdown$$0000000E      0x0000012a   Section        0  libshutdown2.o(.ARM.Collect$$libshutdown$$0000000E)
    .ARM.Collect$$libshutdown$$00000011      0x0000012a   Section        0  libshutdown2.o(.ARM.Collect$$libshutdown$$00000011)
    .ARM.Collect$$libshutdown$$00000012      0x0000012a   Section        2  libshutdown2.o(.ARM.Collect$$libshutdown$$00000012)
    .ARM.Collect$$rtentry$$00000000          0x0000012c   Section        0  __rtentry.o(.ARM.Collect$$rtentry$$00000000)
    .ARM.Collect$$rtentry$$00000002          0x0000012c   Section        0  __rtentry2.o(.ARM.Collect$$rtentry$$00000002)
    .ARM.Collect$$rtentry$$00000004          0x0000012c   Section        6  __rtentry4.o(.ARM.Collect$$rtentry$$00000004)
    .ARM.Collect$$rtentry$$00000009          0x00000132   Section        0  __rtentry2.o(.ARM.Collect$$rtentry$$00000009)
    .ARM.Collect$$rtentry$$0000000A          0x00000132   Section        4  __rtentry2.o(.ARM.Collect$$rtentry$$0000000A)
    .ARM.Collect$$rtentry$$0000000C          0x00000136   Section        0  __rtentry2.o(.ARM.Collect$$rtentry$$0000000C)
    .ARM.Collect$$rtentry$$0000000D          0x00000136   Section        8  __rtentry2.o(.ARM.Collect$$rtentry$$0000000D)
    .ARM.Collect$$rtexit$$00000000           0x0000013e   Section        2  rtexit.o(.ARM.Collect$$rtexit$$00000000)
    .ARM.Collect$$rtexit$$00000002           0x00000140   Section        0  rtexit2.o(.ARM.Collect$$rtexit$$00000002)
    .ARM.Collect$$rtexit$$00000003           0x00000140   Section        4  rtexit2.o(.ARM.Collect$$rtexit$$00000003)
    .ARM.Collect$$rtexit$$00000004           0x00000144   Section        6  rtexit2.o(.ARM.Collect$$rtexit$$00000004)
    .text                                    0x0000014c   Section      128  startup_bat32g137.o(.text)
    .text                                    0x000001cc   Section        0  llmul.o(.text)
    .text                                    0x000001fc   Section        0  lludiv.o(.text)
    .text                                    0x000002fe   Section      346  aeabi_sdiv.o(.text)
    .text                                    0x00000458   Section        0  heapauxi.o(.text)
    .text                                    0x0000045e   Section       62  sys_stackheap_outer.o(.text)
    .text                                    0x0000049c   Section        0  exit.o(.text)
    .text                                    0x000004ac   Section        8  libspace.o(.text)
    .text                                    0x000004b4   Section        0  sys_exit.o(.text)
    .text                                    0x000004c0   Section        2  use_no_semi.o(.text)
    .text                                    0x000004c2   Section        0  indicate_semi.o(.text)
    .text                                    0x000004c2   Section        0  __dczerorl2.o(.text)
    i.ADC_Conv_Single_Channel                0x00000518   Section        0  analog_signals.o(i.ADC_Conv_Single_Channel)
    i.ADC_Data_Calibrate                     0x00000684   Section        0  analog_circuits.o(i.ADC_Data_Calibrate)
    i.ADC_Get_Conversion_Result              0x000006b8   Section        0  adc.o(i.ADC_Get_Conversion_Result)
    i.ADC_Get_Conversion_Status              0x000006e4   Section        0  adc.o(i.ADC_Get_Conversion_Status)
    i.ADC_Init                               0x000006f0   Section        0  adc.o(i.ADC_Init)
    i.ADC_Input_Voltage_Calc                 0x000007a8   Section        0  analog_circuits.o(i.ADC_Input_Voltage_Calc)
    i.ADC_Read_Signal                        0x000007dc   Section        0  analog_signals.o(i.ADC_Read_Signal)
    i.ADC_Read_Signal_Valid                  0x000007f4   Section        0  analog_signals.o(i.ADC_Read_Signal_Valid)
    i.ADC_Start                              0x0000080c   Section        0  adc.o(i.ADC_Start)
    i.ADC_Start_Conversion                   0x0000083c   Section        0  adc.o(i.ADC_Start_Conversion)
    i.ADC_Stop                               0x00000864   Section        0  adc.o(i.ADC_Stop)
    i.ADC_Stop_Conversion                    0x0000088c   Section        0  adc.o(i.ADC_Stop_Conversion)
    i.ADC_Voltage_Calc_Circuit102            0x00000894   Section        0  analog_circuits.o(i.ADC_Voltage_Calc_Circuit102)
    i.Analog_Signal_Conv_Init                0x0000091c   Section        0  analog_signals.o(i.Analog_Signal_Conv_Init)
    i.Analog_Signal_Conv_Real_Time_Run       0x00000988   Section        0  adc.o(i.Analog_Signal_Conv_Real_Time_Run)
    i.Analog_Signal_Conv_Service             0x000009f4   Section        0  analog_signals.o(i.Analog_Signal_Conv_Service)
    i.CLK_GetCoreFreq                        0x00000c48   Section        0  system_bat32g137.o(i.CLK_GetCoreFreq)
    i.Common_Get_ConnectPhoneSts             0x00000cf4   Section        0  common_interface.o(i.Common_Get_ConnectPhoneSts)
    i.Common_Get_DispMode                    0x00000d00   Section        0  common_interface.o(i.Common_Get_DispMode)
    i.Common_Get_IG_Sts                      0x00000d0c   Section        0  common_interface.o(i.Common_Get_IG_Sts)
    i.Common_Get_IG_Sts_Valid                0x00000d18   Section        0  common_interface.o(i.Common_Get_IG_Sts_Valid)
    i.Common_Get_Language                    0x00000d24   Section        0  common_interface.o(i.Common_Get_Language)
    i.Common_Get_Theme                       0x00000d30   Section        0  common_interface.o(i.Common_Get_Theme)
    i.GPIO_Init                              0x00000d3c   Section        0  gpio.o(i.GPIO_Init)
    i.Get_ID_01_Data                         0x00000fa8   Section        0  mcu_core_protocol.o(i.Get_ID_01_Data)
    i.Get_ID_02_Data                         0x00001230   Section        0  mcu_core_protocol.o(i.Get_ID_02_Data)
    i.Get_Uart2_State                        0x00001278   Section        0  sci_user.o(i.Get_Uart2_State)
    i.INTC_ClearPendingIRQ                   0x00001284   Section        0  adc.o(i.INTC_ClearPendingIRQ)
    INTC_ClearPendingIRQ                     0x00001285   Thumb Code    62  adc.o(i.INTC_ClearPendingIRQ)
    i.INTC_ClearPendingIRQ                   0x000012c8   Section        0  sci.o(i.INTC_ClearPendingIRQ)
    INTC_ClearPendingIRQ                     0x000012c9   Thumb Code    62  sci.o(i.INTC_ClearPendingIRQ)
    i.INTC_ClearPendingIRQ                   0x0000130c   Section        0  sci_user.o(i.INTC_ClearPendingIRQ)
    INTC_ClearPendingIRQ                     0x0000130d   Thumb Code    62  sci_user.o(i.INTC_ClearPendingIRQ)
    i.INTC_DisableIRQ                        0x00001350   Section        0  adc.o(i.INTC_DisableIRQ)
    INTC_DisableIRQ                          0x00001351   Thumb Code    60  adc.o(i.INTC_DisableIRQ)
    i.INTC_DisableIRQ                        0x00001390   Section        0  sci.o(i.INTC_DisableIRQ)
    INTC_DisableIRQ                          0x00001391   Thumb Code    60  sci.o(i.INTC_DisableIRQ)
    i.INTC_EnableIRQ                         0x000013d0   Section        0  sci.o(i.INTC_EnableIRQ)
    INTC_EnableIRQ                           0x000013d1   Thumb Code    60  sci.o(i.INTC_EnableIRQ)
    i.IRQ07_Handler                          0x00001410   Section        0  sci_user.o(i.IRQ07_Handler)
    uart2_interrupt_send                     0x00001411   Thumb Code     0  sci_user.o(i.IRQ07_Handler)
    i.IRQ08_Handler                          0x00001458   Section        0  sci_user.o(i.IRQ08_Handler)
    uart2_interrupt_receive                  0x00001459   Thumb Code     0  sci_user.o(i.IRQ08_Handler)
    i.LINE_IN_Get_ABS                        0x00001534   Section        0  line_in.o(i.LINE_IN_Get_ABS)
    i.LINE_IN_Get_Gear_1                     0x0000154a   Section        0  line_in.o(i.LINE_IN_Get_Gear_1)
    i.LINE_IN_Get_Gear_2                     0x00001560   Section        0  line_in.o(i.LINE_IN_Get_Gear_2)
    i.LINE_IN_Get_Gear_3                     0x00001576   Section        0  line_in.o(i.LINE_IN_Get_Gear_3)
    i.LINE_IN_Get_Gear_4                     0x0000158c   Section        0  line_in.o(i.LINE_IN_Get_Gear_4)
    i.LINE_IN_Get_Gear_5                     0x000015a2   Section        0  line_in.o(i.LINE_IN_Get_Gear_5)
    i.LINE_IN_Get_Gear_6                     0x000015b8   Section        0  line_in.o(i.LINE_IN_Get_Gear_6)
    i.LINE_IN_Get_Gear_N                     0x000015ce   Section        0  line_in.o(i.LINE_IN_Get_Gear_N)
    i.LINE_IN_Get_HighBeam                   0x000015e4   Section        0  line_in.o(i.LINE_IN_Get_HighBeam)
    i.LINE_IN_Get_Key1                       0x000015fa   Section        0  line_in.o(i.LINE_IN_Get_Key1)
    i.LINE_IN_Get_Key2                       0x00001610   Section        0  line_in.o(i.LINE_IN_Get_Key2)
    i.LINE_IN_Get_LeftTurn                   0x00001626   Section        0  line_in.o(i.LINE_IN_Get_LeftTurn)
    i.LINE_IN_Get_OilPressure                0x0000163c   Section        0  line_in.o(i.LINE_IN_Get_OilPressure)
    i.LINE_IN_Get_RightTurn                  0x00001652   Section        0  line_in.o(i.LINE_IN_Get_RightTurn)
    i.Line_In_Debounce_Handle                0x00001668   Section        0  line_in.o(i.Line_In_Debounce_Handle)
    Line_In_Debounce_Handle                  0x00001669   Thumb Code   200  line_in.o(i.Line_In_Debounce_Handle)
    i.Line_In_Debounce_Service               0x00001738   Section        0  line_in.o(i.Line_In_Debounce_Service)
    i.Line_In_KL15_OFF_Init                  0x00001790   Section        0  line_in.o(i.Line_In_KL15_OFF_Init)
    i.Line_In_KL15_ON_Init                   0x000017d0   Section        0  line_in.o(i.Line_In_KL15_ON_Init)
    i.Line_In_KL30_Init                      0x00001810   Section        0  line_in.o(i.Line_In_KL30_Init)
    i.MCU_Send_Service                       0x00001848   Section        0  mcu_core_protocol.o(i.MCU_Send_Service)
    i.PORT_ClrBit                            0x000018f4   Section        0  gpio.o(i.PORT_ClrBit)
    i.PORT_GetBit                            0x00001918   Section        0  gpio.o(i.PORT_GetBit)
    i.PORT_Init                              0x00001934   Section        0  gpio.o(i.PORT_Init)
    i.PORT_SetBit                            0x00001acc   Section        0  gpio.o(i.PORT_SetBit)
    i.PowerMemInit                           0x00001af0   Section        0  powermanagement.o(i.PowerMemInit)
    i.Power_IG_LVP_Init                      0x00001b30   Section        0  powermanagement_user.o(i.Power_IG_LVP_Init)
    i.Power_IG_OFF_Init                      0x00001b32   Section        0  powermanagement_user.o(i.Power_IG_OFF_Init)
    i.Power_IG_ON_Init                       0x00001b3a   Section        0  powermanagement_user.o(i.Power_IG_ON_Init)
    i.Power_IG_OVP_Init                      0x00001b42   Section        0  powermanagement_user.o(i.Power_IG_OVP_Init)
    i.Power_KL30_Init                        0x00001b44   Section        0  powermanagement_user.o(i.Power_KL30_Init)
    i.Power_Management_Init                  0x00001b50   Section        0  powermanagement.o(i.Power_Management_Init)
    i.Power_Management_Lib_Init              0x00001b78   Section        0  powermanagement_user.o(i.Power_Management_Lib_Init)
    i.Power_Management_Service               0x00001be0   Section        0  powermanagement.o(i.Power_Management_Service)
    i.Power_Sleep_Init                       0x00001d04   Section        0  powermanagement_user.o(i.Power_Sleep_Init)
    i.Power_Stay_OFF                         0x00001d0e   Section        0  powermanagement_user.o(i.Power_Stay_OFF)
    i.Power_Stay_ON                          0x00001d3a   Section        0  powermanagement_user.o(i.Power_Stay_ON)
    i.Power_Stay_Protect                     0x00001d76   Section        0  powermanagement_user.o(i.Power_Stay_Protect)
    i.Power_Stay_Sleep                       0x00001d7a   Section        0  powermanagement_user.o(i.Power_Stay_Sleep)
    i.Power_Wakeup_Init                      0x00001d7e   Section        0  powermanagement_user.o(i.Power_Wakeup_Init)
    i.RTE_ForceRead_KL15_Voltage             0x00001d8a   Section        0  rte_adc.o(i.RTE_ForceRead_KL15_Voltage)
    i.RTE_ForceRead_KL30_Voltage             0x00001d9a   Section        0  rte_adc.o(i.RTE_ForceRead_KL30_Voltage)
    i.Send_To_Core                           0x00001dac   Section        0  mcu_core_protocol.o(i.Send_To_Core)
    i.SysTick_Handler                        0x00001e30   Section        0  sys_tick.o(i.SysTick_Handler)
    i.Sys_BlockDelay                         0x00001ee0   Section        0  system_monitor_user.o(i.Sys_BlockDelay)
    i.Sys_Exact_100ms_Task_Handler           0x00001f14   Section        0  sys_scheduler.o(i.Sys_Exact_100ms_Task_Handler)
    Sys_Exact_100ms_Task_Handler             0x00001f15   Thumb Code     8  sys_scheduler.o(i.Sys_Exact_100ms_Task_Handler)
    i.Sys_Exact_100ms_Tasks                  0x00001f1c   Section        0  tasks.o(i.Sys_Exact_100ms_Tasks)
    i.Sys_Exact_50us_Task_Handler            0x00001f1e   Section        0  sys_scheduler.o(i.Sys_Exact_50us_Task_Handler)
    Sys_Exact_50us_Task_Handler              0x00001f1f   Thumb Code     8  sys_scheduler.o(i.Sys_Exact_50us_Task_Handler)
    i.Sys_Exact_50us_Tasks                   0x00001f26   Section        0  tasks.o(i.Sys_Exact_50us_Tasks)
    i.Sys_Force_Read_KL15_Voltage            0x00001f2e   Section        0  system_monitor_user.o(i.Sys_Force_Read_KL15_Voltage)
    i.Sys_Force_Read_KL30_Voltage            0x00001f3a   Section        0  system_monitor_user.o(i.Sys_Force_Read_KL30_Voltage)
    i.Sys_Get_ms_Rolling_Counter             0x00001f48   Section        0  system_monitor_user.o(i.Sys_Get_ms_Rolling_Counter)
    i.Sys_Init                               0x00001f54   Section        0  sys_scheduler.o(i.Sys_Init)
    i.Sys_KL30_Init                          0x00001f94   Section        0  system_monitor_user.o(i.Sys_KL30_Init)
    i.Sys_LogicProcess                       0x00001fc0   Section        0  system_monitor_user.o(i.Sys_LogicProcess)
    i.Sys_Rolling                            0x00001fc4   Section        0  system_monitor_user.o(i.Sys_Rolling)
    i.Sys_RollingClear                       0x00001fec   Section        0  system_monitor_user.o(i.Sys_RollingClear)
    i.Sys_Run_Mode_100ms_Tasks               0x00001ff8   Section        0  tasks.o(i.Sys_Run_Mode_100ms_Tasks)
    i.Sys_Run_Mode_10ms_Tasks                0x00002018   Section        0  tasks.o(i.Sys_Run_Mode_10ms_Tasks)
    i.Sys_Run_Mode_20ms_Tasks                0x00002020   Section        0  tasks.o(i.Sys_Run_Mode_20ms_Tasks)
    i.Sys_Run_Mode_2ms_Tasks                 0x00002022   Section        0  tasks.o(i.Sys_Run_Mode_2ms_Tasks)
    i.Sys_Run_Mode_50ms_Tasks                0x00002030   Section        0  tasks.o(i.Sys_Run_Mode_50ms_Tasks)
    i.Sys_Run_Mode_5ms_Tasks                 0x00002032   Section        0  tasks.o(i.Sys_Run_Mode_5ms_Tasks)
    i.Sys_Run_Mode_Pseudo_Real_Time_Tasks    0x00002034   Section        0  tasks.o(i.Sys_Run_Mode_Pseudo_Real_Time_Tasks)
    i.Sys_Scheduling_Service                 0x00002040   Section        0  sys_scheduler.o(i.Sys_Scheduling_Service)
    i.Sys_Set_DebounceTimer                  0x00002128   Section        0  system_monitor.o(i.Sys_Set_DebounceTimer)
    i.Sys_Set_VolRange                       0x0000214c   Section        0  system_monitor.o(i.Sys_Set_VolRange)
    i.Sys_Startup_Init                       0x000021b4   Section        0  init.o(i.Sys_Startup_Init)
    i.Sys_Tick_Timer_Call_Back_Reg           0x000021d8   Section        0  sys_tick.o(i.Sys_Tick_Timer_Call_Back_Reg)
    i.Sys_Tick_Timer_Start                   0x000021e8   Section        0  sys_tick.o(i.Sys_Tick_Timer_Start)
    i.Sys_WakeUp_Init                        0x0000224c   Section        0  system_monitor_user.o(i.Sys_WakeUp_Init)
    i.SystemCoreClockUpdate                  0x00002278   Section        0  system_bat32g137.o(i.SystemCoreClockUpdate)
    i.SystemInit                             0x00002288   Section        0  system_bat32g137.o(i.SystemInit)
    i.System_FUN_KL30_Status_Get             0x000022fc   Section        0  system_monitor.o(i.System_FUN_KL30_Status_Get)
    i.System_Fast_WakeUp                     0x00002308   Section        0  system_monitor.o(i.System_Fast_WakeUp)
    i.System_LINE_KL15                       0x000023e4   Section        0  system_monitor_user.o(i.System_LINE_KL15)
    i.System_Monitor_KL30Init                0x000023f4   Section        0  system_monitor.o(i.System_Monitor_KL30Init)
    i.System_Monitor_WakeupInit              0x00002520   Section        0  system_monitor.o(i.System_Monitor_WakeupInit)
    i.TFT_CreateCRCCheckSum                  0x0000264c   Section        0  mcu_core_protocol.o(i.TFT_CreateCRCCheckSum)
    i.UART2_BaudRate                         0x00002694   Section        0  sci.o(i.UART2_BaudRate)
    i.UART2_Init                             0x000026e4   Section        0  sci.o(i.UART2_Init)
    i.UART2_Start                            0x00002830   Section        0  sci.o(i.UART2_Start)
    i.UART_BaudRateCal                       0x00002880   Section        0  sci.o(i.UART_BaudRateCal)
    i.UART_Ch2_Send_Multiple_Byte            0x000028f8   Section        0  sci_user.o(i.UART_Ch2_Send_Multiple_Byte)
    i.WDT_Restart                            0x00002950   Section        0  wdt.o(i.WDT_Restart)
    i.__ARM_common_switch8                   0x0000295c   Section        0  gpio.o(i.__ARM_common_switch8)
    i.__NVIC_ClearPendingIRQ                 0x00002978   Section        0  adc.o(i.__NVIC_ClearPendingIRQ)
    __NVIC_ClearPendingIRQ                   0x00002979   Thumb Code    18  adc.o(i.__NVIC_ClearPendingIRQ)
    i.__NVIC_ClearPendingIRQ                 0x00002990   Section        0  sci.o(i.__NVIC_ClearPendingIRQ)
    __NVIC_ClearPendingIRQ                   0x00002991   Thumb Code    18  sci.o(i.__NVIC_ClearPendingIRQ)
    i.__NVIC_SetPriority                     0x000029a8   Section        0  sys_tick.o(i.__NVIC_SetPriority)
    __NVIC_SetPriority                       0x000029a9   Thumb Code   110  sys_tick.o(i.__NVIC_SetPriority)
    i.main                                   0x00002a20   Section        0  main.o(i.main)
    i.uart0_callback_error                   0x00002a30   Section        0  sci_user.o(i.uart0_callback_error)
    uart0_callback_error                     0x00002a31   Thumb Code     2  sci_user.o(i.uart0_callback_error)
    i.uart0_callback_receiveend              0x00002a32   Section        0  sci_user.o(i.uart0_callback_receiveend)
    uart0_callback_receiveend                0x00002a33   Thumb Code     2  sci_user.o(i.uart0_callback_receiveend)
    i.uart0_callback_sendend                 0x00002a34   Section        0  sci_user.o(i.uart0_callback_sendend)
    uart0_callback_sendend                   0x00002a35   Thumb Code     2  sci_user.o(i.uart0_callback_sendend)
    i.uart0_callback_softwareoverrun         0x00002a36   Section        0  sci_user.o(i.uart0_callback_softwareoverrun)
    uart0_callback_softwareoverrun           0x00002a37   Thumb Code     2  sci_user.o(i.uart0_callback_softwareoverrun)
    i.uart0_interrupt_receive                0x00002a38   Section        0  sci_user.o(i.uart0_interrupt_receive)
    i.uart0_interrupt_send                   0x00002ac0   Section        0  sci_user.o(i.uart0_interrupt_send)
    i.uart2_callback_error                   0x00002b04   Section        0  sci_user.o(i.uart2_callback_error)
    uart2_callback_error                     0x00002b05   Thumb Code    10  sci_user.o(i.uart2_callback_error)
    i.uart2_callback_receiveend              0x00002b14   Section        0  sci_user.o(i.uart2_callback_receiveend)
    uart2_callback_receiveend                0x00002b15   Thumb Code    10  sci_user.o(i.uart2_callback_receiveend)
    i.uart2_callback_sendend                 0x00002b24   Section        0  sci_user.o(i.uart2_callback_sendend)
    uart2_callback_sendend                   0x00002b25   Thumb Code     8  sci_user.o(i.uart2_callback_sendend)
    .constdata                               0x00002b30   Section      132  analog_signals.o(.constdata)
    .constdata                               0x00002bb4   Section       32  sci.o(.constdata)
    .constdata                               0x00002bd4   Section      168  line_in.o(.constdata)
    .constdata                               0x00002c7c   Section       40  system_monitor_user.o(.constdata)
    SysFun_Range                             0x00002c7c   Data          20  system_monitor_user.o(.constdata)
    SysNM_Range                              0x00002c90   Data          20  system_monitor_user.o(.constdata)
    .constdata                               0x00002ca4   Section      512  mcu_core_protocol.o(.constdata)
    CRC16_TAB_H                              0x00002ca4   Data         256  mcu_core_protocol.o(.constdata)
    CRC16_TAB_L                              0x00002da4   Data         256  mcu_core_protocol.o(.constdata)
    .data                                    0x20000000   Section        4  sys_tick.o(.data)
    .data                                    0x20000004   Section       10  adc.o(.data)
    .data                                    0x2000000e   Section       14  analog_signals.o(.data)
    .data                                    0x2000001c   Section      276  sci.o(.data)
    dummy_sio00                              0x20000124   Data           1  sci.o(.data)
    dummy_sio00                              0x20000125   Data           1  sci.o(.data)
    dummy_sio01                              0x20000126   Data           1  sci.o(.data)
    dummy_sio01                              0x20000127   Data           1  sci.o(.data)
    dummy_sio10                              0x20000128   Data           1  sci.o(.data)
    dummy_sio10                              0x20000129   Data           1  sci.o(.data)
    dummy_sio11                              0x2000012a   Data           1  sci.o(.data)
    dummy_sio11                              0x2000012b   Data           1  sci.o(.data)
    dummy_sio20                              0x2000012c   Data           1  sci.o(.data)
    dummy_sio20                              0x2000012d   Data           1  sci.o(.data)
    dummy_sio21                              0x2000012e   Data           1  sci.o(.data)
    dummy_sio21                              0x2000012f   Data           1  sci.o(.data)
    .data                                    0x20000130   Section       14  sci_user.o(.data)
    lastData                                 0x2000013d   Data           1  sci_user.o(.data)
    .data                                    0x2000013e   Section        1  line_in.o(.data)
    .data                                    0x2000013f   Section        1  powermanagement.o(.data)
    g_Power_St                               0x2000013f   Data           1  powermanagement.o(.data)
    .data                                    0x20000140   Section       54  system_monitor.o(.data)
    SetVolFlag                               0x20000141   Data           1  system_monitor.o(.data)
    t_NM_KL30_Debounce                       0x20000142   Data           2  system_monitor.o(.data)
    t_NM_KL15_Debounce                       0x20000144   Data           2  system_monitor.o(.data)
    t_FUN_KL30_Debounce                      0x20000146   Data           2  system_monitor.o(.data)
    t_FUN_KL15_Debounce                      0x20000148   Data           2  system_monitor.o(.data)
    FUNSysVol_Range                          0x2000014a   Data          20  system_monitor.o(.data)
    NMSysVol_Range                           0x2000015e   Data          20  system_monitor.o(.data)
    DebpounceTimer                           0x20000172   Data           2  system_monitor.o(.data)
    DebpounceTimer                           0x20000174   Data           2  system_monitor.o(.data)
    .data                                    0x20000178   Section        4  system_monitor_user.o(.data)
    .data                                    0x2000017c   Section       30  common_interface.o(.data)
    PowerIgnOnTimeLine                       0x2000017c   Data           4  common_interface.o(.data)
    PowerIgnOffTimeLine                      0x20000180   Data           4  common_interface.o(.data)
    g_Disp_Mode                              0x20000184   Data           1  common_interface.o(.data)
    g_Language                               0x20000185   Data           1  common_interface.o(.data)
    g_Theme                                  0x20000186   Data           1  common_interface.o(.data)
    g_ConnectPhone                           0x20000187   Data           1  common_interface.o(.data)
    PowerSts                                 0x20000188   Data           1  common_interface.o(.data)
    Act_V_Speed                              0x2000018a   Data           2  common_interface.o(.data)
    Act_E_Speed                              0x2000018c   Data           2  common_interface.o(.data)
    Disp_V_Speed                             0x2000018e   Data           2  common_interface.o(.data)
    Disp_E_Speed                             0x20000190   Data           2  common_interface.o(.data)
    PowerSts_Valid                           0x20000192   Data           1  common_interface.o(.data)
    Act_V_Speed_Valid                        0x20000193   Data           1  common_interface.o(.data)
    Act_E_Speed_Valid                        0x20000194   Data           1  common_interface.o(.data)
    Disp_V_Speed_Valid                       0x20000195   Data           1  common_interface.o(.data)
    Disp_E_Speed_Valid                       0x20000196   Data           1  common_interface.o(.data)
    SysRollingCounter                        0x20000198   Data           2  common_interface.o(.data)
    .data                                    0x2000019c   Section       56  mcu_core_protocol.o(.data)
    .data                                    0x200001d4   Section        4  system_bat32g137.o(.data)
    .bss                                     0x200001d8   Section       24  sys_tick.o(.bss)
    .bss                                     0x200001f0   Section       16  analog_signals.o(.bss)
    .bss                                     0x20000200   Section       14  sys_scheduler.o(.bss)
    .bss                                     0x2000020e   Section       84  line_in.o(.bss)
    .bss                                     0x20000264   Section       44  powermanagement.o(.bss)
    .bss                                     0x20000290   Section       48  system_monitor.o(.bss)
    .bss                                     0x200002c0   Section      290  mcu_core_protocol.o(.bss)
    .bss                                     0x200003e4   Section       96  libspace.o(.bss)
    HEAP                                     0x20000448   Section      256  startup_bat32g137.o(HEAP)
    Heap_Mem                                 0x20000448   Data         256  startup_bat32g137.o(HEAP)
    STACK                                    0x20000548   Section     1024  startup_bat32g137.o(STACK)
    Stack_Mem                                0x20000548   Data        1024  startup_bat32g137.o(STACK)
    __initial_sp                             0x20000948   Data           0  startup_bat32g137.o(STACK)

    Global Symbols

    Symbol Name                              Value     Ov Type        Size  Object(Section)

    BuildAttributes$$THM_ISAv3M$S$PE$A:L22$X:L11$S22$IEEE1$IW$USESV6$~STKCKD$USESV7$~SHL$OSPACE$ROPI$EBA8$UX$STANDARDLIB$REQ8$PRES8$EABIv2 0x00000000   Number         0  anon$$obj.o ABSOLUTE
    __ARM_use_no_argv                        0x00000000   Number         0  main.o ABSOLUTE
    __Vectors                                0x00000000   Data           4  startup_bat32g137.o(RESET)
    __ARM_exceptions_init                     - Undefined Weak Reference
    __alloca_initialize                       - Undefined Weak Reference
    __arm_fini_                               - Undefined Weak Reference
    __arm_preinit_                            - Undefined Weak Reference
    __cpp_initialize__aeabi_                  - Undefined Weak Reference
    __cxa_finalize                            - Undefined Weak Reference
    __rt_locale                               - Undefined Weak Reference
    __sigvec_lookup                           - Undefined Weak Reference
    _atexit_init                              - Undefined Weak Reference
    _call_atexit_fns                          - Undefined Weak Reference
    _clock_init                               - Undefined Weak Reference
    _fp_trap_init                             - Undefined Weak Reference
    _fp_trap_shutdown                         - Undefined Weak Reference
    _get_lc_collate                           - Undefined Weak Reference
    _get_lc_ctype                             - Undefined Weak Reference
    _get_lc_monetary                          - Undefined Weak Reference
    _get_lc_numeric                           - Undefined Weak Reference
    _get_lc_time                              - Undefined Weak Reference
    _getenv_init                              - Undefined Weak Reference
    _handle_redirection                       - Undefined Weak Reference
    _init_alloc                               - Undefined Weak Reference
    _init_user_alloc                          - Undefined Weak Reference
    _initio                                   - Undefined Weak Reference
    _rand_init                                - Undefined Weak Reference
    _signal_finish                            - Undefined Weak Reference
    _signal_init                              - Undefined Weak Reference
    _terminate_alloc                          - Undefined Weak Reference
    _terminate_user_alloc                     - Undefined Weak Reference
    _terminateio                              - Undefined Weak Reference
    __Vectors_End                            0x000000c0   Data           0  startup_bat32g137.o(RESET)
    __Vectors_Size                           0x000000c0   Number         0  startup_bat32g137.o ABSOLUTE
    user_opt_data                            0x000000c0   Data           4  system_bat32g137.o(.ARM.__AT_0x000000C0)
    __main                                   0x000000c5   Thumb Code     8  __main.o(!!!main)
    __scatterload                            0x000000cd   Thumb Code     0  __scatter.o(!!!scatter)
    __scatterload_rt2                        0x000000cd   Thumb Code    52  __scatter.o(!!!scatter)
    __scatterload_rt2_thumb_only             0x000000cd   Thumb Code     0  __scatter.o(!!!scatter)
    __scatterload_null                       0x000000dd   Thumb Code     0  __scatter.o(!!!scatter)
    __scatterload_zeroinit                   0x00000109   Thumb Code    28  __scatter_zi.o(!!handler_zi)
    __rt_lib_init                            0x00000125   Thumb Code     0  libinit.o(.ARM.Collect$$libinit$$00000000)
    __rt_lib_init_alloca_1                   0x00000127   Thumb Code     0  libinit2.o(.ARM.Collect$$libinit$$0000002E)
    __rt_lib_init_argv_1                     0x00000127   Thumb Code     0  libinit2.o(.ARM.Collect$$libinit$$0000002C)
    __rt_lib_init_atexit_1                   0x00000127   Thumb Code     0  libinit2.o(.ARM.Collect$$libinit$$0000001B)
    __rt_lib_init_clock_1                    0x00000127   Thumb Code     0  libinit2.o(.ARM.Collect$$libinit$$00000021)
    __rt_lib_init_cpp_1                      0x00000127   Thumb Code     0  libinit2.o(.ARM.Collect$$libinit$$00000032)
    __rt_lib_init_exceptions_1               0x00000127   Thumb Code     0  libinit2.o(.ARM.Collect$$libinit$$00000030)
    __rt_lib_init_fp_1                       0x00000127   Thumb Code     0  libinit2.o(.ARM.Collect$$libinit$$00000002)
    __rt_lib_init_fp_trap_1                  0x00000127   Thumb Code     0  libinit2.o(.ARM.Collect$$libinit$$0000001F)
    __rt_lib_init_getenv_1                   0x00000127   Thumb Code     0  libinit2.o(.ARM.Collect$$libinit$$00000023)
    __rt_lib_init_heap_1                     0x00000127   Thumb Code     0  libinit2.o(.ARM.Collect$$libinit$$0000000A)
    __rt_lib_init_lc_collate_1               0x00000127   Thumb Code     0  libinit2.o(.ARM.Collect$$libinit$$00000011)
    __rt_lib_init_lc_ctype_1                 0x00000127   Thumb Code     0  libinit2.o(.ARM.Collect$$libinit$$00000013)
    __rt_lib_init_lc_monetary_1              0x00000127   Thumb Code     0  libinit2.o(.ARM.Collect$$libinit$$00000015)
    __rt_lib_init_lc_numeric_1               0x00000127   Thumb Code     0  libinit2.o(.ARM.Collect$$libinit$$00000017)
    __rt_lib_init_lc_time_1                  0x00000127   Thumb Code     0  libinit2.o(.ARM.Collect$$libinit$$00000019)
    __rt_lib_init_preinit_1                  0x00000127   Thumb Code     0  libinit2.o(.ARM.Collect$$libinit$$00000004)
    __rt_lib_init_rand_1                     0x00000127   Thumb Code     0  libinit2.o(.ARM.Collect$$libinit$$0000000E)
    __rt_lib_init_return                     0x00000127   Thumb Code     0  libinit2.o(.ARM.Collect$$libinit$$00000033)
    __rt_lib_init_signal_1                   0x00000127   Thumb Code     0  libinit2.o(.ARM.Collect$$libinit$$0000001D)
    __rt_lib_init_stdio_1                    0x00000127   Thumb Code     0  libinit2.o(.ARM.Collect$$libinit$$00000025)
    __rt_lib_init_user_alloc_1               0x00000127   Thumb Code     0  libinit2.o(.ARM.Collect$$libinit$$0000000C)
    __rt_lib_shutdown                        0x00000129   Thumb Code     0  libshutdown.o(.ARM.Collect$$libshutdown$$00000000)
    __rt_lib_shutdown_cpp_1                  0x0000012b   Thumb Code     0  libshutdown2.o(.ARM.Collect$$libshutdown$$00000004)
    __rt_lib_shutdown_fini_1                 0x0000012b   Thumb Code     0  libshutdown2.o(.ARM.Collect$$libshutdown$$00000002)
    __rt_lib_shutdown_fp_trap_1              0x0000012b   Thumb Code     0  libshutdown2.o(.ARM.Collect$$libshutdown$$00000009)
    __rt_lib_shutdown_heap_1                 0x0000012b   Thumb Code     0  libshutdown2.o(.ARM.Collect$$libshutdown$$00000011)
    __rt_lib_shutdown_return                 0x0000012b   Thumb Code     0  libshutdown2.o(.ARM.Collect$$libshutdown$$00000012)
    __rt_lib_shutdown_signal_1               0x0000012b   Thumb Code     0  libshutdown2.o(.ARM.Collect$$libshutdown$$0000000C)
    __rt_lib_shutdown_stdio_1                0x0000012b   Thumb Code     0  libshutdown2.o(.ARM.Collect$$libshutdown$$00000006)
    __rt_lib_shutdown_user_alloc_1           0x0000012b   Thumb Code     0  libshutdown2.o(.ARM.Collect$$libshutdown$$0000000E)
    __rt_entry                               0x0000012d   Thumb Code     0  __rtentry.o(.ARM.Collect$$rtentry$$00000000)
    __rt_entry_presh_1                       0x0000012d   Thumb Code     0  __rtentry2.o(.ARM.Collect$$rtentry$$00000002)
    __rt_entry_sh                            0x0000012d   Thumb Code     0  __rtentry4.o(.ARM.Collect$$rtentry$$00000004)
    __rt_entry_li                            0x00000133   Thumb Code     0  __rtentry2.o(.ARM.Collect$$rtentry$$0000000A)
    __rt_entry_postsh_1                      0x00000133   Thumb Code     0  __rtentry2.o(.ARM.Collect$$rtentry$$00000009)
    __rt_entry_main                          0x00000137   Thumb Code     0  __rtentry2.o(.ARM.Collect$$rtentry$$0000000D)
    __rt_entry_postli_1                      0x00000137   Thumb Code     0  __rtentry2.o(.ARM.Collect$$rtentry$$0000000C)
    __rt_exit                                0x0000013f   Thumb Code     0  rtexit.o(.ARM.Collect$$rtexit$$00000000)
    __rt_exit_ls                             0x00000141   Thumb Code     0  rtexit2.o(.ARM.Collect$$rtexit$$00000003)
    __rt_exit_prels_1                        0x00000141   Thumb Code     0  rtexit2.o(.ARM.Collect$$rtexit$$00000002)
    __rt_exit_exit                           0x00000145   Thumb Code     0  rtexit2.o(.ARM.Collect$$rtexit$$00000004)
    Reset_Handler                            0x0000014d   Thumb Code     8  startup_bat32g137.o(.text)
    NMI_Handler                              0x00000155   Thumb Code     2  startup_bat32g137.o(.text)
    HardFault_Handler                        0x00000157   Thumb Code     2  startup_bat32g137.o(.text)
    MemManage_Handler                        0x00000159   Thumb Code     2  startup_bat32g137.o(.text)
    BusFault_Handler                         0x0000015b   Thumb Code     2  startup_bat32g137.o(.text)
    UsageFault_Handler                       0x0000015d   Thumb Code     2  startup_bat32g137.o(.text)
    SVC_Handler                              0x0000015f   Thumb Code     2  startup_bat32g137.o(.text)
    DebugMon_Handler                         0x00000161   Thumb Code     2  startup_bat32g137.o(.text)
    PendSV_Handler                           0x00000163   Thumb Code     2  startup_bat32g137.o(.text)
    IRQ00_Handler                            0x00000167   Thumb Code     2  startup_bat32g137.o(.text)
    IRQ01_Handler                            0x00000169   Thumb Code     2  startup_bat32g137.o(.text)
    IRQ02_Handler                            0x0000016b   Thumb Code     2  startup_bat32g137.o(.text)
    IRQ03_Handler                            0x0000016d   Thumb Code     2  startup_bat32g137.o(.text)
    IRQ04_Handler                            0x0000016f   Thumb Code     2  startup_bat32g137.o(.text)
    IRQ05_Handler                            0x00000171   Thumb Code     2  startup_bat32g137.o(.text)
    IRQ06_Handler                            0x00000173   Thumb Code     2  startup_bat32g137.o(.text)
    IRQ09_Handler                            0x00000179   Thumb Code     2  startup_bat32g137.o(.text)
    IRQ12_Handler                            0x0000017f   Thumb Code     2  startup_bat32g137.o(.text)
    IRQ13_Handler                            0x00000181   Thumb Code     2  startup_bat32g137.o(.text)
    IRQ14_Handler                            0x00000183   Thumb Code     2  startup_bat32g137.o(.text)
    IRQ15_Handler                            0x00000185   Thumb Code     2  startup_bat32g137.o(.text)
    IRQ16_Handler                            0x00000187   Thumb Code     2  startup_bat32g137.o(.text)
    IRQ17_Handler                            0x00000189   Thumb Code     2  startup_bat32g137.o(.text)
    IRQ18_Handler                            0x0000018b   Thumb Code     2  startup_bat32g137.o(.text)
    IRQ19_Handler                            0x0000018d   Thumb Code     2  startup_bat32g137.o(.text)
    IRQ20_Handler                            0x0000018f   Thumb Code     2  startup_bat32g137.o(.text)
    IRQ21_Handler                            0x00000191   Thumb Code     2  startup_bat32g137.o(.text)
    IRQ22_Handler                            0x00000193   Thumb Code     2  startup_bat32g137.o(.text)
    IRQ23_Handler                            0x00000195   Thumb Code     2  startup_bat32g137.o(.text)
    IRQ24_Handler                            0x00000197   Thumb Code     2  startup_bat32g137.o(.text)
    IRQ25_Handler                            0x00000199   Thumb Code     2  startup_bat32g137.o(.text)
    IRQ26_Handler                            0x0000019b   Thumb Code     2  startup_bat32g137.o(.text)
    IRQ27_Handler                            0x0000019d   Thumb Code     2  startup_bat32g137.o(.text)
    IRQ28_Handler                            0x0000019f   Thumb Code     2  startup_bat32g137.o(.text)
    IRQ29_Handler                            0x000001a1   Thumb Code     2  startup_bat32g137.o(.text)
    IRQ30_Handler                            0x000001a3   Thumb Code     2  startup_bat32g137.o(.text)
    IRQ31_Handler                            0x000001a5   Thumb Code     2  startup_bat32g137.o(.text)
    __user_initial_stackheap                 0x000001a9   Thumb Code    10  startup_bat32g137.o(.text)
    __aeabi_lmul                             0x000001cd   Thumb Code    48  llmul.o(.text)
    _ll_mul                                  0x000001cd   Thumb Code     0  llmul.o(.text)
    __aeabi_uldivmod                         0x000001fd   Thumb Code   258  lludiv.o(.text)
    _ll_udiv                                 0x000001fd   Thumb Code     0  lludiv.o(.text)
    __aeabi_uidiv                            0x000002ff   Thumb Code     0  aeabi_sdiv.o(.text)
    __aeabi_uidivmod                         0x000002ff   Thumb Code    20  aeabi_sdiv.o(.text)
    __aeabi_idiv                             0x00000313   Thumb Code     0  aeabi_sdiv.o(.text)
    __aeabi_idivmod                          0x00000313   Thumb Code   326  aeabi_sdiv.o(.text)
    __use_two_region_memory                  0x00000459   Thumb Code     2  heapauxi.o(.text)
    __rt_heap_escrow$2region                 0x0000045b   Thumb Code     2  heapauxi.o(.text)
    __rt_heap_expand$2region                 0x0000045d   Thumb Code     2  heapauxi.o(.text)
    __user_setup_stackheap                   0x0000045f   Thumb Code    62  sys_stackheap_outer.o(.text)
    exit                                     0x0000049d   Thumb Code    16  exit.o(.text)
    __user_libspace                          0x000004ad   Thumb Code     8  libspace.o(.text)
    __user_perproc_libspace                  0x000004ad   Thumb Code     0  libspace.o(.text)
    __user_perthread_libspace                0x000004ad   Thumb Code     0  libspace.o(.text)
    _sys_exit                                0x000004b5   Thumb Code     8  sys_exit.o(.text)
    __I$use$semihosting                      0x000004c1   Thumb Code     0  use_no_semi.o(.text)
    __use_no_semihosting_swi                 0x000004c1   Thumb Code     2  use_no_semi.o(.text)
    __decompress                             0x000004c3   Thumb Code     0  __dczerorl2.o(.text)
    __decompress1                            0x000004c3   Thumb Code    86  __dczerorl2.o(.text)
    __semihosting_library_function           0x000004c3   Thumb Code     0  indicate_semi.o(.text)
    ADC_Conv_Single_Channel                  0x00000519   Thumb Code   338  analog_signals.o(i.ADC_Conv_Single_Channel)
    ADC_Data_Calibrate                       0x00000685   Thumb Code    48  analog_circuits.o(i.ADC_Data_Calibrate)
    ADC_Get_Conversion_Result                0x000006b9   Thumb Code    36  adc.o(i.ADC_Get_Conversion_Result)
    ADC_Get_Conversion_Status                0x000006e5   Thumb Code     6  adc.o(i.ADC_Get_Conversion_Status)
    ADC_Init                                 0x000006f1   Thumb Code   170  adc.o(i.ADC_Init)
    ADC_Input_Voltage_Calc                   0x000007a9   Thumb Code    52  analog_circuits.o(i.ADC_Input_Voltage_Calc)
    ADC_Read_Signal                          0x000007dd   Thumb Code    20  analog_signals.o(i.ADC_Read_Signal)
    ADC_Read_Signal_Valid                    0x000007f5   Thumb Code    18  analog_signals.o(i.ADC_Read_Signal_Valid)
    ADC_Start                                0x0000080d   Thumb Code    44  adc.o(i.ADC_Start)
    ADC_Start_Conversion                     0x0000083d   Thumb Code    28  adc.o(i.ADC_Start_Conversion)
    ADC_Stop                                 0x00000865   Thumb Code    34  adc.o(i.ADC_Stop)
    ADC_Stop_Conversion                      0x0000088d   Thumb Code     8  adc.o(i.ADC_Stop_Conversion)
    ADC_Voltage_Calc_Circuit102              0x00000895   Thumb Code   132  analog_circuits.o(i.ADC_Voltage_Calc_Circuit102)
    Analog_Signal_Conv_Init                  0x0000091d   Thumb Code    82  analog_signals.o(i.Analog_Signal_Conv_Init)
    Analog_Signal_Conv_Real_Time_Run         0x00000989   Thumb Code    82  adc.o(i.Analog_Signal_Conv_Real_Time_Run)
    Analog_Signal_Conv_Service               0x000009f5   Thumb Code   568  analog_signals.o(i.Analog_Signal_Conv_Service)
    CLK_GetCoreFreq                          0x00000c49   Thumb Code   122  system_bat32g137.o(i.CLK_GetCoreFreq)
    Common_Get_ConnectPhoneSts               0x00000cf5   Thumb Code     6  common_interface.o(i.Common_Get_ConnectPhoneSts)
    Common_Get_DispMode                      0x00000d01   Thumb Code     6  common_interface.o(i.Common_Get_DispMode)
    Common_Get_IG_Sts                        0x00000d0d   Thumb Code     6  common_interface.o(i.Common_Get_IG_Sts)
    Common_Get_IG_Sts_Valid                  0x00000d19   Thumb Code     6  common_interface.o(i.Common_Get_IG_Sts_Valid)
    Common_Get_Language                      0x00000d25   Thumb Code     6  common_interface.o(i.Common_Get_Language)
    Common_Get_Theme                         0x00000d31   Thumb Code     6  common_interface.o(i.Common_Get_Theme)
    GPIO_Init                                0x00000d3d   Thumb Code   616  gpio.o(i.GPIO_Init)
    Get_ID_01_Data                           0x00000fa9   Thumb Code   630  mcu_core_protocol.o(i.Get_ID_01_Data)
    Get_ID_02_Data                           0x00001231   Thumb Code    66  mcu_core_protocol.o(i.Get_ID_02_Data)
    Get_Uart2_State                          0x00001279   Thumb Code     6  sci_user.o(i.Get_Uart2_State)
    IRQ07_Handler                            0x00001411   Thumb Code    60  sci_user.o(i.IRQ07_Handler)
    IRQ08_Handler                            0x00001459   Thumb Code   190  sci_user.o(i.IRQ08_Handler)
    LINE_IN_Get_ABS                          0x00001535   Thumb Code    22  line_in.o(i.LINE_IN_Get_ABS)
    LINE_IN_Get_Gear_1                       0x0000154b   Thumb Code    22  line_in.o(i.LINE_IN_Get_Gear_1)
    LINE_IN_Get_Gear_2                       0x00001561   Thumb Code    22  line_in.o(i.LINE_IN_Get_Gear_2)
    LINE_IN_Get_Gear_3                       0x00001577   Thumb Code    22  line_in.o(i.LINE_IN_Get_Gear_3)
    LINE_IN_Get_Gear_4                       0x0000158d   Thumb Code    22  line_in.o(i.LINE_IN_Get_Gear_4)
    LINE_IN_Get_Gear_5                       0x000015a3   Thumb Code    22  line_in.o(i.LINE_IN_Get_Gear_5)
    LINE_IN_Get_Gear_6                       0x000015b9   Thumb Code    22  line_in.o(i.LINE_IN_Get_Gear_6)
    LINE_IN_Get_Gear_N                       0x000015cf   Thumb Code    22  line_in.o(i.LINE_IN_Get_Gear_N)
    LINE_IN_Get_HighBeam                     0x000015e5   Thumb Code    22  line_in.o(i.LINE_IN_Get_HighBeam)
    LINE_IN_Get_Key1                         0x000015fb   Thumb Code    22  line_in.o(i.LINE_IN_Get_Key1)
    LINE_IN_Get_Key2                         0x00001611   Thumb Code    22  line_in.o(i.LINE_IN_Get_Key2)
    LINE_IN_Get_LeftTurn                     0x00001627   Thumb Code    22  line_in.o(i.LINE_IN_Get_LeftTurn)
    LINE_IN_Get_OilPressure                  0x0000163d   Thumb Code    22  line_in.o(i.LINE_IN_Get_OilPressure)
    LINE_IN_Get_RightTurn                    0x00001653   Thumb Code    22  line_in.o(i.LINE_IN_Get_RightTurn)
    Line_In_Debounce_Service                 0x00001739   Thumb Code    78  line_in.o(i.Line_In_Debounce_Service)
    Line_In_KL15_OFF_Init                    0x00001791   Thumb Code    52  line_in.o(i.Line_In_KL15_OFF_Init)
    Line_In_KL15_ON_Init                     0x000017d1   Thumb Code    52  line_in.o(i.Line_In_KL15_ON_Init)
    Line_In_KL30_Init                        0x00001811   Thumb Code    48  line_in.o(i.Line_In_KL30_Init)
    MCU_Send_Service                         0x00001849   Thumb Code   164  mcu_core_protocol.o(i.MCU_Send_Service)
    PORT_ClrBit                              0x000018f5   Thumb Code    32  gpio.o(i.PORT_ClrBit)
    PORT_GetBit                              0x00001919   Thumb Code    24  gpio.o(i.PORT_GetBit)
    PORT_Init                                0x00001935   Thumb Code   402  gpio.o(i.PORT_Init)
    PORT_SetBit                              0x00001acd   Thumb Code    32  gpio.o(i.PORT_SetBit)
    PowerMemInit                             0x00001af1   Thumb Code    54  powermanagement.o(i.PowerMemInit)
    Power_IG_LVP_Init                        0x00001b31   Thumb Code     2  powermanagement_user.o(i.Power_IG_LVP_Init)
    Power_IG_OFF_Init                        0x00001b33   Thumb Code     8  powermanagement_user.o(i.Power_IG_OFF_Init)
    Power_IG_ON_Init                         0x00001b3b   Thumb Code     8  powermanagement_user.o(i.Power_IG_ON_Init)
    Power_IG_OVP_Init                        0x00001b43   Thumb Code     2  powermanagement_user.o(i.Power_IG_OVP_Init)
    Power_KL30_Init                          0x00001b45   Thumb Code    12  powermanagement_user.o(i.Power_KL30_Init)
    Power_Management_Init                    0x00001b51   Thumb Code    30  powermanagement.o(i.Power_Management_Init)
    Power_Management_Lib_Init                0x00001b79   Thumb Code    58  powermanagement_user.o(i.Power_Management_Lib_Init)
    Power_Management_Service                 0x00001be1   Thumb Code   282  powermanagement.o(i.Power_Management_Service)
    Power_Sleep_Init                         0x00001d05   Thumb Code    10  powermanagement_user.o(i.Power_Sleep_Init)
    Power_Stay_OFF                           0x00001d0f   Thumb Code    44  powermanagement_user.o(i.Power_Stay_OFF)
    Power_Stay_ON                            0x00001d3b   Thumb Code    60  powermanagement_user.o(i.Power_Stay_ON)
    Power_Stay_Protect                       0x00001d77   Thumb Code     4  powermanagement_user.o(i.Power_Stay_Protect)
    Power_Stay_Sleep                         0x00001d7b   Thumb Code     4  powermanagement_user.o(i.Power_Stay_Sleep)
    Power_Wakeup_Init                        0x00001d7f   Thumb Code    12  powermanagement_user.o(i.Power_Wakeup_Init)
    RTE_ForceRead_KL15_Voltage               0x00001d8b   Thumb Code    16  rte_adc.o(i.RTE_ForceRead_KL15_Voltage)
    RTE_ForceRead_KL30_Voltage               0x00001d9b   Thumb Code    16  rte_adc.o(i.RTE_ForceRead_KL30_Voltage)
    Send_To_Core                             0x00001dad   Thumb Code   118  mcu_core_protocol.o(i.Send_To_Core)
    SysTick_Handler                          0x00001e31   Thumb Code   158  sys_tick.o(i.SysTick_Handler)
    Sys_BlockDelay                           0x00001ee1   Thumb Code    48  system_monitor_user.o(i.Sys_BlockDelay)
    Sys_Exact_100ms_Tasks                    0x00001f1d   Thumb Code     2  tasks.o(i.Sys_Exact_100ms_Tasks)
    Sys_Exact_50us_Tasks                     0x00001f27   Thumb Code     8  tasks.o(i.Sys_Exact_50us_Tasks)
    Sys_Force_Read_KL15_Voltage              0x00001f2f   Thumb Code    12  system_monitor_user.o(i.Sys_Force_Read_KL15_Voltage)
    Sys_Force_Read_KL30_Voltage              0x00001f3b   Thumb Code    12  system_monitor_user.o(i.Sys_Force_Read_KL30_Voltage)
    Sys_Get_ms_Rolling_Counter               0x00001f49   Thumb Code     6  system_monitor_user.o(i.Sys_Get_ms_Rolling_Counter)
    Sys_Init                                 0x00001f55   Thumb Code    52  sys_scheduler.o(i.Sys_Init)
    Sys_KL30_Init                            0x00001f95   Thumb Code    34  system_monitor_user.o(i.Sys_KL30_Init)
    Sys_LogicProcess                         0x00001fc1   Thumb Code     2  system_monitor_user.o(i.Sys_LogicProcess)
    Sys_Rolling                              0x00001fc5   Thumb Code    30  system_monitor_user.o(i.Sys_Rolling)
    Sys_RollingClear                         0x00001fed   Thumb Code     8  system_monitor_user.o(i.Sys_RollingClear)
    Sys_Run_Mode_100ms_Tasks                 0x00001ff9   Thumb Code    26  tasks.o(i.Sys_Run_Mode_100ms_Tasks)
    Sys_Run_Mode_10ms_Tasks                  0x00002019   Thumb Code     8  tasks.o(i.Sys_Run_Mode_10ms_Tasks)
    Sys_Run_Mode_20ms_Tasks                  0x00002021   Thumb Code     2  tasks.o(i.Sys_Run_Mode_20ms_Tasks)
    Sys_Run_Mode_2ms_Tasks                   0x00002023   Thumb Code    14  tasks.o(i.Sys_Run_Mode_2ms_Tasks)
    Sys_Run_Mode_50ms_Tasks                  0x00002031   Thumb Code     2  tasks.o(i.Sys_Run_Mode_50ms_Tasks)
    Sys_Run_Mode_5ms_Tasks                   0x00002033   Thumb Code     2  tasks.o(i.Sys_Run_Mode_5ms_Tasks)
    Sys_Run_Mode_Pseudo_Real_Time_Tasks      0x00002035   Thumb Code    12  tasks.o(i.Sys_Run_Mode_Pseudo_Real_Time_Tasks)
    Sys_Scheduling_Service                   0x00002041   Thumb Code   222  sys_scheduler.o(i.Sys_Scheduling_Service)
    Sys_Set_DebounceTimer                    0x00002129   Thumb Code    20  system_monitor.o(i.Sys_Set_DebounceTimer)
    Sys_Set_VolRange                         0x0000214d   Thumb Code    92  system_monitor.o(i.Sys_Set_VolRange)
    Sys_Startup_Init                         0x000021b5   Thumb Code    36  init.o(i.Sys_Startup_Init)
    Sys_Tick_Timer_Call_Back_Reg             0x000021d9   Thumb Code    12  sys_tick.o(i.Sys_Tick_Timer_Call_Back_Reg)
    Sys_Tick_Timer_Start                     0x000021e9   Thumb Code    74  sys_tick.o(i.Sys_Tick_Timer_Start)
    Sys_WakeUp_Init                          0x0000224d   Thumb Code    34  system_monitor_user.o(i.Sys_WakeUp_Init)
    SystemCoreClockUpdate                    0x00002279   Thumb Code    12  system_bat32g137.o(i.SystemCoreClockUpdate)
    SystemInit                               0x00002289   Thumb Code    88  system_bat32g137.o(i.SystemInit)
    System_FUN_KL30_Status_Get               0x000022fd   Thumb Code     6  system_monitor.o(i.System_FUN_KL30_Status_Get)
    System_Fast_WakeUp                       0x00002309   Thumb Code   196  system_monitor.o(i.System_Fast_WakeUp)
    System_LINE_KL15                         0x000023e5   Thumb Code    16  system_monitor_user.o(i.System_LINE_KL15)
    System_Monitor_KL30Init                  0x000023f5   Thumb Code   218  system_monitor.o(i.System_Monitor_KL30Init)
    System_Monitor_WakeupInit                0x00002521   Thumb Code   218  system_monitor.o(i.System_Monitor_WakeupInit)
    TFT_CreateCRCCheckSum                    0x0000264d   Thumb Code    62  mcu_core_protocol.o(i.TFT_CreateCRCCheckSum)
    UART2_BaudRate                           0x00002695   Thumb Code    72  sci.o(i.UART2_BaudRate)
    UART2_Init                               0x000026e5   Thumb Code   282  sci.o(i.UART2_Init)
    UART2_Start                              0x00002831   Thumb Code    76  sci.o(i.UART2_Start)
    UART_BaudRateCal                         0x00002881   Thumb Code   110  sci.o(i.UART_BaudRateCal)
    UART_Ch2_Send_Multiple_Byte              0x000028f9   Thumb Code    68  sci_user.o(i.UART_Ch2_Send_Multiple_Byte)
    WDT_Restart                              0x00002951   Thumb Code     8  wdt.o(i.WDT_Restart)
    __ARM_common_switch8                     0x0000295d   Thumb Code    28  gpio.o(i.__ARM_common_switch8)
    main                                     0x00002a21   Thumb Code    16  main.o(i.main)
    IRQ11_Handler                            0x00002a39   Thumb Code     0  sci_user.o(i.uart0_interrupt_receive)
    uart0_interrupt_receive                  0x00002a39   Thumb Code   116  sci_user.o(i.uart0_interrupt_receive)
    IRQ10_Handler                            0x00002ac1   Thumb Code     0  sci_user.o(i.uart0_interrupt_send)
    uart0_interrupt_send                     0x00002ac1   Thumb Code    54  sci_user.o(i.uart0_interrupt_send)
    u8ADCChList                              0x00002b30   Data           4  analog_signals.o(.constdata)
    stADCChCfg                               0x00002b34   Data          64  analog_signals.o(.constdata)
    stADCResList                             0x00002b74   Data          64  analog_signals.o(.constdata)
    sps_tbl                                  0x00002bb4   Data          32  sci.o(.constdata)
    g_stLineInAttribute                      0x00002bd4   Data         168  line_in.o(.constdata)
    Region$$Table$$Base                      0x00002ea4   Number         0  anon$$obj.o(Region$$Table)
    Region$$Table$$Limit                     0x00002ec4   Number         0  anon$$obj.o(Region$$Table)
    g_u16SysRollingCounter50us               0x20000000   Data           2  sys_tick.o(.data)
    g_u16SysRollingCounter1ms                0x20000002   Data           2  sys_tick.o(.data)
    u8ADCSequenceRunningFlag                 0x20000004   Data           1  adc.o(.data)
    u8ADCChannelCount                        0x20000005   Data           1  adc.o(.data)
    u16ADCChannelResult                      0x20000006   Data           8  adc.o(.data)
    u16ADCRefVoltage                         0x2000000e   Data           2  analog_signals.o(.data)
    stADCCtrl                                0x20000010   Data           4  analog_signals.o(.data)
    u16ADCSample                             0x20000014   Data           8  analog_signals.o(.data)
    gp_uart0_tx_address                      0x2000001c   Data           4  sci.o(.data)
    g_uart0_tx_count                         0x20000020   Data           2  sci.o(.data)
    gp_uart0_rx_address                      0x20000024   Data           4  sci.o(.data)
    g_uart0_rx_count                         0x20000028   Data           2  sci.o(.data)
    g_uart0_rx_length                        0x2000002a   Data           2  sci.o(.data)
    gp_spi00_rx_address                      0x2000002c   Data           4  sci.o(.data)
    g_spi00_rx_length                        0x20000030   Data           2  sci.o(.data)
    g_spi00_rx_count                         0x20000032   Data           2  sci.o(.data)
    gp_spi00_tx_address                      0x20000034   Data           4  sci.o(.data)
    g_spi00_tx_length                        0x20000038   Data           2  sci.o(.data)
    g_spi00_tx_count                         0x2000003a   Data           2  sci.o(.data)
    gp_spi01_rx_address                      0x2000003c   Data           4  sci.o(.data)
    g_spi01_rx_length                        0x20000040   Data           2  sci.o(.data)
    g_spi01_rx_count                         0x20000042   Data           2  sci.o(.data)
    gp_spi01_tx_address                      0x20000044   Data           4  sci.o(.data)
    g_spi01_tx_length                        0x20000048   Data           2  sci.o(.data)
    g_spi01_tx_count                         0x2000004a   Data           2  sci.o(.data)
    g_iic00_master_status_flag               0x2000004c   Data           1  sci.o(.data)
    gp_iic00_tx_address                      0x20000050   Data           4  sci.o(.data)
    g_iic00_tx_count                         0x20000054   Data           2  sci.o(.data)
    gp_iic00_rx_address                      0x20000058   Data           4  sci.o(.data)
    g_iic00_rx_count                         0x2000005c   Data           2  sci.o(.data)
    g_iic00_rx_length                        0x2000005e   Data           2  sci.o(.data)
    g_iic01_master_status_flag               0x20000060   Data           1  sci.o(.data)
    gp_iic01_tx_address                      0x20000064   Data           4  sci.o(.data)
    g_iic01_tx_count                         0x20000068   Data           2  sci.o(.data)
    gp_iic01_rx_address                      0x2000006c   Data           4  sci.o(.data)
    g_iic01_rx_count                         0x20000070   Data           2  sci.o(.data)
    g_iic01_rx_length                        0x20000072   Data           2  sci.o(.data)
    gp_uart1_tx_address                      0x20000074   Data           4  sci.o(.data)
    g_uart1_tx_count                         0x20000078   Data           2  sci.o(.data)
    gp_uart1_rx_address                      0x2000007c   Data           4  sci.o(.data)
    g_uart1_rx_count                         0x20000080   Data           2  sci.o(.data)
    g_uart1_rx_length                        0x20000082   Data           2  sci.o(.data)
    gp_spi10_rx_address                      0x20000084   Data           4  sci.o(.data)
    g_spi10_rx_length                        0x20000088   Data           2  sci.o(.data)
    g_spi10_rx_count                         0x2000008a   Data           2  sci.o(.data)
    gp_spi10_tx_address                      0x2000008c   Data           4  sci.o(.data)
    g_spi10_tx_length                        0x20000090   Data           2  sci.o(.data)
    g_spi10_tx_count                         0x20000092   Data           2  sci.o(.data)
    gp_spi11_rx_address                      0x20000094   Data           4  sci.o(.data)
    g_spi11_rx_length                        0x20000098   Data           2  sci.o(.data)
    g_spi11_rx_count                         0x2000009a   Data           2  sci.o(.data)
    gp_spi11_tx_address                      0x2000009c   Data           4  sci.o(.data)
    g_spi11_tx_length                        0x200000a0   Data           2  sci.o(.data)
    g_spi11_tx_count                         0x200000a2   Data           2  sci.o(.data)
    g_iic10_master_status_flag               0x200000a4   Data           1  sci.o(.data)
    gp_iic10_tx_address                      0x200000a8   Data           4  sci.o(.data)
    g_iic10_tx_count                         0x200000ac   Data           2  sci.o(.data)
    gp_iic10_rx_address                      0x200000b0   Data           4  sci.o(.data)
    g_iic10_rx_count                         0x200000b4   Data           2  sci.o(.data)
    g_iic10_rx_length                        0x200000b6   Data           2  sci.o(.data)
    g_iic11_master_status_flag               0x200000b8   Data           1  sci.o(.data)
    gp_iic11_tx_address                      0x200000bc   Data           4  sci.o(.data)
    g_iic11_tx_count                         0x200000c0   Data           2  sci.o(.data)
    gp_iic11_rx_address                      0x200000c4   Data           4  sci.o(.data)
    g_iic11_rx_count                         0x200000c8   Data           2  sci.o(.data)
    g_iic11_rx_length                        0x200000ca   Data           2  sci.o(.data)
    gp_uart2_tx_address                      0x200000cc   Data           4  sci.o(.data)
    g_uart2_tx_count                         0x200000d0   Data           2  sci.o(.data)
    gp_uart2_rx_address                      0x200000d4   Data           4  sci.o(.data)
    g_uart2_rx_count                         0x200000d8   Data           2  sci.o(.data)
    g_uart2_rx_length                        0x200000da   Data           2  sci.o(.data)
    gp_spi20_rx_address                      0x200000dc   Data           4  sci.o(.data)
    g_spi20_rx_length                        0x200000e0   Data           2  sci.o(.data)
    g_spi20_rx_count                         0x200000e2   Data           2  sci.o(.data)
    gp_spi20_tx_address                      0x200000e4   Data           4  sci.o(.data)
    g_spi20_tx_length                        0x200000e8   Data           2  sci.o(.data)
    g_spi20_tx_count                         0x200000ea   Data           2  sci.o(.data)
    gp_spi21_rx_address                      0x200000ec   Data           4  sci.o(.data)
    g_spi21_rx_length                        0x200000f0   Data           2  sci.o(.data)
    g_spi21_rx_count                         0x200000f2   Data           2  sci.o(.data)
    gp_spi21_tx_address                      0x200000f4   Data           4  sci.o(.data)
    g_spi21_tx_length                        0x200000f8   Data           2  sci.o(.data)
    g_spi21_tx_count                         0x200000fa   Data           2  sci.o(.data)
    g_iic20_master_status_flag               0x200000fc   Data           1  sci.o(.data)
    gp_iic20_tx_address                      0x20000100   Data           4  sci.o(.data)
    g_iic20_tx_count                         0x20000104   Data           2  sci.o(.data)
    gp_iic20_rx_address                      0x20000108   Data           4  sci.o(.data)
    g_iic20_rx_count                         0x2000010c   Data           2  sci.o(.data)
    g_iic20_rx_length                        0x2000010e   Data           2  sci.o(.data)
    g_iic21_master_status_flag               0x20000110   Data           1  sci.o(.data)
    gp_iic21_tx_address                      0x20000114   Data           4  sci.o(.data)
    g_iic21_tx_count                         0x20000118   Data           2  sci.o(.data)
    gp_iic21_rx_address                      0x2000011c   Data           4  sci.o(.data)
    g_iic21_rx_count                         0x20000120   Data           2  sci.o(.data)
    g_iic21_rx_length                        0x20000122   Data           2  sci.o(.data)
    g_iic00_tx_end                           0x20000130   Data           1  sci_user.o(.data)
    g_iic00_rx_end                           0x20000131   Data           1  sci_user.o(.data)
    g_iic01_tx_end                           0x20000132   Data           1  sci_user.o(.data)
    g_iic01_rx_end                           0x20000133   Data           1  sci_user.o(.data)
    g_iic10_tx_end                           0x20000134   Data           1  sci_user.o(.data)
    g_iic10_rx_end                           0x20000135   Data           1  sci_user.o(.data)
    g_iic11_tx_end                           0x20000136   Data           1  sci_user.o(.data)
    g_iic11_rx_end                           0x20000137   Data           1  sci_user.o(.data)
    g_iic20_tx_end                           0x20000138   Data           1  sci_user.o(.data)
    g_iic20_rx_end                           0x20000139   Data           1  sci_user.o(.data)
    g_iic21_tx_end                           0x2000013a   Data           1  sci_user.o(.data)
    g_iic21_rx_end                           0x2000013b   Data           1  sci_user.o(.data)
    g_uart2_tx_state                         0x2000013c   Data           1  sci_user.o(.data)
    g_enLineInPowerStatus                    0x2000013e   Data           1  line_in.o(.data)
    SysWakeUpMode                            0x20000140   Data           1  system_monitor.o(.data)
    u32SysRollingCounter                     0x20000178   Data           4  system_monitor_user.o(.data)
    PackageCnt                               0x2000019c   Data           1  mcu_core_protocol.o(.data)
    Msg_12_Rec_Sta                           0x200001a0   Data           8  mcu_core_protocol.o(.data)
    SendLength                               0x200001a8   Data           1  mcu_core_protocol.o(.data)
    Send_ID_01_00                            0x200001a9   Data           2  mcu_core_protocol.o(.data)
    Send_ID_01_01                            0x200001ab   Data           3  mcu_core_protocol.o(.data)
    Send_ID_01_03                            0x200001ae   Data           6  mcu_core_protocol.o(.data)
    Rec_Dat_12                               0x200001b4   Data           7  mcu_core_protocol.o(.data)
    SendCtrl_Tbl                             0x200001bc   Data          24  mcu_core_protocol.o(.data)
    SystemCoreClock                          0x200001d4   Data           4  system_bat32g137.o(.data)
    pfnSysTickCallBack                       0x200001d8   Data          12  sys_tick.o(.bss)
    g_stSysTickTimer                         0x200001e4   Data          12  sys_tick.o(.bss)
    stADCData                                0x200001f0   Data          16  analog_signals.o(.bss)
    SysScheduling                            0x20000200   Data          14  sys_scheduler.o(.bss)
    g_stLineInControl                        0x2000020e   Data          84  line_in.o(.bss)
    pFuncPower                               0x20000264   Data          44  powermanagement.o(.bss)
    SysFun_KL30Monitor                       0x20000290   Data          12  system_monitor.o(.bss)
    SysFun_KL15Monitor                       0x2000029c   Data          12  system_monitor.o(.bss)
    SysNM_KL30Monitor                        0x200002a8   Data          12  system_monitor.o(.bss)
    SysNM_KL15Monitor                        0x200002b4   Data          12  system_monitor.o(.bss)
    Uart2_tx_buf                             0x200002c0   Data         100  mcu_core_protocol.o(.bss)
    Uart2_rx_buf                             0x20000324   Data         100  mcu_core_protocol.o(.bss)
    Send_ID_01_02                            0x20000388   Data          22  mcu_core_protocol.o(.bss)
    Send_ID_02                               0x2000039e   Data          11  mcu_core_protocol.o(.bss)
    Send_ID_06                               0x200003a9   Data          57  mcu_core_protocol.o(.bss)
    __libspace_start                         0x200003e4   Data          96  libspace.o(.bss)
    __temporary_stack_top$libspace           0x20000444   Data           0  libspace.o(.bss)



==============================================================================

Memory Map of the image

  Image Entry point : 0x000000c5

  Load Region LR_IROM1 (Base: 0x00000000, Size: 0x0000309c, Max: 0x00020000, ABSOLUTE, COMPRESSED[0x00002ef8])

    Execution Region ER_IROM1 (Exec base: 0x00000000, Load base: 0x00000000, Size: 0x00002ec4, Max: 0x00020000, ABSOLUTE)

    Exec Addr    Load Addr    Size         Type   Attr      Idx    E Section Name        Object

    0x00000000   0x00000000   0x000000c0   Data   RO         2447    RESET               startup_bat32g137.o
    0x000000c0   0x000000c0   0x00000004   Data   RO         2458    .ARM.__AT_0x000000C0  system_bat32g137.o
    0x000000c4   0x000000c4   0x00000008   Code   RO         2509  * !!!main             c_p.l(__main.o)
    0x000000cc   0x000000cc   0x0000003c   Code   RO         2686    !!!scatter          c_p.l(__scatter.o)
    0x00000108   0x00000108   0x0000001c   Code   RO         2688    !!handler_zi        c_p.l(__scatter_zi.o)
    0x00000124   0x00000124   0x00000002   Code   RO         2551    .ARM.Collect$$libinit$$00000000  c_p.l(libinit.o)
    0x00000126   0x00000126   0x00000000   Code   RO         2565    .ARM.Collect$$libinit$$00000002  c_p.l(libinit2.o)
    0x00000126   0x00000126   0x00000000   Code   RO         2567    .ARM.Collect$$libinit$$00000004  c_p.l(libinit2.o)
    0x00000126   0x00000126   0x00000000   Code   RO         2570    .ARM.Collect$$libinit$$0000000A  c_p.l(libinit2.o)
    0x00000126   0x00000126   0x00000000   Code   RO         2572    .ARM.Collect$$libinit$$0000000C  c_p.l(libinit2.o)
    0x00000126   0x00000126   0x00000000   Code   RO         2574    .ARM.Collect$$libinit$$0000000E  c_p.l(libinit2.o)
    0x00000126   0x00000126   0x00000000   Code   RO         2577    .ARM.Collect$$libinit$$00000011  c_p.l(libinit2.o)
    0x00000126   0x00000126   0x00000000   Code   RO         2579    .ARM.Collect$$libinit$$00000013  c_p.l(libinit2.o)
    0x00000126   0x00000126   0x00000000   Code   RO         2581    .ARM.Collect$$libinit$$00000015  c_p.l(libinit2.o)
    0x00000126   0x00000126   0x00000000   Code   RO         2583    .ARM.Collect$$libinit$$00000017  c_p.l(libinit2.o)
    0x00000126   0x00000126   0x00000000   Code   RO         2585    .ARM.Collect$$libinit$$00000019  c_p.l(libinit2.o)
    0x00000126   0x00000126   0x00000000   Code   RO         2587    .ARM.Collect$$libinit$$0000001B  c_p.l(libinit2.o)
    0x00000126   0x00000126   0x00000000   Code   RO         2589    .ARM.Collect$$libinit$$0000001D  c_p.l(libinit2.o)
    0x00000126   0x00000126   0x00000000   Code   RO         2591    .ARM.Collect$$libinit$$0000001F  c_p.l(libinit2.o)
    0x00000126   0x00000126   0x00000000   Code   RO         2593    .ARM.Collect$$libinit$$00000021  c_p.l(libinit2.o)
    0x00000126   0x00000126   0x00000000   Code   RO         2595    .ARM.Collect$$libinit$$00000023  c_p.l(libinit2.o)
    0x00000126   0x00000126   0x00000000   Code   RO         2597    .ARM.Collect$$libinit$$00000025  c_p.l(libinit2.o)
    0x00000126   0x00000126   0x00000000   Code   RO         2601    .ARM.Collect$$libinit$$0000002C  c_p.l(libinit2.o)
    0x00000126   0x00000126   0x00000000   Code   RO         2603    .ARM.Collect$$libinit$$0000002E  c_p.l(libinit2.o)
    0x00000126   0x00000126   0x00000000   Code   RO         2605    .ARM.Collect$$libinit$$00000030  c_p.l(libinit2.o)
    0x00000126   0x00000126   0x00000000   Code   RO         2607    .ARM.Collect$$libinit$$00000032  c_p.l(libinit2.o)
    0x00000126   0x00000126   0x00000002   Code   RO         2608    .ARM.Collect$$libinit$$00000033  c_p.l(libinit2.o)
    0x00000128   0x00000128   0x00000002   Code   RO         2639    .ARM.Collect$$libshutdown$$00000000  c_p.l(libshutdown.o)
    0x0000012a   0x0000012a   0x00000000   Code   RO         2665    .ARM.Collect$$libshutdown$$00000002  c_p.l(libshutdown2.o)
    0x0000012a   0x0000012a   0x00000000   Code   RO         2667    .ARM.Collect$$libshutdown$$00000004  c_p.l(libshutdown2.o)
    0x0000012a   0x0000012a   0x00000000   Code   RO         2669    .ARM.Collect$$libshutdown$$00000006  c_p.l(libshutdown2.o)
    0x0000012a   0x0000012a   0x00000000   Code   RO         2672    .ARM.Collect$$libshutdown$$00000009  c_p.l(libshutdown2.o)
    0x0000012a   0x0000012a   0x00000000   Code   RO         2675    .ARM.Collect$$libshutdown$$0000000C  c_p.l(libshutdown2.o)
    0x0000012a   0x0000012a   0x00000000   Code   RO         2677    .ARM.Collect$$libshutdown$$0000000E  c_p.l(libshutdown2.o)
    0x0000012a   0x0000012a   0x00000000   Code   RO         2680    .ARM.Collect$$libshutdown$$00000011  c_p.l(libshutdown2.o)
    0x0000012a   0x0000012a   0x00000002   Code   RO         2681    .ARM.Collect$$libshutdown$$00000012  c_p.l(libshutdown2.o)
    0x0000012c   0x0000012c   0x00000000   Code   RO         2511    .ARM.Collect$$rtentry$$00000000  c_p.l(__rtentry.o)
    0x0000012c   0x0000012c   0x00000000   Code   RO         2521    .ARM.Collect$$rtentry$$00000002  c_p.l(__rtentry2.o)
    0x0000012c   0x0000012c   0x00000006   Code   RO         2533    .ARM.Collect$$rtentry$$00000004  c_p.l(__rtentry4.o)
    0x00000132   0x00000132   0x00000000   Code   RO         2523    .ARM.Collect$$rtentry$$00000009  c_p.l(__rtentry2.o)
    0x00000132   0x00000132   0x00000004   Code   RO         2524    .ARM.Collect$$rtentry$$0000000A  c_p.l(__rtentry2.o)
    0x00000136   0x00000136   0x00000000   Code   RO         2526    .ARM.Collect$$rtentry$$0000000C  c_p.l(__rtentry2.o)
    0x00000136   0x00000136   0x00000008   Code   RO         2527    .ARM.Collect$$rtentry$$0000000D  c_p.l(__rtentry2.o)
    0x0000013e   0x0000013e   0x00000002   Code   RO         2556    .ARM.Collect$$rtexit$$00000000  c_p.l(rtexit.o)
    0x00000140   0x00000140   0x00000000   Code   RO         2612    .ARM.Collect$$rtexit$$00000002  c_p.l(rtexit2.o)
    0x00000140   0x00000140   0x00000004   Code   RO         2613    .ARM.Collect$$rtexit$$00000003  c_p.l(rtexit2.o)
    0x00000144   0x00000144   0x00000006   Code   RO         2614    .ARM.Collect$$rtexit$$00000004  c_p.l(rtexit2.o)
    0x0000014a   0x0000014a   0x00000002   PAD
    0x0000014c   0x0000014c   0x00000080   Code   RO         2448    .text               startup_bat32g137.o
    0x000001cc   0x000001cc   0x00000030   Code   RO         2499    .text               c_p.l(llmul.o)
    0x000001fc   0x000001fc   0x00000102   Code   RO         2501    .text               c_p.l(lludiv.o)
    0x000002fe   0x000002fe   0x0000015a   Code   RO         2503    .text               c_p.l(aeabi_sdiv.o)
    0x00000458   0x00000458   0x00000006   Code   RO         2507    .text               c_p.l(heapauxi.o)
    0x0000045e   0x0000045e   0x0000003e   Code   RO         2537    .text               c_p.l(sys_stackheap_outer.o)
    0x0000049c   0x0000049c   0x00000010   Code   RO         2540    .text               c_p.l(exit.o)
    0x000004ac   0x000004ac   0x00000008   Code   RO         2552    .text               c_p.l(libspace.o)
    0x000004b4   0x000004b4   0x0000000c   Code   RO         2609    .text               c_p.l(sys_exit.o)
    0x000004c0   0x000004c0   0x00000002   Code   RO         2628    .text               c_p.l(use_no_semi.o)
    0x000004c2   0x000004c2   0x00000000   Code   RO         2630    .text               c_p.l(indicate_semi.o)
    0x000004c2   0x000004c2   0x00000056   Code   RO         2684    .text               c_p.l(__dczerorl2.o)
    0x00000518   0x00000518   0x0000016c   Code   RO          468    i.ADC_Conv_Single_Channel  analog_signals.o
    0x00000684   0x00000684   0x00000034   Code   RO          370    i.ADC_Data_Calibrate  analog_circuits.o
    0x000006b8   0x000006b8   0x0000002c   Code   RO          218    i.ADC_Get_Conversion_Result  adc.o
    0x000006e4   0x000006e4   0x0000000c   Code   RO          219    i.ADC_Get_Conversion_Status  adc.o
    0x000006f0   0x000006f0   0x000000b8   Code   RO          220    i.ADC_Init          adc.o
    0x000007a8   0x000007a8   0x00000034   Code   RO          371    i.ADC_Input_Voltage_Calc  analog_circuits.o
    0x000007dc   0x000007dc   0x00000018   Code   RO          469    i.ADC_Read_Signal   analog_signals.o
    0x000007f4   0x000007f4   0x00000018   Code   RO          470    i.ADC_Read_Signal_Valid  analog_signals.o
    0x0000080c   0x0000080c   0x00000030   Code   RO          228    i.ADC_Start         adc.o
    0x0000083c   0x0000083c   0x00000028   Code   RO          229    i.ADC_Start_Conversion  adc.o
    0x00000864   0x00000864   0x00000028   Code   RO          230    i.ADC_Stop          adc.o
    0x0000088c   0x0000088c   0x00000008   Code   RO          231    i.ADC_Stop_Conversion  adc.o
    0x00000894   0x00000894   0x00000088   Code   RO          383    i.ADC_Voltage_Calc_Circuit102  analog_circuits.o
    0x0000091c   0x0000091c   0x0000006c   Code   RO          471    i.Analog_Signal_Conv_Init  analog_signals.o
    0x00000988   0x00000988   0x0000006c   Code   RO          232    i.Analog_Signal_Conv_Real_Time_Run  adc.o
    0x000009f4   0x000009f4   0x00000254   Code   RO          472    i.Analog_Signal_Conv_Service  analog_signals.o
    0x00000c48   0x00000c48   0x000000ac   Code   RO         2454    i.CLK_GetCoreFreq   system_bat32g137.o
    0x00000cf4   0x00000cf4   0x0000000c   Code   RO         2185    i.Common_Get_ConnectPhoneSts  common_interface.o
    0x00000d00   0x00000d00   0x0000000c   Code   RO         2186    i.Common_Get_DispMode  common_interface.o
    0x00000d0c   0x00000d0c   0x0000000c   Code   RO         2192    i.Common_Get_IG_Sts  common_interface.o
    0x00000d18   0x00000d18   0x0000000c   Code   RO         2193    i.Common_Get_IG_Sts_Valid  common_interface.o
    0x00000d24   0x00000d24   0x0000000c   Code   RO         2194    i.Common_Get_Language  common_interface.o
    0x00000d30   0x00000d30   0x0000000c   Code   RO         2195    i.Common_Get_Theme  common_interface.o
    0x00000d3c   0x00000d3c   0x0000026c   Code   RO            4    i.GPIO_Init         gpio.o
    0x00000fa8   0x00000fa8   0x00000288   Code   RO         2394    i.Get_ID_01_Data    mcu_core_protocol.o
    0x00001230   0x00001230   0x00000048   Code   RO         2395    i.Get_ID_02_Data    mcu_core_protocol.o
    0x00001278   0x00001278   0x0000000c   Code   RO         1228    i.Get_Uart2_State   sci_user.o
    0x00001284   0x00001284   0x00000044   Code   RO          233    i.INTC_ClearPendingIRQ  adc.o
    0x000012c8   0x000012c8   0x00000044   Code   RO          566    i.INTC_ClearPendingIRQ  sci.o
    0x0000130c   0x0000130c   0x00000044   Code   RO         1229    i.INTC_ClearPendingIRQ  sci_user.o
    0x00001350   0x00001350   0x00000040   Code   RO          234    i.INTC_DisableIRQ   adc.o
    0x00001390   0x00001390   0x00000040   Code   RO          567    i.INTC_DisableIRQ   sci.o
    0x000013d0   0x000013d0   0x00000040   Code   RO          568    i.INTC_EnableIRQ    sci.o
    0x00001410   0x00001410   0x00000048   Code   RO         1230    i.IRQ07_Handler     sci_user.o
    0x00001458   0x00001458   0x000000dc   Code   RO         1231    i.IRQ08_Handler     sci_user.o
    0x00001534   0x00001534   0x00000016   Code   RO         1570    i.LINE_IN_Get_ABS   line_in.o
    0x0000154a   0x0000154a   0x00000016   Code   RO         1571    i.LINE_IN_Get_Gear_1  line_in.o
    0x00001560   0x00001560   0x00000016   Code   RO         1572    i.LINE_IN_Get_Gear_2  line_in.o
    0x00001576   0x00001576   0x00000016   Code   RO         1573    i.LINE_IN_Get_Gear_3  line_in.o
    0x0000158c   0x0000158c   0x00000016   Code   RO         1574    i.LINE_IN_Get_Gear_4  line_in.o
    0x000015a2   0x000015a2   0x00000016   Code   RO         1575    i.LINE_IN_Get_Gear_5  line_in.o
    0x000015b8   0x000015b8   0x00000016   Code   RO         1576    i.LINE_IN_Get_Gear_6  line_in.o
    0x000015ce   0x000015ce   0x00000016   Code   RO         1577    i.LINE_IN_Get_Gear_N  line_in.o
    0x000015e4   0x000015e4   0x00000016   Code   RO         1578    i.LINE_IN_Get_HighBeam  line_in.o
    0x000015fa   0x000015fa   0x00000016   Code   RO         1579    i.LINE_IN_Get_Key1  line_in.o
    0x00001610   0x00001610   0x00000016   Code   RO         1580    i.LINE_IN_Get_Key2  line_in.o
    0x00001626   0x00001626   0x00000016   Code   RO         1581    i.LINE_IN_Get_LeftTurn  line_in.o
    0x0000163c   0x0000163c   0x00000016   Code   RO         1582    i.LINE_IN_Get_OilPressure  line_in.o
    0x00001652   0x00001652   0x00000016   Code   RO         1583    i.LINE_IN_Get_RightTurn  line_in.o
    0x00001668   0x00001668   0x000000d0   Code   RO         1584    i.Line_In_Debounce_Handle  line_in.o
    0x00001738   0x00001738   0x00000058   Code   RO         1585    i.Line_In_Debounce_Service  line_in.o
    0x00001790   0x00001790   0x00000040   Code   RO         1587    i.Line_In_KL15_OFF_Init  line_in.o
    0x000017d0   0x000017d0   0x00000040   Code   RO         1588    i.Line_In_KL15_ON_Init  line_in.o
    0x00001810   0x00001810   0x00000038   Code   RO         1589    i.Line_In_KL30_Init  line_in.o
    0x00001848   0x00001848   0x000000ac   Code   RO         2396    i.MCU_Send_Service  mcu_core_protocol.o
    0x000018f4   0x000018f4   0x00000024   Code   RO           12    i.PORT_ClrBit       gpio.o
    0x00001918   0x00001918   0x0000001c   Code   RO           13    i.PORT_GetBit       gpio.o
    0x00001934   0x00001934   0x00000198   Code   RO           14    i.PORT_Init         gpio.o
    0x00001acc   0x00001acc   0x00000024   Code   RO           15    i.PORT_SetBit       gpio.o
    0x00001af0   0x00001af0   0x00000040   Code   RO         1716    i.PowerMemInit      powermanagement.o
    0x00001b30   0x00001b30   0x00000002   Code   RO         1754    i.Power_IG_LVP_Init  powermanagement_user.o
    0x00001b32   0x00001b32   0x00000008   Code   RO         1755    i.Power_IG_OFF_Init  powermanagement_user.o
    0x00001b3a   0x00001b3a   0x00000008   Code   RO         1756    i.Power_IG_ON_Init  powermanagement_user.o
    0x00001b42   0x00001b42   0x00000002   Code   RO         1757    i.Power_IG_OVP_Init  powermanagement_user.o
    0x00001b44   0x00001b44   0x0000000c   Code   RO         1758    i.Power_KL30_Init   powermanagement_user.o
    0x00001b50   0x00001b50   0x00000028   Code   RO         1717    i.Power_Management_Init  powermanagement.o
    0x00001b78   0x00001b78   0x00000068   Code   RO         1759    i.Power_Management_Lib_Init  powermanagement_user.o
    0x00001be0   0x00001be0   0x00000124   Code   RO         1718    i.Power_Management_Service  powermanagement.o
    0x00001d04   0x00001d04   0x0000000a   Code   RO         1760    i.Power_Sleep_Init  powermanagement_user.o
    0x00001d0e   0x00001d0e   0x0000002c   Code   RO         1761    i.Power_Stay_OFF    powermanagement_user.o
    0x00001d3a   0x00001d3a   0x0000003c   Code   RO         1762    i.Power_Stay_ON     powermanagement_user.o
    0x00001d76   0x00001d76   0x00000004   Code   RO         1763    i.Power_Stay_Protect  powermanagement_user.o
    0x00001d7a   0x00001d7a   0x00000004   Code   RO         1764    i.Power_Stay_Sleep  powermanagement_user.o
    0x00001d7e   0x00001d7e   0x0000000c   Code   RO         1765    i.Power_Wakeup_Init  powermanagement_user.o
    0x00001d8a   0x00001d8a   0x00000010   Code   RO         2068    i.RTE_ForceRead_KL15_Voltage  rte_adc.o
    0x00001d9a   0x00001d9a   0x00000010   Code   RO         2069    i.RTE_ForceRead_KL30_Voltage  rte_adc.o
    0x00001daa   0x00001daa   0x00000002   PAD
    0x00001dac   0x00001dac   0x00000084   Code   RO         2397    i.Send_To_Core      mcu_core_protocol.o
    0x00001e30   0x00001e30   0x000000b0   Code   RO          158    i.SysTick_Handler   sys_tick.o
    0x00001ee0   0x00001ee0   0x00000034   Code   RO         1956    i.Sys_BlockDelay    system_monitor_user.o
    0x00001f14   0x00001f14   0x00000008   Code   RO         1475    i.Sys_Exact_100ms_Task_Handler  sys_scheduler.o
    0x00001f1c   0x00001f1c   0x00000002   Code   RO         1376    i.Sys_Exact_100ms_Tasks  tasks.o
    0x00001f1e   0x00001f1e   0x00000008   Code   RO         1476    i.Sys_Exact_50us_Task_Handler  sys_scheduler.o
    0x00001f26   0x00001f26   0x00000008   Code   RO         1377    i.Sys_Exact_50us_Tasks  tasks.o
    0x00001f2e   0x00001f2e   0x0000000c   Code   RO         1957    i.Sys_Force_Read_KL15_Voltage  system_monitor_user.o
    0x00001f3a   0x00001f3a   0x0000000c   Code   RO         1958    i.Sys_Force_Read_KL30_Voltage  system_monitor_user.o
    0x00001f46   0x00001f46   0x00000002   PAD
    0x00001f48   0x00001f48   0x0000000c   Code   RO         1959    i.Sys_Get_ms_Rolling_Counter  system_monitor_user.o
    0x00001f54   0x00001f54   0x00000040   Code   RO         1477    i.Sys_Init          sys_scheduler.o
    0x00001f94   0x00001f94   0x0000002c   Code   RO         1960    i.Sys_KL30_Init     system_monitor_user.o
    0x00001fc0   0x00001fc0   0x00000002   Code   RO         1961    i.Sys_LogicProcess  system_monitor_user.o
    0x00001fc2   0x00001fc2   0x00000002   PAD
    0x00001fc4   0x00001fc4   0x00000028   Code   RO         1966    i.Sys_Rolling       system_monitor_user.o
    0x00001fec   0x00001fec   0x0000000c   Code   RO         1967    i.Sys_RollingClear  system_monitor_user.o
    0x00001ff8   0x00001ff8   0x00000020   Code   RO         1378    i.Sys_Run_Mode_100ms_Tasks  tasks.o
    0x00002018   0x00002018   0x00000008   Code   RO         1379    i.Sys_Run_Mode_10ms_Tasks  tasks.o
    0x00002020   0x00002020   0x00000002   Code   RO         1380    i.Sys_Run_Mode_20ms_Tasks  tasks.o
    0x00002022   0x00002022   0x0000000e   Code   RO         1381    i.Sys_Run_Mode_2ms_Tasks  tasks.o
    0x00002030   0x00002030   0x00000002   Code   RO         1382    i.Sys_Run_Mode_50ms_Tasks  tasks.o
    0x00002032   0x00002032   0x00000002   Code   RO         1383    i.Sys_Run_Mode_5ms_Tasks  tasks.o
    0x00002034   0x00002034   0x0000000c   Code   RO         1384    i.Sys_Run_Mode_Pseudo_Real_Time_Tasks  tasks.o
    0x00002040   0x00002040   0x000000e8   Code   RO         1478    i.Sys_Scheduling_Service  sys_scheduler.o
    0x00002128   0x00002128   0x00000024   Code   RO         1853    i.Sys_Set_DebounceTimer  system_monitor.o
    0x0000214c   0x0000214c   0x00000068   Code   RO         1854    i.Sys_Set_VolRange  system_monitor.o
    0x000021b4   0x000021b4   0x00000024   Code   RO         1522    i.Sys_Startup_Init  init.o
    0x000021d8   0x000021d8   0x00000010   Code   RO          159    i.Sys_Tick_Timer_Call_Back_Reg  sys_tick.o
    0x000021e8   0x000021e8   0x00000064   Code   RO          160    i.Sys_Tick_Timer_Start  sys_tick.o
    0x0000224c   0x0000224c   0x0000002c   Code   RO         1968    i.Sys_WakeUp_Init   system_monitor_user.o
    0x00002278   0x00002278   0x00000010   Code   RO         2456    i.SystemCoreClockUpdate  system_bat32g137.o
    0x00002288   0x00002288   0x00000074   Code   RO         2457    i.SystemInit        system_bat32g137.o
    0x000022fc   0x000022fc   0x0000000c   Code   RO         1859    i.System_FUN_KL30_Status_Get  system_monitor.o
    0x00002308   0x00002308   0x000000dc   Code   RO         1860    i.System_Fast_WakeUp  system_monitor.o
    0x000023e4   0x000023e4   0x00000010   Code   RO         1969    i.System_LINE_KL15  system_monitor_user.o
    0x000023f4   0x000023f4   0x0000012c   Code   RO         1862    i.System_Monitor_KL30Init  system_monitor.o
    0x00002520   0x00002520   0x0000012c   Code   RO         1863    i.System_Monitor_WakeupInit  system_monitor.o
    0x0000264c   0x0000264c   0x00000048   Code   RO         2398    i.TFT_CreateCRCCheckSum  mcu_core_protocol.o
    0x00002694   0x00002694   0x00000050   Code   RO          633    i.UART2_BaudRate    sci.o
    0x000026e4   0x000026e4   0x0000014c   Code   RO          634    i.UART2_Init        sci.o
    0x00002830   0x00002830   0x00000050   Code   RO          637    i.UART2_Start       sci.o
    0x00002880   0x00002880   0x00000078   Code   RO          639    i.UART_BaudRateCal  sci.o
    0x000028f8   0x000028f8   0x00000058   Code   RO         1232    i.UART_Ch2_Send_Multiple_Byte  sci_user.o
    0x00002950   0x00002950   0x0000000c   Code   RO          134    i.WDT_Restart       wdt.o
    0x0000295c   0x0000295c   0x0000001c   Code   RO           97    i.__ARM_common_switch8  gpio.o
    0x00002978   0x00002978   0x00000018   Code   RO          236    i.__NVIC_ClearPendingIRQ  adc.o
    0x00002990   0x00002990   0x00000018   Code   RO          640    i.__NVIC_ClearPendingIRQ  sci.o
    0x000029a8   0x000029a8   0x00000078   Code   RO          162    i.__NVIC_SetPriority  sys_tick.o
    0x00002a20   0x00002a20   0x00000010   Code   RO         1333    i.main              main.o
    0x00002a30   0x00002a30   0x00000002   Code   RO         1233    i.uart0_callback_error  sci_user.o
    0x00002a32   0x00002a32   0x00000002   Code   RO         1234    i.uart0_callback_receiveend  sci_user.o
    0x00002a34   0x00002a34   0x00000002   Code   RO         1235    i.uart0_callback_sendend  sci_user.o
    0x00002a36   0x00002a36   0x00000002   Code   RO         1236    i.uart0_callback_softwareoverrun  sci_user.o
    0x00002a38   0x00002a38   0x00000088   Code   RO         1237    i.uart0_interrupt_receive  sci_user.o
    0x00002ac0   0x00002ac0   0x00000044   Code   RO         1238    i.uart0_interrupt_send  sci_user.o
    0x00002b04   0x00002b04   0x00000010   Code   RO         1239    i.uart2_callback_error  sci_user.o
    0x00002b14   0x00002b14   0x00000010   Code   RO         1240    i.uart2_callback_receiveend  sci_user.o
    0x00002b24   0x00002b24   0x0000000c   Code   RO         1241    i.uart2_callback_sendend  sci_user.o
    0x00002b30   0x00002b30   0x00000084   Data   RO          475    .constdata          analog_signals.o
    0x00002bb4   0x00002bb4   0x00000020   Data   RO          642    .constdata          sci.o
    0x00002bd4   0x00002bd4   0x000000a8   Data   RO         1592    .constdata          line_in.o
    0x00002c7c   0x00002c7c   0x00000028   Data   RO         1970    .constdata          system_monitor_user.o
    0x00002ca4   0x00002ca4   0x00000200   Data   RO         2400    .constdata          mcu_core_protocol.o
    0x00002ea4   0x00002ea4   0x00000020   Data   RO         2682    Region$$Table       anon$$obj.o


    Execution Region RW_IRAM1 (Exec base: 0x20000000, Load base: 0x00002ec4, Size: 0x00000948, Max: 0x00003000, ABSOLUTE, COMPRESSED[0x00000034])

    Exec Addr    Load Addr    Size         Type   Attr      Idx    E Section Name        Object

    0x20000000   COMPRESSED   0x00000004   Data   RW          164    .data               sys_tick.o
    0x20000004   COMPRESSED   0x0000000a   Data   RW          237    .data               adc.o
    0x2000000e   COMPRESSED   0x0000000e   Data   RW          476    .data               analog_signals.o
    0x2000001c   COMPRESSED   0x00000114   Data   RW          643    .data               sci.o
    0x20000130   COMPRESSED   0x0000000e   Data   RW         1242    .data               sci_user.o
    0x2000013e   COMPRESSED   0x00000001   Data   RW         1593    .data               line_in.o
    0x2000013f   COMPRESSED   0x00000001   Data   RW         1720    .data               powermanagement.o
    0x20000140   COMPRESSED   0x00000036   Data   RW         1868    .data               system_monitor.o
    0x20000176   COMPRESSED   0x00000002   PAD
    0x20000178   COMPRESSED   0x00000004   Data   RW         1971    .data               system_monitor_user.o
    0x2000017c   COMPRESSED   0x0000001e   Data   RW         2210    .data               common_interface.o
    0x2000019a   COMPRESSED   0x00000002   PAD
    0x2000019c   COMPRESSED   0x00000038   Data   RW         2401    .data               mcu_core_protocol.o
    0x200001d4   COMPRESSED   0x00000004   Data   RW         2459    .data               system_bat32g137.o
    0x200001d8        -       0x00000018   Zero   RW          163    .bss                sys_tick.o
    0x200001f0        -       0x00000010   Zero   RW          474    .bss                analog_signals.o
    0x20000200        -       0x0000000e   Zero   RW         1479    .bss                sys_scheduler.o
    0x2000020e        -       0x00000054   Zero   RW         1591    .bss                line_in.o
    0x20000262   COMPRESSED   0x00000002   PAD
    0x20000264        -       0x0000002c   Zero   RW         1719    .bss                powermanagement.o
    0x20000290        -       0x00000030   Zero   RW         1867    .bss                system_monitor.o
    0x200002c0        -       0x00000122   Zero   RW         2399    .bss                mcu_core_protocol.o
    0x200003e2   COMPRESSED   0x00000002   PAD
    0x200003e4        -       0x00000060   Zero   RW         2553    .bss                c_p.l(libspace.o)
    0x20000444   COMPRESSED   0x00000004   PAD
    0x20000448        -       0x00000100   Zero   RW         2446    HEAP                startup_bat32g137.o
    0x20000548        -       0x00000400   Zero   RW         2445    STACK               startup_bat32g137.o


==============================================================================

Image component sizes


      Code (inc. data)   RO Data    RW Data    ZI Data      Debug   Object Name

       640         92          0         10          0      35115   adc.o
       240          8          0          0          0       2516   analog_circuits.o
      1116         98        132         14         16       5631   analog_signals.o
        72         36          0         30          0       3750   common_interface.o
      1156         30          0          0          0      60746   gpio.o
        36          0          0          0          0        487   init.o
       788         50        168          1         84      12427   line_in.o
        16          0          0          0          0        455   main.o
      1096         56        512         56        290       9946   mcu_core_protocol.o
       396         42          0          1         44       4235   powermanagement.o
       270         46          0          0          0       8149   powermanagement_user.o
        32          0          0          0          0       1122   rte_adc.o
       832         92         32        276          0      35444   sci.o
       716        124          0         14          0      19565   sci_user.o
       128         28        192          0       1280       2140   startup_bat32g137.o
       312         22          0          0         14       3128   sys_scheduler.o
       412         58          0          4         24      16567   sys_tick.o
       304         94          4          4          0       2795   system_bat32g137.o
       972        222          0         54         48       7781   system_monitor.o
       246         44         40          4          0       6966   system_monitor_user.o
        82          6          0          0          0       4204   tasks.o
        12          4          0          0          0        430   wdt.o

    ----------------------------------------------------------------------
      9880       1152       1112        472       1804     243599   Object Totals
         0          0         32          0          0          0   (incl. Generated)
         6          0          0          4          4          0   (incl. Padding)

    ----------------------------------------------------------------------

      Code (inc. data)   RO Data    RW Data    ZI Data      Debug   Library Member Name

        86          0          0          0          0          0   __dczerorl2.o
         8          0          0          0          0         68   __main.o
         0          0          0          0          0          0   __rtentry.o
        12          0          0          0          0          0   __rtentry2.o
         6          0          0          0          0          0   __rtentry4.o
        60          8          0          0          0          0   __scatter.o
        28          0          0          0          0          0   __scatter_zi.o
       346          0          0          0          0         92   aeabi_sdiv.o
        16          0          0          0          0         68   exit.o
         6          0          0          0          0        136   heapauxi.o
         0          0          0          0          0          0   indicate_semi.o
         2          0          0          0          0          0   libinit.o
         2          0          0          0          0          0   libinit2.o
         2          0          0          0          0          0   libshutdown.o
         2          0          0          0          0          0   libshutdown2.o
         8          4          0          0         96         68   libspace.o
        48          0          0          0          0         72   llmul.o
       258          0          0          0          0         88   lludiv.o
         2          0          0          0          0          0   rtexit.o
        10          0          0          0          0          0   rtexit2.o
        12          4          0          0          0         60   sys_exit.o
        62          0          0          0          0         80   sys_stackheap_outer.o
         2          0          0          0          0         68   use_no_semi.o

    ----------------------------------------------------------------------
       980         16          0          0        100        800   Library Totals
         2          0          0          0          4          0   (incl. Padding)

    ----------------------------------------------------------------------

      Code (inc. data)   RO Data    RW Data    ZI Data      Debug   Library Name

       978         16          0          0         96        800   c_p.l

    ----------------------------------------------------------------------
       980         16          0          0        100        800   Library Totals

    ----------------------------------------------------------------------

==============================================================================


      Code (inc. data)   RO Data    RW Data    ZI Data      Debug   

     10860       1168       1112        472       1904     238495   Grand Totals
     10860       1168       1112         52       1904     238495   ELF Image Totals (compressed)
     10860       1168       1112         52          0          0   ROM Totals

==============================================================================

    Total RO  Size (Code + RO Data)                11972 (  11.69kB)
    Total RW  Size (RW Data + ZI Data)              2376 (   2.32kB)
    Total ROM Size (Code + RO Data + RW Data)      12024 (  11.74kB)

==============================================================================

